:020000040800F2
:1000000000000120754000089D2700089F27000878
:10001000A1270008A3270008A5270008000000006A
:10002000000000000000000000000000A7270008FA
:10003000A927000800000000AB270008AD27000832
:10004000C5400008C5400008B1270008C5400008A9
:10005000C5400008C5400008BD270008C3270008A8
:10006000C5400008C5400008EB270008C54000084F
:10007000C9270008CB270008CD270008D92700088A
:10008000E5270008E7270008C5400008C54000082C
:1000900000000000C5400008ED270008C54000082A
:1000A000C5400008C5400008C5400008C54000081C
:1000B000C5400008C5400008C5400008C54000080C
:1000C000C5400008C5400008C5400008C5400008FC
:1000D000C5400008F1270008C5400008C5400008D9
:1000E000C5400008EF270008FD270008C5400008AC
:1000F000C54000080000000000000000C5400008E6
:10010000C5400008C540000809280008C54000088F
:10011000C5400008C5400008C5400008C5400008AB
:10012000C5400008C5400008C5400008C54000089B
:08013000C5400008C5400008AD
:1001380010B5054C237833B9044B13B10448AFF319
:1001480000800123237010BD4C0100200000000036
:10015800C80E010808B5034B1BB103490348AFF3A8
:10016800008008BD0000000050010020C80E0108F2
:1001780014214160704714207047406A704700009E
:10018800790100087F01000883010008990100082F
:1001980010B5044604F1100000F05CFCC4F8F80047
:1001A8000148C4F87C0110BD88010008F8B5E6B024
:1001B80004460D4616461F460A4906A800F0CAFE20
:1001C80070996F9A05910492009733466E996D9ACB
:1001D800039102922A466C990191214600F060F839
:1001E80067B0F0BD94010008F8B5E6B004460D46C6
:1001F80016461F46094906A800F0ACFE6F996E9A8C
:100208000491039200976D996C9A0291019233467A
:100218002A46214600F087F867B0F0BD940100082F
:1002280038B500281CBF01680029184A23D1184B8B
:100238001C684FF6F0710C404CF24025AC421FBFD1
:100248001B6819404CF27024A14212D1114D296843
:1002580079B911490B68C3F30B03B3F58A6F1FBF54
:100268000968C1F30B0140F28343994204BF01219D
:10027800117028B905E0094B994204BF012111709A
:100288004068BDE8324001F09FBE00BF6801002011
:1002980000ED00E0002004E00010005C000037489A
:1002A8002DE9F04104460D46216816464A681F4666
:1002B80090478046B8F5403F2ED122680A99936846
:1002C800204698478046B8F5403F25D12368089ACC
:1002D8000799D3F80CC02046E0478046B8F5403F60
:1002E8001AD12368069A39461F692046B8478046BE
:1002F800B8F5403F10D1236829465D69324620464B
:10030800A8478046B8F5403F06D123680B9A09995B
:100318009D692046A847804621680A68204690477C
:100328004046BDE8F0812DE9F04104460D462168BC
:1003380016464A681F4690478046B8F5403F2ED17A
:1003480022680A999368204698478046B8F5403F46
:1003580025D12368089A0799D3F80CC02046E047AE
:100368008046B8F5403F1AD12368069A39461F6976
:100378002046B8478046B8F5403F10D12368294643
:100388005D6932462046A8478046B8F5403F06D109
:1003980023680999DD6900222046A847804621681C
:1003A8000A68204690474046BDE8F0814FF4403047
:1003B80070470000F0B50C4685B0114600281A4673
:1003C8001CBF0568002D0B4B11D082B104B971B95F
:1003D8000D9860B10F9E0E9F0A9B0290049603979A
:1003E8000B980C9E009001962046A8470346184695
:1003F80005B0F0BD020003002DE9F04F0646D0B06D
:100408000868F56DD6F860E0726EB76EF36E00BAE4
:1004180000906C46486800BA60600DF14008886832
:1004280000BAA060C86800BAE060086900BA206134
:10043800486900BA6061886900BAA061C86900BAF1
:10044800E061086A00BA2062486A00BA6062886A95
:1004580000BAA062C86A00BAE062086B00BA2063FA
:10046800486B00BA6063886B00BAA063C86B00BAB7
:10047800E063402058F80C1C58F820CC58F838ACE9
:100488008CEA010158F840CC8AEA01018CEA01099A
:100498004FEAF979401E48F8049BEBD187EA02003D
:1004A80000EA0E00784010EBF5610098DFF824C4EC
:1004B80041186144C81882EABE032B404FEAF06134
:1004C80053405918636859186144CF194FEAB50366
:1004D80083EABE01014081EABE0111EBF765A1681C
:1004E8004D196544A91883EAB0023A404FEAF1650C
:1004F8005A405519E26855194FEAB70282EAB0071F
:1005080065440F4005EBBE0E97EAB00717EBFE6592
:1005180027697D194FEAB10782EA0701654401EAB4
:100528000E01EB18514011EBF36561694D194FEA63
:10053800BE0187EA010E65440EEA030E15EBB00012
:100548008EEA070E0EEBF065D4F818E075446544A2
:10055800AA1881EAB30505404FEAF26E4D40AE4451
:10056800E569AE44E64477444FEAB00080EAB30E4A
:100578000EEA020E8EEAB30E0EEBF765D4F820E011
:1005880075446544691880EAB2053D404FEAF16E4A
:100598004540AE44656AAE44E6440EEBB3034FEA09
:1005A800B70787EAB20E0EEA010E8EEAB20E0EEB1C
:1005B800F365D4F828E075446544281887EAB1053E
:1005C8001D404FEAF06E7D40AE44E56AAE44E64415
:1005D8000EEBB2024FEAB30383EAB10E0EEA000E45
:1005E8008EEAB10E0EEBF265D4F830E0754465443E
:1005F800EF1983EAB00515404FEAF76E5D40AE4447
:10060800656BAE44E6440EEBB1014FEAB20282EAF2
:10061800B00E0EEA070E8EEAB00E0EEBF165D4F8B6
:1006280038E075446544EB1882EAB7050D404FEA97
:10063800F36E5540AE44E56BAE44E6440EEBB000B5
:100648004FEAB10181EAB70E0EEA030E8EEAB70E41
:100658000EEBF065D4F840E07544654481EAB30ECA
:10066800AA180EEA000E4FEAF2658EEA010E7544EA
:10067800DDF844E04FEAB000754480EAB30E654403
:100688000EEA020E15EBB7078EEAB30E0EEBF7650E
:10069800DDF848E04FEAB202754480EA020E65448C
:1006A8000EEA070E69188EEA000E0EEBF165DDF80A
:1006B8004CE07544654405EBB3034FEAB70E1427C5
:1006C8000DF1500CDFF810528EEA010B82EA0B0B89
:1006D8000BEBF36A5CF804BBDA44AA44504483EA9F
:1006E800B10B4FEAF06A8EEA0B0BDA445CF804BBF4
:1006F800DA44AA44524480EAB30B4FEAF26A8BEA1E
:10070800B10BDA445CF804BBDA444FEAB000AA44FF
:1007180080EA020BD6448BEAB30B0BEBFE6A5CF85B
:1007280004BBDA444FEAB202AA4482EA0E0B0AEB8F
:10073800B10180EA0B0B0BEBF16A5CF804BBDA44FD
:100748007F1DAA44282F0AEBB3034FEABE0EBBD382
:100758003C2F61D3502F4DD204EB870CC7F15407BF
:100768005E4CA7FB04A504465D4FA8088EEA010A63
:1007780082EA0A0A5CF804BB0AEBF3655D447D195A
:100788002C1983EAB10A4FEAF4658EEA0A0A55443D
:100798005CF804AB5CF804BB55447D19AA1884EADC
:1007A800B30A4FEAF2658AEAB10A55445D444FEA52
:1007B800B4047D1984EA020AAE448AEAB30A0AEB51
:1007C800FE655CF804AB55444FEAB2027D1982EA33
:1007D8000E0A15EBB10184EA0A0A5CF804BB0AEBBD
:1007E800F1655D447D1915EBB303401E4FEABE0E5B
:1007F800BCD12046F46D1B19F365336EC9183166F8
:10080800716E71447166B36ED218B266F16E40189B
:10081800F06650B0BDE8F08F4EEA010B0EEA010A0F
:100828000BEA020B4BEA0A0A0AEBF36554F827A015
:10083800DFF8B0C0554443EAB10B654403EAB10A96
:100848000BEA0E0B28184BEA0A0A7F1C0AEBF06524
:1008580054F827A0554440EAB30B654400EAB30AAC
:100868000BEAB10BAA184BEA0A0A7F1C0AEBF265DD
:1008780054F827A055444FEAB00040EA020B6544FB
:1008880000EA020A0BEAB30BAE444BEA0A0A7F1CE1
:100898000AEBFE6554F827A055444FEAB20242EA33
:1008A8000E0B654402EA0E0A0BEA000B15EBB101C8
:1008B8004BEA0A0A7F1C0AEBF16554F827A0554455
:1008C8007F1C65443C2F05EBB3034FEABE0EA3D350
:1008D80040E700BF9979825AA1EBD96ECDCCCCCC38
:1008E800D6C162CADCBC1B8F00B581B00168074A5B
:1008F800914200D110B9064801B000BD7C2110F02A
:1009080047FA4FF4003001B000BD00BFFC090008F1
:10091800030002002DE9F0410B4A92E8F85188B033
:10092800694681E8F8510268084B9A4200D118B923
:10093800074808B0BDE8F0811422083000F04FFBEA
:1009480008B0BDE8F08100BFDC090008FC09000818
:1009580003000200152904D20268044B9A4200D110
:1009680008B903487047083000F048BBFC09000884
:100978000300020010B481B013460268074CA2427B
:1009880000D118B901B010BC0548704701B000F19A
:10099800240210BC083000F035BB00BFFC09000879
:1009A8000300020010B481B013460268074CA2424B
:1009B80000D118B901B010BC054870470A4601B00B
:1009C80000F1240110BC083000F070BBFC090008DD
:1009D800030002000123456789ABCDEFFEDCBA981E
:1009E80076543210F0E1D2C300000000000000008D
:1009F80000000000F10800081D0900085D09000852
:100A08007D090008AD09000801040008790F0008F5
:100A1800C50F0008810F0008F0B5A3B004460B48C5
:100A280002900D4616461F46094B0822402104A88D
:100A380000F0D1FA28980190009733462A462146BB
:100A480002A800F01BF823B0F0BD00BFFC090008A5
:100A5800100A000810B5040008BF002408D0054893
:100A6800054B20600822402104F1080000F0B3FA89
:100A7800204610BDFC090008100A00082DE9F041C5
:100A880004460E46216817464A681D469047804628
:100A9800B8F5003F19D1226806999368204698470F
:100AA8008046B8F5003F10D123683146DE683A46E3
:100AB8002046B0478046B8F5003F06D12368079A1C
:100AC80029461D692046A847804621680A682046AD
:100AD80090474046BDE8F08110B500F033FA4FF476
:100AE800403400280EBF034C4FF4C07110F050F989
:100AF800204610BD0200030010B5044600F022FA9B
:100B080008B9054810BD0021A160D0F87C21116802
:100B180088474FF4403010BD0200030070B504460A
:100B28000D4600F00FFA064E40B1D0F87C0141683E
:100B38008847A84224BF65604FF44036304670BDF0
:100B4800020003002DE9FF4715000C4600D02CB128
:100B5800064600F0F7F95FEA000801D16448C3E0EF
:100B6800D8F8F80001684A689047B0F5003F17D1F7
:100B7800D8F87C118A68404690478146B9F1810FC0
:100B880080F09E80A94508F1FC0A17D2D8F8F80031
:100B98000368D3F80CC02A462146E047B0F5003F69
:100BA80040F08E80D8F8F8000368D3F810C06A4681
:100BB8005146E047B0F5003F76D10AE0002004E056
:100BC800215C0AF800100098401C00900098A84288
:100BD800F6D34FF0000C4749474A484B01AC009800
:100BE800844558D2D3E9007001ADC5E9007010788A
:100BF80000281ABF042086464FF0000E085854F803
:100C08000E5028443E4D05600127D0F800E087606B
:100C1800019D4F681AF80C007D408EEA050585F0A5
:100C2800040E65680F687D4085F0FC05754485F005
:100C3800A30568400AF80C000CF1010CCFE7D3E9D2
:100C4800004501A8C0E9004510782E4D002814BFC2
:100C58004FF0040E4FF0000E01A8744651F80EE054
:100C68000459A6440127CEF80050DEF80040CEF81B
:100C780008704D68019F40687D406C400D68684071
:100C880084F0040480F0FC00041984F057040AF886
:100C98000C400CF1010CCC45D1D3D8F8F800016810
:100CA8004A689047B0F5003F0AD1D8F8F8000368C1
:100CB800D3F80C804A465146C047B0F5003F01D0F2
:100CC800114811E0002006E05AF8201081F06A313E
:100CD8004AF82010401CB0EB990FF5D3B06840F0EB
:100CE8000100B0604FF4403004B0BDE8F08700BFA9
:100CF80002000300600F010868010020240F0008AB
:100D0800ADBE4ED70DBE75A10100030038B50C4627
:100D1800017A1546CA0702D500F014F908B908483F
:100D280032BDD0F8F80003682146DC682A46A0479F
:100D3800B0F5003F01D0034832BD4FF4403032BD1A
:100D480002000300010003002DE9F84191B00546B7
:100D58000E461746402101A810F01AF8297AC8074C
:100D680004D5284600F0EEF8040002D1DFF8A4808C
:100D78004BE0D4F8F800DFF8A0800368D3F810C07F
:100D88006A4601A9E047B0F5003F3ED1D4F8F80023
:100D980001684A689047B0F5003F36D1D4F87C1115
:100DA8008A6820469047D4F8F830024618461B68EF
:100DB800D3F80CC004F1FC01E047B0F5003F24D1A2
:100DC800D4F87C0141688847D4F8F83002461846C0
:100DD8001B68D3F80CC001A9E047B0F5003F14D157
:100DE800D4F8F8000268696893689847B0F5003F3E
:100DF8000BD1D4F8F80003681C693A463146A0477D
:100E0800B0F5003F08BF4FF44038404612B0BDE887
:100E1800F08100BF02000300010003002DE9F84142
:100E2800A5B0074688461646402115A80FF0B0FF22
:100E380000220492402105A80FF0AAFF387AC107C2
:100E48005ED5384600F07EF8050059D0D5F8F80090
:100E58002D4C0368D3F810C06A4605A9E047B0F5E1
:100E6800003F3CD1D5F8F80001684A689047B0F5D2
:100E7800003F34D1D5F87C118A6828469047D5F8C8
:100E8800F830024618461B68D3F80CC005F1FC017F
:100E9800E047B0F5003F22D1D5F87C01416888478A
:100EA800D5F8F830024618461B68D3F80CC005A9D7
:100EB800E047B0F5003F12D1D5F8F800026879682C
:100EC80093689847B0F5003F09D1D5F8F800036852
:100ED8001D6904AA15A9A847B0F5003F01D020460E
:100EE8000FE00A4B0A490B4A0396029101924046C9
:100EF8001C68049B009415AA796800F0E5F900E0E5
:100F0800054826B0BDE8F08101000300680F01081C
:100F1800936E030026C703000200030004B001011A
:100F280000170145E10A0008010B0008250B00081D
:100F3800B50300084D0B0008150D0008510D0008F9
:100F4800250E00080168024A914218BF0020704728
:100F58002C0F000810B5040008BF002404D0034873
:100F68002060204609688847204610BD2C0F0008DD
:100F780020225C300FF00ABFF0B58468A308002275
:100F880004F0030407E000F15C0555F8226035BA67
:100F980041F82250521C9A42F5D300220BE000F18E
:100FA8005C0502EB830755F82360D500C5F11805E9
:100FB800EE40CE55521CA242F1D3F0BD30B5C46804
:100FC80003690022E31AD5188C5C0544521C082AD0
:100FD8002C77F8D330BD0360C1600261704738B523
:100FE800044615460022626023685A68904700202C
:100FF8006061A061A5604FF4003032BD81604FF49C
:10100800003070472DE9F84304462079D4F80C8065
:10101800450748BF244845D466691D46A8F1010024
:1010280000EAD60306EBC506B6EBC50F666102D229
:10103800A669761CA6611746A66906EB5576A661D1
:101048000E46E918884225D2A8EB03094A463146DC
:10105800F8180FF09BFE2268136839460FE04246E5
:1010680038460FF093FE23681A68394620469047A1
:1010780007E0311811F00300F1D122681368204607
:101088009847484600EB0809A9F10101A942F0D3A5
:10109800002300E000202A1A3118F8180FF076FE15
:1010A8004FF40030BDE8F283040002002DE9FC4F44
:1010B800024685B0D0681369DFF86CC1DFF86C812F
:1010C800A0EB030A506840F004005060002703A812
:1010D80002900DF10C0ED8E9003403A8544DC0E974
:1010E80000342878534D00280CBF00230423994668
:1010F8005CF803305EF80940234401261D601C6833
:101108009E60DCF80430039DDCF80090DEF8046093
:101118005D406540484C654089EA0606474C664094
:101128007519474C6540D8E9006B03AC0028C4E941
:10113800006B0EBF002404200424029E5CF800000B
:10114800345920183F4C04600126046886600398CF
:10115800029E43406340384C7068634089EA00004F
:10116800364C6040034438484340280018BF0120EB
:101178005B1E9B41042F2CBFC0B2D80F02F1140391
:1011880053F8200007F00303C3F10303DB00D84042
:101198000DF807007F1C082F9DD315460C466A6979
:1011A800AB69E868D20842EA4372401E00EA0207C7
:1011B800002302409B420AD8524508D28020E055BD
:1011C8007F1C574516D2AAEB0701E01910E08020D2
:1011D800E05500E0E355E8687F1C8742FAD32A68A7
:1011E800136828469847BAF1000F03D051462046A5
:1011F8000FF0CEFD2A68069E059F9368694628462B
:1012080098472A68D2F8009021462846C8472B6894
:10121800DA683946284690470EB1A86830604FF41E
:10122800003007B0BDE8F08F600F010854120008C5
:10123800680100205FC5109304850012FC68017ADC
:10124800C0F524FF24AF33D426AF698B04B0010165
:1012580000170145F8B501240094002300240DE08F
:10126800009D065D0F5D7E40F643761CF60F86F006
:10127800010635400095641C009DEB189442EFD39D
:101288001846F2BDF8B5002301240094002A11E0A5
:10129800009C85188F1815F8016C17F8015C6E40D2
:1012A800F643761CF60F86F0010634400094009C45
:1012B800E318521EECD11846F2BD00005D1200087A
:1012C8008D120008010000002DE9F84F1D46DDF8D9
:1012D80028900B9F0D9C4FF0FF3300930E469246CB
:1012E800D9F800B0804632465146D847834664B3A1
:1012F800D9F8043032465146404698476FEA0B0207
:10130800521C42EA0B0200996FEAD2735B1C194027
:10131800C2430091521C024300996FEAD2735B1CCE
:101328001940009186F05531484087EA000181F064
:101338005531216080F05531C943491C0843009A52
:101348006FEAD070401C82430092D9F80800012847
:1013580009D17540E943491C0D4300986FEAD572DD
:10136800521C90430AE0F11C85EA9102D243521CB8
:10137800154300986FEAD5735B1C984386F0AA362C
:10138800009086EA0B0686F0AA33F243DB430C98FA
:10139800C2F3C0725B1C42EAD3720099D243521C5A
:1013A80091430091774000998843009987F0AA37C4
:1013B8000F403843BDE8F28F034613F8012B002A8B
:1013C800FBD1181A0138704781F0004102E000BFD4
:1013D80083F0004330B54FEA41044FEA430594EAED
:1013E800050F08BF90EA020F1FBF54EA000C55EA28
:1013F800020C7FEA645C7FEA655C00F0E2804FEAF9
:101408005454D4EB5555B8BF6D420CDD2C4480EADA
:10141800020281EA030382EA000083EA010180EA0A
:10142800020281EA0303362D88BF30BD11F0004F58
:101438004FEA01314FF4801C4CEA113102D040428E
:1014480061EB410113F0004F4FEA03334CEA1333C9
:1014580002D0524263EB430394EA050F00F0A780E1
:10146800A4F10104D5F1200E0DDB02FA0EFC22FADC
:1014780005F2801841F1000103FA0EF2801843FAD0
:1014880005F359410EE0A5F120050EF1200E012AC1
:1014980003FA0EFC28BF4CF0020C43FA05F3C018FF
:1014A80051EBE37101F0004507D54FF0000EDCF178
:1014B800000C7EEB00006EEB0101B1F5801F1BD321
:1014C800B1F5001F0CD349085FEA30004FEA3C0C25
:1014D80004F101044FEA445212F5800F80F09A801B
:1014E800BCF1004F08BF5FEA500C50F1000041EB1F
:1014F800045141EA050130BD5FEA4C0C404141EB23
:101508000101013C28BFB1F5801FE9D291F0000F1D
:1015180004BF01460020B1FA81F308BF2033A3F1CC
:101528000B03B3F120020CDA0C3208DD02F1140CC3
:10153800C2F10C0201FA0CF021FA02F10CE002F1FE
:101548001402D8BFC2F1200C01FA02F120FA0CFCF7
:10155800DCBF41EA0C019040E41AA2BF01EB045140
:10156800294330BD6FEA04041F3C1CDA0C340EDC3E
:1015780004F11404C4F1200220FA04F001FA02F381
:1015880040EA030021FA04F345EA030130BDC4F13F
:101598000C04C4F1200220FA02F001FA04F340EA34
:1015A8000300294630BD21FA04F0294630BD94F0E5
:1015B800000F83F4801306BF81F480110134013DCC
:1015C8004EE77FEA645C18BF7FEA655C29D094EA3D
:1015D800050F08BF90EA020F05D054EA000C04BFBB
:1015E8001946104630BD91EA030F1EBF00210020A6
:1015F80030BD5FEA545C05D14000494128BF41F045
:10160800004130BD14F580043CBF01F5801130BDA8
:1016180001F0004545F0FE4141F470014FF0000033
:1016280030BD7FEA645C1ABF194610467FEA655CE4
:101638001CBF0B46024650EA013406BF52EA033586
:1016480091EA030F41F4002130BD00BF90F0000F74
:1016580004BF0021704730B54FF4806404F13204B0
:101668004FF000054FF0000150E700BF90F0000F69
:1016780004BF0021704730B54FF4806404F1320490
:1016880010F0004548BF40424FF000013EE700BF60
:1016980042004FEAE2014FEA31014FEA02701FBFF0
:1016A80012F07F4393F07F4F81F06051704732F022
:1016B8007F4208BF704793F07F4F04BF41F4002179
:1016C800704730B54FF4607401F0004521F00041D7
:1016D8001CE700BF50EA010208BF704730B54FF061
:1016E80000050AE050EA010208BF704730B511F062
:1016F800004502D5404261EB41014FF4806404F19A
:1017080032045FEA915C3FF4D8AE4FF003025FEA1F
:10171800DC0C18BF03325FEADC0C18BF033202EBA3
:10172800DC02C2F1200300FA03FC20FA02F001FAFD
:1017380003FE40EA0E0021FA02F11444BDE600BFA0
:101748004FF0FF3C06E000BF4FF0010C02E000BF85
:101758004FF0010C4DF804CD4FEA410C7FEA6C5C68
:101768004FEA430C18BF7FEA6C5C1BD001B050EA0B
:10177800410C0CBF52EA430C91EA030F02BF90EAF6
:10178800020F0020704710F1000F91EA030F58BFB5
:10179800994208BF90422CBFD8176FEAE37040F017
:1017A800010070474FEA410C7FEA6C5C02D150EAB5
:1017B800013C07D14FEA430C7FEA6C5CD6D152EA70
:1017C800033CD3D05DF8040B704700BF8446104635
:1017D80062468C461946634600E000BF01B5FFF734
:1017E800B7FF002848BF10F1000F01BD4DF808ED04
:1017F800FFF7F4FF0CBF012000205DF808FB00BFD5
:101808004DF808EDFFF7EAFF34BF012000205DF82E
:1018180008FB00BF4DF808EDFFF7E0FF94BF01207B
:1018280000205DF808FB00BF4DF808EDFFF7CEFF7C
:1018380094BF012000205DF808FB00BF4DF808EDBB
:10184800FFF7C4FF34BF012000205DF808FB00BF8C
:101858004FEA410212F5001215D211D56FF47873D0
:10186800B3EB625212D94FEAC12343F0004343EA73
:10187800505311F0004F23FA02F018BF404270474E
:101888004FF00000704750EA013005D111F00040D8
:1018980008BF6FF0004070474FF00000704700BF6E
:1018A80080F0004002E000BF81F0004142001FBF0D
:1018B8005FEA410392EA030F7FEA226C7FEA236C16
:1018C8006AD04FEA1262D2EB1363C1BFD21841400B
:1018D80048404140B8BF5B42192B88BF704710F0A1
:1018E800004F40F4000020F07F4018BF404211F044
:1018F800004F41F4000121F07F4118BF494292EAAC
:10190800030F3FD0A2F1010241FA03FC10EB0C00D7
:10191800C3F1200301FA03F100F0004302D5494264
:1019280060EB4000B0F5000F13D3B0F1807F06D311
:1019380040084FEA310102F10102FE2A51D2B1F109
:10194800004F40EBC25008BF20F0010040EA0300FE
:101958007047490040EB0000013A28BFB0F5000F7E
:10196800EDD2B0FA80FCACF1080CB2EB0C0200FA34
:101978000CF0AABF00EBC25052421843BCBFD04083
:101988001843704792F0000F81F4000106BF80F4FD
:1019980000000132013BB5E74FEA41037FEA226CC0
:1019A80018BF7FEA236C21D092EA030F04D092F08B
:1019B800000F08BF0846704790EA010F1CBF0020BF
:1019C800704712F07F4F04D1400028BF40F000401C
:1019D800704712F100723CBF00F50000704700F03C
:1019E800004343F0FE4040F4000070477FEA226263
:1019F80016BF08467FEA23630146420206BF5FEA34
:101A0800412390EA010F40F4800070474FF0000333
:101A180004E000BF10F0004348BF40425FEA000CFA
:101A280008BF704743F0964301464FF000001CE0A2
:101A380050EA010208BF70474FF000030AE000BFF8
:101A480050EA010208BF704711F0004302D5404236
:101A580061EB41015FEA010C02BF844601460020A8
:101A680043F0B64308BFA3F18053A3F50003BCFAC3
:101A78008CF2083AA3EBC25310DB01FA02FC634470
:101A880000FA02FCC2F12002BCF1004F20FA02F277
:101A980043EB020008BF20F00100704702F120026A
:101AA80001FA02FCC2F1200250EA4C0021FA02F2CB
:101AB80043EB020008BF20EADC7070474FEA40029F
:101AC800B2F1FE4F0FD34FF09E03B3EB12620DD964
:101AD8004FEA002343F0004310F0004F23FA02F0CE
:101AE80018BF404270474FF00000704712F1610F75
:101AF80001D1420205D110F0004008BF6FF000404C
:101B080070474FF00000704753B94AB9002908BF21
:101B180000281CBF4FF0FF314FF0FF3000F070B9C4
:101B2800ADF1080C6DE904CE00F006F8DDF804E02C
:101B3800DDE9022304B070472DE9F047089E0D4601
:101B480004460F46002B4AD18A42944665D9B2FA18
:101B580082F343B102FA03FCC3F120029F4020FA4A
:101B680002F217439C404FEA1C4E1FFA8CF5B7FB54
:101B7800FEF1220C0EFB117742EA074201FB05F049
:101B880090420AD91CEB020201F1FF3780F01B8159
:101B9800904240F2188102396244121AA4B2B2FB90
:101BA800FEF00EFB102244EA024400FB05F5A542B4
:101BB8000AD91CEB040400F1FF3280F00681A5422B
:101BC80040F203816444023840EA0140641B00216A
:101BD8001EB1DC400023C6E90043BDE8F0878B4214
:101BE80008D9002E00F0EC800021C6E9000508465F
:101BF800BDE8F087B3FA83F1002949D1AB4202D39B
:101C0800824200F2F780841A65EB0302012017462E
:101C1800002EE2D0C6E90047DFE702B9FFDEB2FADC
:101C280082F3002B40F08F808A1A4FEA1C471FFA74
:101C38008CFE0121B2FBF7F507FB1520220C42EAC6
:101C480000420EFB05F0904208D91CEB020205F198
:101C5800FF3802D2904200F2CA804546121AA4B256
:101C6800B2FBF7F007FB102244EA02440EFB00FE29
:101C7800A64508D91CEB040400F1FF3202D2A645A0
:101C880000F2BA801046A4EB0E0440EA05409FE734
:101C9800C1F120078B4022FA07FC4CEA030C05FA35
:101CA80001F420FA07F3FD40234300FA01F94FEA53
:101CB8001C401FFA8CFEB5FBF0F81C0C00FB1855F5
:101CC80044EA054408FB0EF5A54202FA01F20BD9D5
:101CD8001CEB040408F1FF3A80F08780A54240F22B
:101CE8008480A8F102086444641B9DB2B4FBF0F33D
:101CF80000FB134445EA044403FB0EFEA64508D93D
:101D08001CEB040403F1FF306BD2A64569D9023BF2
:101D1800644443EA0840A0FB0283A4EB0E049C42FF
:101D2800C6461D4655D352D056B1B9EB0E0364EBE7
:101D3800050404FA07F7CB40CC401F43C6E90074FA
:101D48000021BDE8F087C3F1200102FA03FC20FA64
:101D580001F225FA01F19D402A434FEA1C471FFA78
:101D68008CFEB1FBF7F007FB1015110C41EA054199
:101D780000FB0EF58D4204FA03F408D91CEB0101AF
:101D880000F1FF382FD28D422DD902386144491B0A
:101D980092B2B1FBF7F507FB151142EA014205FBC8
:101DA8000EF1914208D91CEB020205F1FF3816D258
:101DB800914214D9023D6244521A45EA004139E77A
:101DC8003146304609E73946E7E61046FCE6C145A4
:101DD800AAD2B8EB020E63EB0C050138A4E745461E
:101DE800EAE7034695E74046D1E7D0467CE7023D5F
:101DF800624433E708460BE76444023843E700BF10
:101E0800704700BF1348144A08B54FF00043C0E9B3
:101E180000230422002342610122C2614FF4805151
:101E280007220383C0E90233C0E90933C0E90C1271
:101E38000361837680F8203080F82C30826380F844
:101E48003C30C36402F090F918B1BDE8084000F0D6
:101E5800FDBB08BD6C010020002401400268084B4E
:101E68009A4282B00AD14FF0B0431A6E42F400721F
:101E78001A661B6E03F400730193019B02B070474E
:101E8800002401400268054B9A4201BF4FF0B0425E
:101E9800136E23F400731366704700BF00240140DB
:101EA80030B585B000240546CDE901440394FFF719
:101EB800A9FF144802F0F0FC08B100F0C7FB114874
:101EC800039401A9CDE9015402F0ACFA08B100F07D
:101ED800BDFB0C4802F00AFC08B100F0B7FB4FF05C
:101EE800FF31084802F040FA064802F0B7FC0548FE
:101EF80002F094FA0446034802F05AFC204605B062
:101F080030BD00BF6C010020014B024A1A607047C7
:101F18006C0100200024014008B50948FFF7C0FF04
:101F280068B1084BB3F8AA304FF6FF72934216BF58
:101F380040F6E442044B5343B3FBF0F398B208BDB8
:101F4800002000B40075FF1FD8084C0013B500230B
:101F5800ADF80630FFF7E0FF04461948FFF7A0FF89
:101F6800184BB3F8C820B3F8A8108A4204FB00F055
:101F780018D040F6E443B0FBF3F364205B1A434304
:101F8800521A93FBF2F31E331BB2ADF80630BDF8BC
:101F980006305BB21B02ADF80630BDF8060000B291
:101FA80002B010BD4FF47A7240F6FF73B0FBF3F342
:101FB8005343A3F53923A3F50C6340F6C412E0E7B5
:101FC800001000B00075FF1F4FF0B04382B09A6A4E
:101FD80022F480529A629A6C42F480529A649B6C02
:101FE80003F480530193019B002002B070474FF027
:101FF800B04382B09A6C02439A649B6C034001938D
:10200800019B02B0704708B50420FFF7F0FF0120DC
:10201800FFF7EDFF0220FFF7EAFF002211460B2031
:1020280002F0D8FC0B2002F007FD002211460C201C
:1020380002F0D0FC0C2002F0FFFC002211460D201B
:1020480002F0C8FC0D2002F0F7FC002211460E2019
:1020580002F0C0FC0E2002F0EFFC002211460F2017
:1020680002F0B8FC0F2002F0E7FC00221146112014
:1020780002F0B0FC112002F0DFFC002236201146ED
:1020880002F0A8FCBDE80840362002F0D5BC0000EC
:1020980008B502F019FF10B16FF0040008BD064B37
:1020A8009A6942F040429A614CF2FA321A6102F09F
:1020B8001DFF0028F2D0EFE700400058F0B585B0CA
:1020C80000230C4600930646A8B3FFF7E1FF054638
:1020D80070BB02F0F9FE88BB1A481B4A0223019321
:1020E800D0F8E01506F1784302EA8121B3FBF1F755
:1020F80001FB1733DB0A0293D0F8E00504F17841BD
:102108000139314402EA8022B1FBF2F002FB1011DE
:10211800C3EBD1230133694601A8039302F066FF9C
:1021280020B102280CBF01256FF0010502F0DEFE88
:10213800284605B0F0BD6FF00505F9E76FF0040516
:10214800F6E700BF0070FF1F00FCFF03014B18609B
:1021580000207047D00100202DE9F04F89B0B0F180
:10216800006F06460F460092C0F0C580DFF89881E0
:10217800664DD8F8E03505EA832303F10063013B97
:10218800984200F2B880002800F0B880002900F0DA
:10219800B58040EA02035B0740F0B080FFF778FFA4
:1021A8000446A0BB02F090FE002840F0AA80D8F8B0
:1021B800E01506F1784205EA8121B2FBF1F301FB53
:1021C8001322009B03F17843013B3344B3FBF1F046
:1021D80001FB1033DB0A01334FEAD22AA3EBD222E8
:1021E800012A039388BFC6F30A050AF58038C6F1A9
:1021F800080398BF009D069388BFC5F500654FEAA0
:10220800C828B346039B9A4505D302F06FFE2046C3
:1022180009B0BDE8F08FA6F10803069A1A44954262
:1022280019D804950197CDF814B04FF00009059B13
:1022380009EB0301049B99453ED3009BAB442F4413
:102248005D1BB5F5006F28BF4FF400650AF1010A60
:1022580008F50068D6E753F8081F5A68B2F1FF3F3F
:1022680008BFB1F1FF3FD8D0294B186810B96FF0FB
:102278000504CAE7B8F1000F04D04FF400624146E4
:102288000EF020F9DFF88890D9F80030CBF30A0077
:1022980039461844AAB20EF015F94FF400614046C9
:1022A800FFF70CFF08BBD9F8003001934FF4006327
:1022B800CDF814800493B8E7019B07914B4402932F
:1022C8000120D3E9002302F04BFE88B90799019B4E
:1022D800D1E9000259F80310029B5B689A4208BFD3
:1022E800884205D109F10809A1E76FF001048CE7DC
:1022F8006FF0030489E74FF0FF3488E76FF00504B7
:1023080085E76FF0040482E70070FF1F00FCFF03FD
:10231800D0010020B1F1006F70B511D30B4BD3F889
:10232800E0650B4B03EA862303F10063013B994206
:1023380006D840B139B192B20EF0C4F8002070BD91
:102348004FF0FF30FBE76FF00500F8E70070FF1F64
:1023580000FCFF03B0F1006F10B40DD3084BD3F8A5
:10236800E045084B03EA842303F10063013B9842EC
:1023780002D810BCFFF7A2BE4FF0FF3010BC704768
:102388000070FF1F00FCFF034FF0B04382B0DA6C0F
:102398000243DA64DB6C03400193019B02B070478F
:1023A80070B5012086B00024CDE90444FFF7ECFFA6
:1023B8000220FFF7E9FF0420FFF7E6FF01250222CC
:1023C8000DEB00014FF404134FF09040CDE90123C9
:1023D800204E039502F058FE4FF4441301A94FF024
:1023E8009040CDE90235019502F04EFE04230DEB35
:1023F80003013046CDE90135CDE9034402F044FE3E
:1024080022463046082102F065FF4FF4806301A997
:102418004FF09040CDE90134039402F035FE0823D3
:1024280001A93046CDE90135CDE9034402F02CFE7F
:1024380022462146062002F0CDFA062002F0FCFAD8
:1024480022462146072002F0C5FA072002F0F4FAD6
:1024580006B070BD0004004808B51248124A134B74
:10246800C0E9002300230122C0E90232C0E9043395
:10247800C0E90633036202F03FFF08B100F0E6F856
:102488000848002102F089FF08B100F0DFF805488C
:10249800002102F0A8FF18B1BDE8084000F0D6B846
:1024A80008BD00BF94020020005800405D3E302067
:1024B80070B596B005461422002103A80EF03AFC28
:1024C8003822002108A80EF035FC2A68304B9A42C1
:1024D8005BD18023089308A84FF440230E9303F0A0
:1024E800DDFC08B100F0B2F84FF0B0444FF4C05032
:1024F800E36C43F00103E364E36C03F0010302932C
:10250800029B12230026CDE903030323CDE90563CB
:102518004FF09040042303A9079302F0B5FDA36D83
:10252800DFF870C043F48003A365A36D1A4C03F46D
:1025380080030193019B26620D23C4E900C3204652
:102548008023C4E90266C4E90436C4E9066602F0D9
:10255800D3FA08B100F07AF8104AEC63A562104C7F
:102568000E23C4E900231021002380222046C4E959
:102578000213C4E90423C4E90633236202F0BCFA57
:1025880008B100F063F8AC63A56216B070BD00BF77
:102598000058004044000240D40100205800024086
:1025A8003402002000B59BB04822002108A80EF094
:1025B800C1FB1822002102A80EF0BCFB02F038FF74
:1025C8004FF0B0420120D2F8903023F01803C2F83F
:1025D8009030D2F8003423F4C06343F40073C2F897
:1025E8000034D2F8003403F4C0630193019B242320
:1025F800089381230B930023CDE91003B02208A888
:10260800CDE9122303F08CF808B172B6FEE74F2328
:10261800CDE90230CDE90400CDE90600022102A887
:1026280003F018FB08B172B6FEE71BB05DF804FBB7
:1026380008B501F047FDFFF7B5FFFFF7B1FEFFF75B
:10264800E2FC00F0A0FD00F0A5FDFCE772B6FEE795
:1026580000B58DB02C22002101A80EF06BFB1748A5
:10266800174B03601F2383604FF080420023C0E9AB
:102678000433C0E9072383614FF48073436203F096
:1026880093FD08B1FFF7E2FF0C4803F0B9FE08B16B
:10269800FFF7DCFF4FF0005300220793074808922A
:1026A8004FF4807301A9029206920B9303F0DCFDAC
:1026B80008B1FFF7CBFF0DB05DF804FBE80200207E
:1026C8000028004010B5044690B03822002102A826
:1026D8000EF030FB2268194B9A422CD14FF480330C
:1026E800029302A84FF480730F9303F0D7FB08B14D
:1026F800FFF7ACFF4FF0B0430220D3F8902042F42C
:102708000042C3F890209A6D42F480629A659B6DEE
:10271800002203F4806311460193019B02F05AF9E9
:10272800022002F089F900222A20114602F052F90B
:102738002A2002F081F910B010BD00BF0028004027
:102748007047000008B501F0D3FC044B0120C3F822
:102758008800BDE8084002F0C3BE00BF000400586E
:1027680001F0CDBC08B501F0CAFC00F033FCFFF75E
:1027780017FEFFF748FCBDE80840FFF76DBE08B537
:1027880001F0B6FCBDE808400121002002F058BE67
:1027980070477047FEE7FEE7FEE7FEE7FEE7704793
:1027A8007047704770470000014803F04FBE00BFF4
:1027B800E8020020012002F093BD022002F090BD43
:1027C80070477047014802F011BB00BFD4010020D8
:1027D800014802F00BBB00BF600300207047FFF701
:1027E800F7BF704770477047014804F0F3B900BF5E
:1027F800C0030020014803F05BBC00BFE8020020D2
:10280800014804F04EB800BF4C0300202DE9F04306
:1028180089B080460020109E0790894615461F46BD
:10282800FDF7FEFCF0B9104CCDE90090CDE90204AB
:1028380007AB0E480593142304933A4643462946AA
:102848000068FDF7B7FD2346324604F1140153F83A
:10285800044B42F8044B8B42F9D1079B337509B0FE
:10286800BDE8F0830120FAE7200300205C0F01088F
:102878001FB50E4C00233C2202A8CDE90233627535
:10288800237500F0BBF8042303AA0094122108481A
:10289800FFF7BCFF0749142220460EF03BFAB0FAB6
:1028A80080F35B09637504B010BD00BF34030020DA
:1028B800840F01087E060020054808B50823036038
:1028C80003F00AFE18B1BDE80840FFF7BFBE08BD17
:1028D8004C0300204FF0B04307B55A6E42F0010296
:1028E8005A665B6E002203F0010301931146322001
:1028F800019B02F06FF8322003B05DF804EB02F0A0
:102908009BB800000CB407B5054A05AB102101932C
:102918000EF0E2F803B05DF804EB02B0704700BFB8
:10292800960F010830B585B0044602A80D460DF093
:10293800FFFEBDF90C30064A00931021029B204689
:10294800FFF7E0FF2046FEF737FD288005B030BDD1
:10295800960F01084FF0B04210B5936823F4004376
:1029680093600DF06DFF0F4B01241C7000F0B8F858
:102978000DF036FC0C480DF04DFC0C4B4FF40042AA
:102988001A6100200DF04CFCFFF7BEFA00F014F9B4
:1029980000F0ECFB0DF040FD21462046BDE810405C
:1029A8000DF05ABD580300202D290008004000589A
:1029B8000DF068BD08B5FFF7AFFA40F6B833984296
:1029C8000CD8B0F5E16F0BD3FE23A0F5E1605843B6
:1029D8004FF49663B0FBF3F0C0B208BDFE20FCE7ED
:1029E8000020FAE77FB5684600F0CAF80198FFF7BB
:1029F80065F800B207B05DF804FB0000194A38B565
:102A0800D2F88035591C044619D101F07FFB0546E0
:102A180001F088FB054401F07FFB2B0EE3712B0CC2
:102A2800A3712B0A6371030EE370C0F30742C0F36E
:102A380007232571C0B2A2706370207038BD190ACF
:102A4800C3718171190C1B0E41710371D2F8843561
:102A5800C370D2F88405C0F30722C0F30743000E01
:102A6800E9E700BF0070FF1F38B5094BD3F8803580
:102A780003600133054609D101F048FB044601F023
:102A88004BFB444001F04EFB44402C6038BD00BF76
:102A98000070FF1F012102200DF0C8BC0021022098
:102AA8000DF0C4BC00207047024B187808B100F044
:102AB800BBB870475803002082B00190019802B05B
:102AC80000F04EB94FF0B04382B0DA6C42F0020227
:102AD800DA64DB6C03F002030193019B02B07047D8
:102AE8002DE9F043254C87B001F022FB01F028FBCB
:102AF80001F02EFB0123002502934FF48059032394
:102B080001A9204604934FF4005803950595FFF753
:102B1800D9FFFFF7D7FFFFF7D5FFFFF7D3FFCDF8B2
:102B2800049002F0B1FA01A920464FF40067CDF8ED
:102B3800048002F0A9FA01A920464FF40046019743
:102B480002F0A2FA01A92046019602F09DFA2A464F
:102B58004946204602F0BEFB2A464146204602F07E
:102B6800B9FB2A463946204602F0B4FB2A463146CC
:102B7800204602F0AFFB07B0BDE8F0830004004830
:102B880010B50446FFF7E2F9074BA36040F30F20A6
:102B9800FEF740FF054B064A2360064B6060C4E918
:102BA8000323002010BD00BF0000484200007A4403
:102BB8000D093E00AB03050000207047014B186863
:102BC800704700BF5C0300200320704708B501462A
:102BD8004FF47A7200238002890DFEF795FF08BD35
:102BE8004FF47A73A0FB0303800A40EA83507047CE
:102BF800034B98689A689042FBD1C043704700BF66
:102C08000028004008B5FFF7F3FF014B186008BD26
:102C18005C03002008B5FFF7EBFF024B1B68C01AE6
:102C280008BD00BF5C030020024B187808B1FFF70D
:102C3800DFBF70475903002010B5074B074C01222E
:102C4800DA654FF48071204603F0F8F94FF0FF334E
:102C58002363002010BD00BF00280040E8020020C8
:102C680002460021014803F002BC00BFE802002030
:102C780002460121014803F0FABB00BFE802002028
:102C880010B58CB02C220021044601A80EF052F891
:102C9800FFF7D2FF0C4B0D481B681C440023089318
:102CA80006934FF00053E443079301224FF48073D7
:102CB80001A902940B9303F0D7FA08B1FFF7C6FCF9
:102CC80000200CB010BD00BF5C030020E80200200B
:102CD80038B50546FFF78CFF02210446074803F084
:102CE800CDFBC4F309024FF47A71A2FB0121920AC9
:102CF800A30A2A8043EA805038BD00BFE8020020BA
:102D08000148002103F0BABBE80200200148012174
:102D180003F0B4BBE8020020F8B50F4D2E78CEB909
:102D28000E4C4FF0FF372763FFF792FCFFF784FF45
:102D38004FF48071204603F081F92046276303F0A1
:102D480041FB32462046022103F091FBFFF75AFF70
:102D580001232B700020F8BD59030020E802002051
:102D6800014610B54FF47A7200238002890DFEF7F0
:102D7800CBFE0146FFF73CFF0446FFF739FF031B74
:102D88008B4200D310BD00BFF7E70DF061BE000015
:102D980010B5064C0221204603F070FB0221421CAC
:102DA8002046BDE8104003F062BB00BFE8020020E7
:102DB8001648174A08B54FF4E133C0E90023002349
:102DC8000C22C0E90233C0E90523C0E90733C0E992
:102DD8000933036104F0DFFC08B1FFF737FC0B4847
:102DE800002104F054FE08B1FFF730FC0748002129
:102DF80004F06DFE08B1FFF729FC044804F027FE33
:102E080018B1BDE80840FFF721BC08BDC003002089
:102E18000044004070B596B006461422002103A86D
:102E28000DF088FF3822002108A80DF083FF3268D2
:102E3800274B9A424AD10223089308A8254B0A93A4
:102E480003F02CF808B1FFF701FC4FF0B043002560
:102E58009A6D214C42F400329A659A6D02F4003260
:102E68000292029ADA6C42F00102DA64DB6C03F037
:102E780001030193019B0C220223CDE903230323C1
:102E8800CDE9055303A907234FF09040079302F0BB
:102E9800FBF8124925621423C4E900131023C4E97E
:102EA800023520468023C4E90435C4E9065501F0FB
:102EB80023FE08B1FFF7CAFB2520F4670022022190
:102EC800A66201F087FD252001F0B6FD16B070BDA1
:102ED8000044004004000C00600300208000024011
:102EE80002680C4B9A4210B5044612D14FF0B0421A
:102EF8000C21936D23F4003393654FF0904002F05A
:102F08006FF9E06F01F06CFEBDE81040252001F07C
:102F1800A1BD10BD0044004008B50A46014602485C
:102F280003F0BCFD002008BDC003002013B5114B01
:102F3800114C18604FF40013009302AB13E906001C
:102F4800204604F028FD2368DA69D103FCD4DA6945
:102F58005202FCD59A68084842F480029A6004F04C
:102F680060FD06490448012204F0CEFC002002B0AE
:102F780010BD00BF54040020C00300205C040020E2
:102F880008B5074B1860FFF73EF8FFF711FF054A31
:102F9800D2F8803043F00063C2F88030002008BDCA
:102FA800580400200008005808B54FF0B0430848FE
:102FB8009A6B42F400329A639A6B22F400329A6355
:102FC800FFF78EFF0F2001F045FD002008BD00BF70
:102FD800C003002008B5074804F0DDFB08B1FFF77F
:102FE80035FB054801F088FD18B1BDE80840FFF73A
:102FF8002DBB08BDC0030020600300200268044BFD
:103008009A4203D1034B00201B681847704700BF42
:10301800004400405804002002680B4B9A4210B547
:1030280004460FD1094B1B682BB1D0F8902012B978
:1030380007480121984720460549BDE8104001226C
:1030480004F062BC10BD00BF0044004054040020DE
:103058005C04002010B50A4C23780BB9E37C6BB1F3
:10306800FFF706FC0038074B18BF01204000187016
:103078001B78022B02BF00232370E37410BD00BF2E
:103088007E0600207004002038B5114C2378F3B96F
:10309800E37CE3B90F4D2B68012B07D92B68042B70
:1030A80004D80D4A0421012000F02EFA2B68042BC5
:1030B8000DD9FFF7DDFB0038084B18BF0120400091
:1030C80018701B78022B02BF00232370E37438BDED
:1030D8007E0600206C040020F00F01087004002018
:1030E80038B50C4D0C4C01220821284602F0F2F8A4
:1030F8004FF47A70FFF7E0FC4FF480614FF0904096
:1031080002F0E2F8002220700821284602F0E2F8D6
:10311800237838BD000400487104002070477047C8
:10312800022808B50ED801221021074802F0D2F86B
:103138003220FFF7C1FCBDE80840034800221021F7
:1031480002F0C8B808BD00BF00040048054B1B7852
:10315800B3FA83F35B09037100234371024B012225
:103168001A707047710400207D060020034A00236E
:1031780013715371024A1370704700BF5E04002038
:103188007D060020704708B5FFF7E4FBBDE808405E
:1031980000F058BB4FF0FF300DF0D8B970477047BA
:1031A800014BD870704700BF5C000020014B1874B9
:1031B800704700BF5C00002020B1037813B10248BB
:1031C8000DF0F4BB704700BFB405002008B502201D
:1031D80000210DF083F9BDE8084001480DF0E6BB79
:1031E800CC050020002101200DF078B910B5094C5C
:1031F80060B1206008480DF08BFB216806480DF08F
:103208000FFCBDE8104004480DF0D0BB42F210732B
:103218002360EFE774000020CC05002010B5094CAE
:10322800206023680BB9084B236008480DF070FB39
:10323800216806480DF0F4FBBDE8104003480DF086
:10324800B5BB00BF0C000020A0860100E4050020EB
:1032580010B5044680B190F906306BB909480DF0F5
:1032680057FB094BE2791A70084B1868FFF7D6FF2D
:10327800074B1868FFF7BAFFBDE81040002102208D
:103288000DF02CB968050020980500200C000020DE
:103298007400002038B504460D4607484FF4006115
:1032A800FFF758F830B92A4621460348BDE83840A8
:1032B800FEF752BF38BD00BF00F003080A460149B7
:1032C800FFF728B800F0030838B50C480DF020FBCC
:1032D80005F062F860B90A4C0A480125257004F027
:1032E800EDFE2078294604F03FFC04480DF05EFB13
:1032F800BDE8384004480DF059BB00BFCC0500209C
:10330800000000205C0000209C05002005F0E0B8CB
:1033180030B585B0FFF74EFB044604F01BFD0546AB
:1033280080B100243B480DF0F3FA3B4B394819684B
:10333800A14238BF21460DF073FB36480DF036FB2D
:1033480005B030BD01464FF480600DF0C7F86846FF
:10335800FFF7FCFE23B203EB4303FE2203EB431308
:10336800B3FBF2F32D4A072111702D490878DBB21F
:103378008DF80C3038B30D70082111702949506848
:10338800097861F07F01017051684B700221264B6A
:10339800264C1B78012B637A88BF0021517033B10A
:1033A80004F0C4FC012802D120460DF0B1FA204BEC
:1033B8001A48D978002204F0E3FC0630B1D104F0B1
:1033C800AFFC0446AEE71B481B4C017821B92578B1
:1033D80005F0FF01002DDAD000212170114C017099
:1033E800506824780470506841705168562088707D
:1033F80051680120C87051680B71536802215971D6
:1034080053689DF80510997153689DF80410D97197
:103418000821BCE7CC05002074000020040000202F
:10342800FC050020640500207004002068050020C9
:103438005C000020930600207D06002008B5104B94
:103448000122002102201A700DF048F80D480DF0F5
:10345800ADFA0D4B1B788BB10C4B1A7872B9DB7C2B
:1034680063B90B4B1A68042A9EBF1A6801321A60A6
:103478000021BDE8084010200DF030B808BD00BF9D
:10348800FC050020E4050020980500207E060020A9
:103498006C040020044B1B78022B03D10021082068
:1034A8000DF01CB8704700BF0000002008B504F0FC
:1034B8007CFF80B904F03AFC01280CD1BFF34F8F90
:1034C8000549064BCA6802F4E0621343CB60BFF3B8
:1034D8004F8F00BFFDE708BD00ED00E00400FA05CE
:1034E80070477047704770477047012808B50AD180
:1034F80000214FF480600CF0F1FFBDE80840002186
:1035080002200CF0EBBF08BD70B505460C46164608
:1035180004F020FC0346002834D000241A480DF09B
:10352800F7F91A4B18481968A14238BF21460DF01F
:1035380077FABDE8704014480DF038BA4A68F05C74
:10354800D0540133DAB29442F8D8114B0D701B787D
:10355800012B88BF00244C700E4C637A33B104F001
:10356800E5FB012802D120460DF0D2F90A4B0B48A1
:10357800D978002204F004FC0630CED104F0D0FB48
:103588000446CBE70549DDE7CC05002074000020A0
:1035980070040020680500205C0000200400002062
:1035A800044B1B7823B9044A05210120FFF7ACBF5F
:1035B800704700BF70040020F50F010810B5002403
:1035C80090B03C22214601A800940DF0B3FB2F4B8C
:1035D8002022DA7219788DF8001059788DF80110C8
:1035E80099788DF80210D9788DF8031019798DF82B
:1035F800041059798DF8051099798DF80610D97944
:103608008DF80710197A8DF80810597A8DF8091075
:10361800997A8DF80A108DF80B2021460DF10B02CE
:1036280058180131007B02F8010F1C29F8D193F8D2
:1036380028208DF8282093F829208DF8292093F840
:103648002A208DF82A2093F82B208DF82B2093F828
:103658002C206AB193F83F2052B10DF12B010022C2
:103668009818013290F82C0001F8010F142AF7D1AC
:1036780007484FF40061FEF76DFE20B90448402268
:103688006946FEF769FD10B010BD00BF7800002044
:1036980000F80308014940220CF014BF00F80308A1
:1036A80070B52A4D28796B794D2BC0B233D1C0EB58
:1036B800001080000A2838BF0A204FF47A73584354
:1036C800234BAC791860EB794D2BE4B22BD1C4EBCA
:1036D8000414A40095F82C301E4E63BB95F83F30B7
:1036E8004BBB42F21070FFF781FD3068FFF796FD83
:1036F8002B7A194A1949DBB213706B7A184ADBB274
:1037080013700023EA1892F82C20D2B2CA5401335D
:10371800142BF7D170BD6B79482B0ABF4FF4616346
:103728006B795843C6E7EB79482B0ABF4FF46163BE
:10373800EB795C43CEE7FFF759FD012C38BF012434
:103748004FF47A735C433460CFE700BF7800002001
:10375800740000200C000020920600207E06002045
:103768007004002010B590B000213C2201A80091FF
:103778000DF0E0FA4022314968460CF0A3FE9DF8AE
:1037880000203AB99DF80100562803D19DF802108F
:10379800012909D0FFF712FF4FF47A70FFF78CF96F
:1037A800FFF77EFF10B010BD254B1A705870997046
:1037B8009DF80310D9709DF8041019719DF8051033
:1037C80059719DF8061099719DF80710D9719DF8E7
:1037D800081019729DF8091059729DF80A1099720B
:1037E8009DF80B1001F03F01D972D87AD1B2884206
:1037F8001BD89DF8282083F828209DF8292083F8D5
:1038080029209DF82A2083F82A209DF82B2083F868
:103818002B200DF12B0100229818013211F8014FCD
:1038280080F82C40142AF7D1BAE701F14000684427
:10383800194410F8340C08730132D6E700F803086D
:10384800780000201FB5002403A92046039404F043
:103858008FFD03A9012004F08BFD384B38480094F4
:1038680022464FF4FA710CF0F5FF364B36480094B7
:1038780022464FF4FA710CF0EDFF344B34480094B3
:1038880001224FF4FA710CF0E5FF2046FEF75EFCCA
:1038980008B1FEF7DBFE2F4B009400224FF4FA61CB
:1038A8002D480CF0D7FF2D4A002101200CF0D2FE44
:1038B8002B4A002102200CF0CDFE2A4A00210420C8
:1038C8000CF0C8FE284A002108200CF0C3FE00F0C6
:1038D80051FB2649264804F001FD264804F0EEFB7A
:1038E8001B480DF063F8244B0021187804F03CF9CC
:1038F80022490094224B0968224800220CF0AAFFB2
:1039080020480DF053F8FFF72DFF1F4A0021102023
:103918000CF0A0FE1D4A00214FF480600CF09AFEC6
:103928001B4B1C4819681C4B009400220CF092FF9A
:1039380018480DF03BF804B010BD00BFED34000886
:10394800B4050020EF34000880050020E9340008A1
:10395800680500209D3400089C050020BD7E0008F5
:103968001933000815330008D1320008000003019C
:10397800100000205C0000200000002074000020DF
:10398800D5310008CC05002091300008E930000846
:103998000C000020E40500204534000830B5002460
:1039A800A3B07C22214603A802940DF0C3F9532347
:1039B8008DF808304FF4AB73ADF80A3001238DF859
:1039C8000C30ADF80440FEF7F5FF00B200EB400004
:1039D80000EB4010FE23B0FBF3F08DF80D0001A8BA
:1039E80000F06DFBC0B143000133DBB20B4C8DF826
:1039F8000E302C228021201D1D460DF09BF90298C7
:103A0800BDF80C302060A380A57122460721012053
:103A1800FFF77AFD23B030BD5823E7E7FD05002006
:103A280070B50378592B90B0044640F0BE81052943
:103A380059D84378443B162B55D8DFE813F00E01CC
:103A48005400FE0054000601540054005400540071
:103A580073005400E90054005400540075015400E8
:103A680054008F0054005400540017008578482DE6
:103A780011D1A54A14210120FFF746FD41F28830F3
:103A8800FFF71AF840F6B830FFF716F810B0BDE89F
:103A98007040FFF70BBD532D0ED1302280219B487B
:103AA8000DF048F9FFF77AFF41F28830FFF704F884
:103AB800964A1521012063E0432D16D1002468465B
:103AC8008DF8004004F072FA904A4C231370562384
:103AD80093709DF80030547001204133D0701371F9
:103AE8000521FFF711FD10B070BD442DFBD1874CA7
:103AF8002C228021201D0DF01DF9002325706370F4
:103B080001255623A370E5702571FEF753FFFE23A8
:103B1800B0FBF3F000EB400000EB40106071224670
:103B28000621C7E78378303BDBB2092BDBD878491D
:103B3800784A0B700B78DBB25372744A59231370AE
:103B48004D2353700B783033937003210120FFF716
:103B5800DBFC10B0BDE87040FFF730BD8578482D1C
:103B680013D16A4A0021562351701821137093709B
:103B78000120032351710821D07013719371D17101
:103B880010B0BDE87040FFF7BFBC432DABD15F4C10
:103B980000213C2201A800910DF0CCF86846FFF7FF
:103BA80079FD2422802104F10C000DF0C3F89DF862
:103BB800003063709DF80130A3709DF80230E37007
:103BC8009DF8033023719DF8043063719DF805302A
:103BD800A3719DF80630E3719DF8073023729DF8B4
:103BE8000830257063729DF80B509DF80930A37258
:103BF8009DF80A30E3722A4603A9257304F10D00E3
:103C08000DF0C9F805F10D012246C9B2012068E797
:103C1800807839280CD83038C0B2FFF77FFA3B4A91
:103C28002378137063785370A3789370032141E766
:103C380010B0BDE87040FFF7B3BC80783928F7D8DA
:103C48003038C0B2FFF76BFAE9E780783928EFD847
:103C58003038C0B2FFF764FAE1E78378303BDAB274
:103C6800092AE5D8C0783038C2B2092AE0D82179C3
:103C7800A1F14802D2B20B2ADAD8274D45FA02F24E
:103C8800D207D5D40A224D2902FB030036D13C23A2
:103C980058434FF47A735843204B1860204B1860F0
:103CA800FFF7A4FA194A2378137063785370A3783E
:103CB8009370E378D3702379137105210120FFF7FE
:103CC80023FC144B00221A7056225A7001229A7053
:103CD800DA70A278303A02EB8201E278303A02EBED
:103CE8004102D2B21A7122795A710E4A1278D2B2AE
:103CF8001A72074A1278D2B25A722AE74829C8D1EA
:103D08004FF46163C4E700BFFB0F0108FD05002005
:103D18007004002078000020DEF7FFFF7400002008
:103D28000C000020920600208678A6F13003092BAB
:103D38003FF67EAFC078A0F13003092B3FF678AF8D
:103D48002179A1F14802D2B20B2A3FF671AF5A4B42
:103D5800134113F001057FF46BAF584A59231370D0
:103D680053235370D0701171967005210120FFF70D
:103D7800CBFB534956230D704B7001238B70CB70CE
:103D8800A378303B03EB8302E378303B03EB420339
:103D9800DBB28B712379CB714A4B1B78DBB20B7288
:103DA800494B1B78DBB24B72D3E6502B48D1022922
:103DB8007FF699AE4378303B012B3FF694AE83787B
:103DC800312B7FF490AE0B2904D8FFF7E9FB0021D3
:103DD8003A4A6FE63A4D0234002214F8013FA91816
:103DE800303B0132DBB20C2A0B73F6D1FFF7CAF96C
:103DF800324B502256211A709970002201215A70B4
:103E0800D97003F8041FA9180132097B0C2A01F1A3
:103E1800300103F8011FF6D100232B7056236B7075
:103E28000123AB70EB70274B1B78DBB22B72264B50
:103E38001B78DBB26B72EA72FFF7C0FB1121C7E790
:103E4800412B7FF450AE4378432B7FF44CAE1629B8
:103E58007FF449AE1D4D421C002312F8011FE9549E
:103E68000133142BF9D1FFF7F5F8194B5B7D012BC2
:103E780019D113490023EA5CC8180133D2B2142BB4
:103E880080F82C20F7D1104B00221A701B78DBB277
:103E98004B72FFF793FB094A631E1534A34206D100
:103EA800064A162106E6084B02221A70F3E713F8B1
:103EB800011F02F8011BF1E7DEF7FFFFFD050020F7
:103EC8007800002092060020700400207E06002062
:103ED8003403002037B504460D46002939D022485E
:103EE8000CF064FD2B78A3B39CB36068237880B38F
:103EF800032B0DD0072B2ED0022B2AD16178012954
:103F080027D00B0625D403B0BDE83040FFF788BDA5
:103F18006378012B07D10078012802D0022800D04D
:103F280008B903F0F9FF00240DF107008DF80740E8
:103F380004F03CF80D4A4C231370562393709DF8F7
:103F48000730547001204133D07013710521FFF7F9
:103F5800DBFA03B030BD6378012BFAD10378044A49
:103F680003F001031370F4E780050020FD0500202D
:103F780064050020034B0022C3E902220122C3E9A1
:103F880000227047940600200048704794060020DD
:103F98004FF0B04382B0DA6C0243DA64DB6C034062
:103FA8000193019B02B070472DE9F04186B00024CF
:103FB8000220154D0594FFF7EBFF0420FFF7E8FFFB
:103FC800124F03944FF4807601230DEB0001CDE9E5
:103FD80001632846032304934FF4005801F054F872
:103FE80001A93846CDF8048001F04EF82246414632
:103FF800384601F06FF928462246314601F06AF941
:10400800204606B0BDE8F0810004004800080048DA
:10401800032810B50ED8012810D868B902460B48F5
:104028004FF4807101F056F9002209484FF400510D
:1040380001F050F9002010BD0122F0E700220348EA
:104048004FF4807101F046F90122EEE700040048C0
:104058000008004802207047002070470120704780
:1040680000280CBF0F201620704700000D48854619
:1040780000F027F80C480D490D4A002302E0D458F7
:10408800C4500433C4188C42F9D30A4A0A4C00239A
:1040980001E013600432A242FBD30CF053FEFEF79A
:1040A800C7FAFEE700000120000000204C010020B4
:1040B800F41A01084C01002030240020FEE70020FB
:1040C8007047704710B5032000F072FC01F018FB30
:1040D800064B18600F20FEF7E5FC044618B9FEF7FA
:1040E80058FB204610BD0124FBE700BFB8000020A4
:1040F8004FF0E022136923F00203136170474FF079
:10410800E022136943F0020313617047014BD3F8AF
:10411800900570470070FF1F014BD3F89405704756
:104128000070FF1F014BD3F8980570470070FF1F00
:10413800024A536823F0010353607047002004E0EB
:10414800024A536823F0020353607047002004E0DA
:10415800024A536823F0040353607047002004E0C8
:104168008068C0F380007047F7B5002301930446C8
:10417800002800F0E980856D25B9FDF76FFEE5653B
:1041880084F8545023689A68D00040F1A1809A6856
:10419800D10000F1B480A26D42F01002A265E26D78
:1041A80042F00102E26501251846FFF7D9FFA26D2A
:1041B80002F01002024340F0C980A26D206922F487
:1041C800817242F00202A2659A68D2075DD4226B1E
:1041D800A67E94F82CC0003A18BF01221703D4E930
:1041E80002120A43217E42EA8132617E42EAC132EA
:1041F80042EA4632002842EA4C02B4BF20F00041AD
:104208004FF400113A430A4394F82010012903D1CE
:10421800002E76D142F48032616A21B1A66A01F497
:10422800E07131430A43D968E66C21F4FE3121F488
:10423800FF711143D96094F83C206168012A01F0AC
:10424800404C4CEA060609D1D4E910273A433243D8
:10425800A66C324342EA0C0242F001061F693E4A4C
:104268003A4032431A6121F00042B2F1804F0CD03B
:10427800B1F1004F09D0394ED6F8082701F4701172
:1042880022F470120A43C6F808275A69666BA16BB4
:1042980022F0070232435A615A6922F0700242EA58
:1042A80001125A61002835D19A6A62F00F029A62A7
:1042B8005B6903F007039E423CD10023E365A36DCD
:1042C80023F0030343F00103A365284603B0F0BDC0
:1042D8009A68234922F0104222F0170242F08052D5
:1042E8009A60204A1268B2FBF1F201325200019240
:1042F800019A002A3FF44BAF019A013AF7E70025EB
:1043080052E7A16D41F02001A165E16D41F0010185
:10431800E16581E7B0F5001FCAD19A6AE269013AFE
:1043280092006FF00F0102F01C0201FA02F2216EF6
:104338000A43BCE7A36D23F0120343F01003A365FF
:10434800E36D43F00103E3650125BEE7A36D43F088
:104358001003A365F8E700BF02FCFF1F002001401F
:10436800400D0300B8000020F8B54569082D044643
:104378000E460AD00368DB68D80705D5A36D43F05D
:104388002003A3650120F8BD0425FEF78DFB074631
:1043980023681A682A4221D0A26D42F40072A265ED
:1043A800DA6812F4406F14D1A27E92B91A68120723
:1043B8000FD51846FFF7D4FE28BB5A6822F00C0226
:1043C8005A60A26D22F4807222F0010242F00102CA
:1043D800A265207E00BB0C221A60D4E7711CD8D0DD
:1043E800FEF762FBC01BB04201D8002ED0D1236873
:1043F8001B682B40CCD1A26D84F8543042F00402E3
:10440800A2650320BFE7A26D42F02002A265E26D1B
:1044180042F00102E265DCE70020B4E70368186CAB
:1044280070470000F7B50023019390F85430012B32
:10443800044600F0C58005680669012380F85430F9
:104448002846FFF78DFE002840F0B480D1E900200F
:10445800022826F0040300F08280B3F1004FC2F373
:10446800110E13D1AB6A43EA0E03AB628B6868691D
:1044780003EA022323F07C4323F0FF0320EA02210E
:104488000B43002A6B6126DB002055E0236E00F009
:104498001F074FF00F0C0CFA07FC6FEA0C0623EA13
:1044A8000C0CBEF1000F11D1C2F38463BB4043EA88
:1044B8000C0323668008E36901309842D6D8A86ABD
:1044C800C2F38363BB4006403343CEE792FAA2F3BC
:1044D800B3FA83F3EAE73B493B48D1F8083782420D
:1044E80003F0E07519D11B02CED4D1F8083723F0B8
:1044F800E0732B4343F40003C1F80837334B1A68C1
:10450800334BB2FBF3F20C2302FB03330193019B01
:10451800002BB9D0019B013BF8E72E48824210D10D
:1045280013F08070B0D1D1F8083723F0E0732B4333
:1045380043F08073C1F80837002384F8543003B07F
:10454800F0BD254882429FD113F480009CD1D1F858
:10455800083723F0E0732B4343F48003EAE7B3F111
:10456800004F01BFAB6AC2F311018B43AB62002A53
:104578008ADA154813498242D1F8083709D1D1F8A7
:10458800082703F0A07322F0E0721343C1F808373C
:104598007AE71048824204D1D1F8082703F440038F
:1045A800F1E70D4882427FF46FAFD1F8082703F096
:1045B800C073E8E7A26D42F02002A2651846BBE787
:1045C8000220BCE700200140001000B0B800002025
:1045D800400D0300004000B8002000B4026838B560
:1045E80004461046FFF7BCFD08B9002038BD9368A3
:1045F800990707D4936823F0004323F0170343F087
:1046080010039360FEF750FA054623689B685B0722
:10461800EBD5FEF749FA401B0228F6D923689B68B8
:104628005A07F2D5A36D43F01003A365E36D43F079
:104638000103E3650120D9E773B5002302680193FC
:104648009368DD07044602D5002002B070BD91686A
:10465800214B194209D0A36D43F01003A365E36D04
:1046680043F00103E3650120EFE7936823F000437B
:1046780023F0170343F001039360184BD3F808376E
:1046880018021CD4637E012BDED0FEF70DFA144EFF
:10469800054622681368DB07D6D49368D9075FBF3D
:1046A8009368334043F001039360FEF7FDF9401B24
:1046B8000228EED923681B68DA07EAD4CBE7094B4E
:1046C800094A1B68B3FBF2F301330193019B002BEA
:1046D800D8D0019B013BF8E717000080002001407B
:1046E800E8FFFF7FB8000020400D030038B50446FE
:1046F8000068FFF735FD054620BB94F85430012BC0
:1047080020D0012384F854302046FFF795FFB0B934
:10471800A36D226823F4706323F0010343F48073CC
:10472800A3651C23E065136084F85400936823F0A4
:10473800004323F0170343F00403936038BD84F863
:104748005450FBE70220F9E7026838B5936891688E
:104758000446C80701D4002038BD9907FBD49368E4
:1047680003F00503012B19D1936823F0004323F0CC
:10477800170343F00203936003231360FEF794F9D1
:10478800054623689B68DB07E5D5FEF78DF9401BD6
:104798000228F6D923689B68DA07F2D5A36D43F09F
:1047A8001003A365E36D43F00103E3650120D3E73C
:1047B80070B5044600284BD0836D43F0020383652F
:1047C800FFF70CFF054668B92046FFF7BDFF054611
:1047D80008B90123A3652268936823F0104323F0E6
:1047E8001703936023685A6822F4677222F0030261
:1047F8005A6040F29F321A60D968164A0A40DA6055
:104808001A6922F040421A615A6922F007025A6175
:104818001A6A02F0F0221A625A6A02F0F0225A6208
:10482800DA6A02F0F022DA629A6A0B4A00269E627D
:10483800D2F8083723F0FE73C2F808372046FDF790
:1048480021FBE6652666A66584F85460284670BD97
:104858000125FBE700023E830020014010B590F8D7
:104868005430012B044615D0012380F85430FFF74B
:10487800B5FE58B92046FFF767FF38B9A36D23F492
:10488800807323F0010343F00103A365002384F838
:10489800543010BD0220FCE7F7B50023019390F8CF
:1048A8005430012B04467FD0012380F85430FFF7A1
:1048B8004BFF23689A6812F00102054607D0A36DE2
:1048C80043F01003A365002384F854302DE0A16D54
:1048D800364F21F4817141F00201A165DE68D96883
:1048E80026F4FF4626F07C0621F40041360421F028
:1048F8000301360CD96008209968394041F000411D
:1049080099609968002913DA019901310191019997
:10491800B1F52E3FF5D3A36D23F0120343F0100336
:10492800A365002384F854300125284603B0F0BD60
:10493800D3F8B410013801F07F010A44DCD199683A
:104948001A48014041F001019960D3F8B41021F0F0
:104958007F0141EAD202C3F8B4209A68024042F0CB
:1049680002029A60FEF7A0F8074623689A68D20701
:1049780008D4DA683243DA60A36D23F0030343F006
:1049880001039FE7FEF790F8C01B0228EDD92368C2
:104998009B68D907E9D5A36D43F01003A365E36DC0
:1049A80043F00103E365BFE70225BEE7E8FFFF7FA9
:1049B8000749CA6822F4E0620302120403F4E063C0
:1049C800120C134343F0BF6343F40033CB607047CA
:1049D80000ED00E0164B30B5DC68C4F30224C4F1E6
:1049E8000703251D042B28BF0423062D4FF0FF3590
:1049F8008CBF033C002405FA03F321EA0303A54016
:104A080022EA0502A340002843EA0203ACBF00F1F2
:104A18006040084A4FEA0313B8BF00F00F00DBB24A
:104A2800AABF00F56140135480F8003330BD00BFC1
:104A380000ED00E014ED00E0002807DB044A41091E
:104A4800012300F01F00834042F82130704700BF67
:104A580000E100E000280CDB4309064900F01F00D4
:104A680020330122824041F82320BFF34F8FBFF348
:104A78006F8F704700E100E070B5D0E913456560BD
:104A8800446D14B1D0E916456560D0E9105404F0BE
:104A98001C060124B4406C60046863608368102BB2
:104AA8000BBFA260A160E160E26070BD0268416C6A
:104AB800D3B210B5083B1424B3FBF4F30B4CA24259
:104AC80088BF0B4A21F0030199BF01F1804202F52A
:104AD8000232521807338264064AC26403F01F0385
:104AE800012202FA03F3036510BD00BF0704024068
:104AF8001C0802408008024038B500285ED00268D1
:104B08002F4B9A424FF014014CD82E4B1344B3FB51
:104B1800F1F32D499B00C0E91013022380F82530DA
:104B28001368056923F4FF4323F070031360D0E989
:104B3800024323432B43456911682B4385692B4363
:104B4800C5692B43056A2B430B431360FFF7AEFF80
:104B5800B4F5804F04BF002343604268816C02F0C3
:104B68007F030B60D0E91314013A032A4C6020D864
:104B7800164A174981651A44013B9200012103F046
:104B8800030301FA03F300214265C3651160114A6A
:104B9800536400230122C36380F8243080F8252061
:104BA800184638BD0C4B1344B3FBF1F30B499B007B
:104BB800B1E70023C0E91533C365EAE70120F0E750
:104BC80007040240F8FFFDBF000002403F820010CA
:104BD8004009024000090240F8FBFDBF0004024002
:104BE80038B5002841D00268136823F00103136028
:104BF8001F4B9A424FF0140130D81E4B1344B3FB9D
:104C0800F1F31D499B00C0E91013012403F01C03B4
:104C180004FA03F3002515604B60FFF747FF836C28
:104C280041681D60D0E913325A604A1E032A06D82B
:104C3800124B0B449B0094401D60114B5C64002395
:104C4800C363C0E91533C0E90B33C0E90D33C3654D
:104C580080F8253080F82430184638BD094B1344B5
:104C6800B3FBF1F308499B00CDE70120F5E700BF4E
:104C780007040240F8FFFDBF000002403F82001019
:104C880000090240F8FBFDBF0004024070B590F82F
:104C98002450012D04463BD090F825600125AE42F2
:104CA80080F824504FF000062CD1022580F82550BA
:104CB8000568C6632E6826F001062E60FFF7DCFE45
:104CC800036BBBB12B6843F00E032B60A36C1A680F
:104CD800D20342BF1A6842F480721A60636D1BB136
:104CE8001A6842F480721A602B6843F001032B6043
:104CF800002070BD2B6823F004032B602B6843F061
:104D08000A03E2E78023C36380F824602846F0E7BB
:104D18000220EEE7034640B190F82520022A06D08B
:104D28000422C263002280F8242001207047026810
:104D3800806C116821F00E011160016821F4807106
:104D48000160116821F001011160D3E9100202F03D
:104D58001C0101228A404260D3E9132151605A6D37
:104D680032B1116821F480711160D3E916215160C4
:104D78000122002083F8252083F82400704710B50D
:104D880090F82530022B03D00423C363012010BD03
:104D980003681A6822F00E021A601A6822F00102EB
:104DA8001A60826C136823F480731360D0E91013BF
:104DB80003F01C02012393404B60D0E913325A6080
:104DC800436D33B11A6822F480721A60D0E9163242
:104DD8005A60012380F82530836B002480F8244032
:104DE80013B198472046D2E71846D0E770B4426C12
:104DF800046C036826681D6802F01C0204219140B7
:104E080031420FD015F0040F0CD01A6892065EBF1D
:104E18001A6822F004021A60036B6160002B33D019
:104E280070BC184702219140314217D015F0020F8B
:104E380014D01A68940606D41A6822F00A021A6076
:104E4800012280F82520114A93428CBF104B114B48
:104E58005960002380F82430C36ADFE708219140B5
:104E6800314211D029070FD5196821F00E011960B8
:104E7800012303FA02F26260C36380F8253000233D
:104E880080F82430436BC9E770BC7047800002404B
:104E980000040240000002400A4A536943F4802398
:104EA80030B55361EFF3108472B60023CD58C55066
:104EB8000433B3F5807FF9D11369DB03FCD484F3A1
:104EC800108830BD00400058064B5A69002ABFBF01
:104ED800054A9A6002F188329A60BABF5869C00FD1
:104EE800002070470040005823016745044B5A6969
:104EF80042F000425A615869C043C00F704700BF72
:104F08000040005870B50546FDF7CEFD124E044628
:104F18003369D90313D43369DA0744BF01223261F4
:104F28004CF2FA32134011D10B4E306910F4802044
:104F38000BD0FDF7B9FD001BA842F6D304E0FDF73E
:104F4800B3FD001BA842E3D3032070BD024A1361DE
:104F5800024A01205360F8E700400058A4060020E8
:104F68002DE9F041184D98462B78012B06460C4642
:104F7800174626D001232B704FF47A7000236B60FC
:104F8800FFF7C0FFA0B9012E16D1104A536943F0AC
:104F9800010353612760BFF36F8FC4F804804FF497
:104FA8007A70FFF7AFFF094A536923EA0603536192
:104FB80000232B70BDE8F08139462046FFF76CFFCF
:104FC800EDE70220F6E700BFA406002000400058E5
:104FD800054A536923F47E7343EAC00040F48030E5
:104FE80040F0020050617047004000582DE9F04140
:104FF800234F3B78012B054688463FD001233B7061
:105008004FF47A7000237B60FFF77CFF044688B971
:105018002B68042B13D11B4A536943F4803343F0A4
:10502800040353614FF47A70FFF76CFF0446154B85
:105038001A681B6800233B702046BDE8F0814FF0DA
:10504800FF33C8F800306E68D5E901321344B34223
:105058000AD93046FFF7BCFF4FF47A70FFF752FFCA
:1050680050B1C8F800600446064A536923F47E73B9
:1050780023F002035361DAE70136E5E70224DBE7B0
:10508800A4060020004000582DE9F04F524C0023A0
:105098004FF00F090A6832FA03F501D1BDE8F08F25
:1050A800012505FA03F818EA020200F08E804E681E
:1050B800032706F003054FEA430E07FA0EFC6F1E9E
:1050C800012F6FEA0C0C32D8876807EA0C0ACF6800
:1050D80007FA0EF747EA0A078760476827EA0808C9
:1050E800C6F300179F4047EA08074760C76807EA02
:1050F8000C088F6807FA0EF747EA0807022DC76001
:1051080017D14FEAD30800EB880803F0070AD8F84C
:1051180020704FEA8A0A09FA0AFB27EA0B0B0F6983
:1051280007FA0AF747EA0B07C8F8207001E0032DD1
:10513800DCD1076805FA0EF507EA0C073D4316F4BB
:10514800403F056041D023F0030707F1804707F58A
:10515800803703F0030CBD684FEA8C0C4FF0070E44
:105168000EFA0CFEB0F1904F25EA0E0E2FD01B4D13
:10517800A8422ED005F58065A8420CBF0225072558
:1051880005FA0CF545EA0E05BD602568D74316F407
:10519800801F0CBF3D4015432560656816F4001F4D
:1051A8000CBF3D4015436560D4F8805016F4803F2D
:1051B8000CBF3D401543C4F88050D4F88450B60362
:1051C80054BF3D401543C4F88450013362E70025BD
:1051D800D6E70125D4E700BF0008005800040048BE
:1051E800374A2DE9F04F00234FF0010A4FF0070B23
:1051F8004FF00F0931FA03F401D1BDE8F08F0AFA34
:1052080003FC1CEA010654D023F0030404F1804493
:1052180004F5803403F00307A568BF000BFA07F80C
:10522800B0F1904F08EA050E45D0264DA84244D06B
:1052380005F58065A8420CBF02250725BD407545C8
:1052480017D1D2F8805025EA0605C2F88050D2F866
:10525800845025EA0605C2F88450156825EA060533
:105268001560556825EA06055560A56825EA08050C
:10527800A560056803265C0006FA04F423FA06F61E
:10528800254300EB8606056003F00705376AAD0085
:1052980009FA05F527EA05073762856825EA04054E
:1052A8008560456825EA0C054560C56825EA04045B
:1052B800C46001339EE70025C0E70125BEE700BFB3
:1052C80000080058000400480369194214BF01206F
:1052D800002070470AB18161704781627047000001
:1052E800044AD168014208B502D0D060FEF7FDF843
:1052F80008BD00BF0008005810B5044600284AD071
:1053080090F8413003F0FF021BB980F84020FDF708
:10531800CFF8242384F8413023681A6822F0010268
:105328001A60626822F070621A619A6822F4004278
:105338009A60D4E90221012924D142F400429A60FA
:105348005A6842F0007242F400425A60DA6822F465
:105358000042DA60D4E904210A43A16942EA012241
:10536800DA60D4E907210A431A601A6842F0010298
:105378001A6000202023606484F84130206384F898
:10538800420010BD42F4044202299A6004BF4FF45F
:1053980000625A60D4E70120F3E710B590F8412085
:1053A800202A0346D4B21CD190F84020012A18D0F4
:1053B800242280F841200268106820F00100106063
:1053C800106820F480501060106801431160116863
:1053D800002041F00101116083F8414083F840004A
:1053E80010BD0220FCE710B590F84120202A0346A2
:1053F800D4B21BD190F84020012A17D0242280F87B
:1054080041200268106820F001001060106820F444
:10541800706040EA012111601168002041F001012B
:10542800116083F8414083F8400010BD0220FCE77A
:10543800024A136843F480731360704700040058ED
:105448000D4B10B55B690C4628B99A0507D500F0D5
:1054580027F820B110BD9B0501D400F019F8074AC0
:105468001369012C23F00403136101D130BFF1E764
:1054780040BF20BF20BFEDE70004005800ED00E06A
:10548800024B186800F4C060704700BF0004005861
:10549800024A136843F480431360704700040058BD
:1054A8000C4A136823F4804313600B4B1B683221AA
:1054B8004B430A49B3FBF1F35169890500D533B968
:1054C800536913F4007F14BF032000207047013B89
:1054D800F2E700BF00040058B800002040420F0067
:1054E8000B4A136823F0070343F002031360094BC8
:1054F8001A69012842F004021A6105D130BF1A69FD
:1055080022F004021A61704740BF20BF20BFF6E7AF
:105518000004005800ED00E04FF0B0431868C0F3F5
:10552800404070474FF0B0431868C0F340007047E0
:105538004FF0B042536823F47F4343EA002353609B
:1055480070474FF0B0431868C0F3406070470000E0
:105558007FB54FF0B0432C4AD3F80831C0F303109D
:1055680003F00F0352F82040284A52F82330B4FBC6
:10557800F3F4FFF785FF264B054693E80700B5F5DA
:10558800007F04AB03E9070010D0224B9C4218D3DC
:1055980003F5B70303F67F539C4229D903F5741327
:1055A80003F510639C4225D802230BE01A4B9C425A
:1055B80007D91A4B9C421BD903F5370303F5D85377
:1055C800F0E7002304AA02EB830353F80C4C144DB4
:1055D8002B6823F0070323432B60FDF765FA064683
:1055E8002B6803F007039C4206D1002004B070BD6D
:1055F8000123E7E70024EAE7FDF756FA801B0228B3
:10560800EED90320F2E700BF70100108101001085E
:10561800E00E0108C0CF6A00BFEA21013F933402BF
:10562800004000584FF0B04310B59A68D96812F09E
:105638000C0205D00C2A4AD101F00303012B50D1EA
:105648004FF0B0412B480B6813F0080306D00B68E5
:1056580013F0080337D1D1F8941007E00C68240739
:1056680056BFD1F894300968C3F3032350F82330A8
:10567800002A0CBF184600204FF0B0418A6802F09B
:105688000C020C2A1ED1CA6802F00302022A2ED08C
:10569800032A06D10B68184A13F4801F174B18BF4A
:1056A80013464FF0B042D068D168D268C0F30620E4
:1056B8005843C1F302130133B0FBF3F0530F013326
:1056C800B0FBF3F010BD0B68C3F30313CEE7042A55
:1056D8000AD0082A05D11B6813F4801304D107489F
:1056E800CAE700231846C7E703480023C4E7024B6C
:1056F800D7E700BF701001080024F4000048E80153
:1057080008B5FFF78FFF4FF0B043044A9B68C3F317
:10571800031352F82330B0FBF3F008BD1010010852
:105728002DE9F0410446002853D04FF0B0439D685E
:10573800DE6803689B0605F00C0506F0030668D5CD
:10574800026A1DB10C2D46D1012E44D1002A40D049
:105758004FF0B043A16A1A68170756BFD3F89430C0
:105768001B681B0903F0F00399421FD90846FFF78D
:10577800EFFE00282DD14FF0B042136843F0080324
:1057880013601368A16A23F0F0030B431360606A87
:10579800FFF7CEFEFFF7B4FFAB4B1860AB4B1868B2
:1057A800FDF780F9002834D0BDE8F0814FF0B04211
:1057B800136843F008031360136823F0F0030B43E6
:1057C8001360606AFFF7B4FE0846FFF7C1FE0028C1
:1057D800E0D00120E8E74FF0B043002A54D01A681F
:1057E80042F001021A60FDF75FF90746FFF79AFEDB
:1057F800002842D04FF0B042136843F0080313600A
:105808001368A16A23F0F0030B431360606AFFF783
:105818008FFE2368D80748D42368990700F18C8045
:1058280023681E0740F1FA80A3694FF0B046002BA9
:1058380000F0E180D6F89430E16903F0100291425B
:1058480000F0C48003F00302022AC2D0D80740F156
:10585800B380D6F8943023F00103C6F89430FDF7EE
:1058680023F90746D6F89430990740F1A580FDF74B
:105878001BF9C31B112BF5D904E0FDF715F9C01B63
:105888000228B3D903208FE71A6822F001021A60B0
:10589800FDF70AF90746FFF745FE0028B9D0FDF7DE
:1058A80003F9C01B0228F6D9ECE7082D03D00C2D0C
:1058B80005D1032E03D16368002BADD189E74FF0E2
:1058C800B043A1681A6822F480120A431A60626819
:1058D800B2F5803F10D11A6842F480321A60FDF7A1
:1058E800E3F80746FFF718FE002895D1FDF7DCF826
:1058F800C01B6428F6D9C5E7B2F5041F04D11A689D
:1059080042F400121A60E6E7196821F48031196040
:10591800196821F400111960002AE0D1FDF7C4F8D4
:105928000746FFF7F9FD00283FF476AFFDF7BCF80E
:10593800C01B6428F5D9A5E7042D236903D00C2DD5
:105948000ED1022E0CD1002B3FF443AF4FF0B042E2
:105958006169536823F0FE4343EA016353605FE7DC
:105968004FF0B046BBB1336843F480733360FDF742
:105978009BF8074633685A0507D57368626923F0B0
:10598800FE4343EA026373604AE7FDF78DF8C31BE1
:10599800022BEFD976E7336823F480733360FDF781
:1059A80083F8074633685B057FF53AAFFDF77CF867
:1059B800C31B022BF6D965E74FF0B042E169D2F874
:1059C800943023F010030B43C2F894304FF0B047E3
:1059D800D7F8943043F00103C7F89430FDF764F822
:1059E8000646D7F894309A0718D4FDF75DF8831B5C
:1059F800112BF6D946E7D6F8943023F00103C6F800
:105A08009430FDF751F80746D6F894309B0705D532
:105A1800FDF74AF8C31B112BF6D933E7236858075B
:105A280054D50B4F3B68D90514D4FFF701FDFDF79A
:105A38003BF806463B68DA050CD4FDF735F8831BBE
:105A4800022BF7D91EE700BFB8000020BC000020D9
:105A580000040058E3684FF0B046002B58D023F0FC
:105A68008003052B02BFD6F8903043F00403C6F834
:105A780090304FF0B046FDF717F8D6F8903043F065
:105A880001030746C6F8903041F28838D6F89030BE
:105A98009B0705D4FDF708F8C31B4345F6D9F1E683
:105AA800E36823F00403812B1BD1FCF7FDFFD6F834
:105AB800903043F08003C6F8903007464FF0B04668
:105AC80041F28838D6F89030180504D5E06A0028E5
:105AD8004AD1002068E6FCF7E7FFC01B4045F1D932
:105AE800D0E6FCF7E1FFD6F8903023F08003C6F843
:105AF800903007464FF0B04641F28838D6F89030DB
:105B08001905E3D5FCF7D0FFC01B4045F6D9B9E627
:105B1800FCF7CAFFD6F8903023F080030746C6F892
:105B2800903041F28838D6F890301A0516D4FCF730
:105B3800BBFFD6F8903023F00103C6F89030074633
:105B48004FF0B04841F28836D8F890309B07BDD561
:105B5800FCF7AAFFC31BB342F6D993E6FCF7A4FFF0
:105B6800C01B4045DFD98DE60C2D4ED04FF0B04319
:105B780002281A6822F080721A6033D1FCF794FF69
:105B88000546FFF7DEFC38BBD4E90C314FF0B042D4
:105B98000B43D0682D4901400B43E16B0B43216C4B
:105BA8000B43616C0B43A16B43EA0123D360136879
:105BB80043F080731360D36843F08053D360FCF7DD
:105BC80073FF0446FFF7BDFC002882D1FCF76CFF89
:105BD800001B0A28F6D955E6FCF766FF401B0A2881
:105BE800CFD94FE6FCF760FF0446FFF7AAFC30B9AF
:105BF8004FF0B042164BD1680B40D360D4E5FCF7A8
:105C080053FF001B0A28F0D93CE601283FF4CCAD2D
:105C18004FF0B043226BDB6803F0030191427FF43D
:105C2800D8AD616B03F070028A427FF4D2ADA16BEC
:105C380003F4FE42B2EB012F7FF4CBAD626C03F0AC
:105C4800604393423FF445AFC3E500BF8C80C11168
:105C5800FCFFFEEE2DE9F0410D46044610B9012087
:105C6800BDE8F081684E336803F007038B4216D312
:105C780023689A0727D54FF0B047A268BB6823F07E
:105C8800F0031343BB60FCF70FFF0646BB68DB035A
:105C980019D4FCF709FF831B022BF7D911E03368ED
:105CA80023F007030B433360FCF7FEFE0746336817
:105CB80003F00703AB42DBD0FCF7F6FEC01B02285B
:105CC800F5D90320CCE72368580617D54FF0B0471D
:105CD8006269D7F8083123F00F0343EA1213C7F8B3
:105CE8000831FCF7E1FE0646D7F80831D90305D498
:105CF800FCF7DAFE831B022BF6D9E2E723685A0782
:105D080013D54FF0B047E268BB6823F4E063134350
:105D1800BB60FCF7C9FE0646BB689B0305D4FCF7CD
:105D2800C3FE831B022BF7D9CBE72368180714D5CA
:105D38004FF0B0472269BB6823F4605343EAC203BB
:105D4800BB60FCF7B1FE0646BB68590305D4FCF7F7
:105D5800ABFE831B022BF7D9B3E72368DA070FD40E
:105D6800294C236803F00703AB4239D8FFF7C8FC76
:105D7800264B1860264BBDE8F0411868FCF792BE28
:105D88006268022A1DD1FFF7C7FB00283FF467AFFE
:105D98004FF0B04641F28838B36823F00303134349
:105DA800B360FCF781FE0746B368626803F00C0332
:105DB800B3EB820FD4D0FCF777FEC01B4045F3D974
:105DC8007FE7032A02D1FFF7BCFBDEE712B9FFF732
:105DD800A9FBDAE74FF0B0431B685B05D8D43EE770
:105DE800236823F007032B432360FCF75DFE064678
:105DF800236803F00703AB42B8D0FCF755FE801BBD
:105E08000228F5D95DE700BF00400058B80000201F
:105E1800BC00002008B5FFF773FC4FF0B043044AFC
:105E28009B68C3F3022352F82330D84008BD00BF53
:105E38005010010808B5FFF763FC4FF0B043044A5F
:105E48009B68C3F3C22352F82330D84008BD00BF73
:105E5800501001084FF0B043D3F89000C0F3400051
:105E680070474FF0B0410209D1F8883002F47F2220
:105E7800000123EA020300F47F200343C1F88830BD
:105E880070474FF0B041020CD1F88830120423EA71
:105E9800020343EA0040C1F88800704770B50668FD
:105EA80016F48036044638D0FFF7C2FAFCF7FCFD3A
:105EB800614E05463368DB0529D54FF0B043616B69
:105EC800D3F8902002F44072914214D0D3F8901085
:105ED800D3F8902042F48032C3F89020D3F8902071
:105EE80021F4407022F480328D07C3F89020C3F863
:105EF800900000F190804FF0B042616BD2F8903082
:105F080023F440730B43C2F89030002605E0FCF7F9
:105F1800CBFD401B0228CDD903262568E8070AD502
:105F28004FF0B0416268D1F8883023EA124392B248
:105F38001343C1F88830A9070AD54FF0B041A268C9
:105F4800D1F8883023EA124392B21343C1F888305B
:105F5800AA0609D54FF0B0422169D2F8883023F457
:105F680040630B43C2F88830AB0502D5206AFFF7BF
:105F780088FF680502D5606AFFF783FF290502D507
:105F8800A06AFFF77EFF6A0602D56069FFF769FF1E
:105F98002B0602D5A069FFF764FFE80502D5E06982
:105FA800FFF75FFFE90610D54FF0B042E168D2F87D
:105FB800883023F440730B43C2F88830B1F5807FF2
:105FC80002BFD36843F08073D3602A040ED54FF024
:105FD800B042216BD2F8883023F040430B43C2F81B
:105FE800883019B9D36843F08073D3606B0410D537
:105FF8004FF0B042E16AD2F8883023F040530B43A7
:10600800B1F1005FC2F8883003D1D36843F480331C
:10601800D360304670BDFCF747FD41F2883605462F
:10602800FFF718FF01283FF466AFFCF73DFD401B62
:10603800B042F5D970E700BF0004005830B590F8B9
:106048002C30012B02464FF0020022D0174B82F869
:106058002D00CA24012582F82C505C6253245C620E
:10606800B1F5807F146B996914D121F48851996135
:10607800596C24F0010421F0004159641463DD6572
:106088000A4BFF2159620020012382F82D3082F843
:106098002C0030BD21F408519961D96C24F0020418
:1060A80021F00041D9641463D865E9E7002800406D
:1060B80070B50B4E036B756D1D40EA07044603D59A
:1060C8000123F365FCF761FEAB0704D50223F365F2
:1060D800204600F0CBF9012384F82D3070BD00BFB5
:1060E8000028004038B50A4CE36823F02003E36039
:1060F800FCF7DAFC0546E3689B0601D5002038BDAD
:10610800FCF7D2FC401BB0F57A7FF4D90320F6E700
:10611800002800402DE9F041114DEC6814F04004CE
:1061280007461AD1EB6843F08003EB60FCF7BCFC30
:106138004FF003080646EB685B0601D4032C02D136
:106148002046BDE8F081FCF7AFFC801BB0F57A7FF4
:1061580084BF87F82D800324EDE70024F0E700BF13
:106168000028004038B50F4CE36823F08003E36053
:10617800A3699B06054606D4FFF7B4FF10B10320B8
:1061880085F82D0038BDA36923F02003A361FFF72C
:10619800A9FF10B1032085F82D00A36943F020035F
:1061A800A361EFE70028004038B5044600284BD02B
:1061B80090F82D3003F0FF021BB980F82C20FCF773
:1061C80081FA0223214D84F82D30EB68DB0632D4A6
:1061D800CA236B6253236B622046FFF79BFF78BB91
:1061E800AB6923F08E6323F04003AB6121696368D8
:1061F800AA690B431343A2691343AB61D4E9022391
:1062080043EA02432B61D4E90931EA680B4322F4DB
:10621800F8521343EB602046FFF7A4FF80B9D4E996
:106228000713AA690B4322F06042134362691343C0
:10623800AB61FF236B62012384F82D30002002E05C
:10624800024BFF225A6238BD0120FCE700280040BB
:106258000023092803D840EA0310C0B270470A385F
:106268000133C0B2F5E700002DE9F04790F82C3073
:10627800012B05464FF0020069D0012385F82C3028
:106288004E4B85F82D00DE6806F44076B6F5807F23
:1062980078D04C69087891F8019091F802A091F8AB
:1062A8002470002A55D19B6913F0400308BFCB70B6
:1062B800FFF7CEFF80464846FFF7CAFF0246504622
:1062C800FFF7C6FF81463846FFF7C2FF0B6ACF7853
:1062D800234343EA875343EA090343EA084343EA6B
:1062E800022343EA0063354ACA20506253205062B1
:1062F8008C6A8869B4F5807F946945D124F4885400
:1063080094610124D465B6F5807F09BFCB69136415
:106318000343536418BF5064284B4A681A672A6BB2
:1063280042F001022A639A6942F488529A61244A27
:10633800D2F8803043F40033C2F880301F4BFF227C
:106348005A620020012385F82D3085F82C00BDE81D
:10635800F087B4F1803F07D0B4F5000F04D09B69F3
:1063680013F0400308BFCB700B6ACA781C4344EA99
:106378000A0444EA004343EA092343EA825343EA0E
:106388000763B0E70023AEE724F4085494610224BD
:10639800D465B6F5807F09BFCB6993640343D364A2
:1063A80018BFD064054B4A685A672A6B42F002024C
:1063B8002A639A6942F40852B8E700BF00280040EF
:1063C8000008005890F82C20012A03464FF00200DC
:1063D80012D00A4A83F82D00CA2151625321516212
:1063E800916941F020019161FF2151620020012251
:1063F80083F82D2083F82C00704700BF0028004048
:1064080090F82C20012A03464FF0020019D00D4ABB
:1064180083F82D00CA2151625321516291690A48BB
:1064280041F080019161D0F8801041F48021C0F8DA
:106438008010FF2151620020012283F82D2083F86B
:106448002C0070470028004000080058064B5A6D81
:10645800520610B5044603D54022DA65FCF798FCCD
:10646800012384F82D3010BD0028004070478900B2
:1064780001F1804101F531410A607047890001F15D
:10648800804101F53141086870470000034AD2F89D
:10649800903043F40043C2F890307047000400582D
:1064A800034AD2F8903023F40043C2F89030704782
:1064B80000040058074B1A6822F040021A6040F4A2
:1064C80041704FF4B85218605A601A6842F040029E
:1064D8001A6070470000015837B5054600284ED0AD
:1064E800837903F0FF046BB1032C0BD0254B4FF4D9
:1064F80000629A612868FFF7DDFF002401232B71F1
:10650800AC602FE000236B712846FCF7E3F91E4AC4
:10651800D2F8903043F48053C2F89030002CE5D183
:1065280002234FF0B042AB71D2F8943023F4004309
:10653800C2F89430154B1B681C214B43DB0C6421BB
:106548004B430193019B93B90124AC60FFF79EFF75
:106558000C4B9A6842F400629A604FF400629A61A8
:10656800002CC7D00123AB71204603B030BD019B7E
:10657800013B0193D2F894305B04E3D4E6E70124AD
:10658800F2E700BF0004005800080058B8000020D7
:1065980037B5174D2B6802461C204343DB0C64209B
:1065A800434314480193019B93B901209060114C17
:1065B80021732B681C214B43DB0C64214B43019353
:1065C800019B6BB9012090600A4BDB6803B030BDBA
:1065D800019B013B019383689C07E4D50020E6E713
:1065E800019B013B0193A368DB07E9D5ECE700BFFA
:1065F800B80000200000015837B5184D2B68024636
:106608001C204343DB0C6420434315480193019B42
:10661800A3B901209060124CFF2323732B681C251B
:106628006B43DB0C64256B430193019B73B9012019
:1066380090600B4BDB680B7003B030BD019B013BD6
:10664800019383689C07E2D50020E4E7019B013BA6
:106658000193A368DB07E8D5EBE700BFB80000208B
:10666800000001580F4B13B51B680F4C18225343F9
:106678001B0D64225343014601936269019B02F09A
:10668800040223B902238B60012002B010BD019BD4
:10669800013B0193606910F00200F6D0002AECD1AA
:1066A8001046F2E7B80000200004005807B5037947
:1066B800012B0FD10A4B1B68182253431B0C019363
:1066C800FFF7EEFE019B013B0193019B002BF9D1E3
:1066D800FFF7DCFE03B05DF804EBFFF7C3BF00BFB4
:1066E800B8000020F8B51E468379012B15460446EC
:1066F8000F46DAB22DD14379012B2AD002234271F9
:106708008371FFF7D3FF0D212046FFF7C9FEFFF77E
:106718003FFF390A2046FFF73BFFF9B22046FFF753
:1067280037FF2E44B5420ED12046FFF7AFFEFFF7E4
:1067380099FFA06801230038A3714FF0000318BF28
:1067480001206371F8BD15F8011B2046FFF720FFF3
:10675800E8E70220F6E7F8B51E468379012B1546CF
:1067680004460F46DAB22FD14379012B2CD042715F
:10677800FFF79CFF1D212046FFF792FEFFF708FF59
:10678800390A2046FFF704FFF9B22046FFF700FF59
:1067980000212046FFF7FCFE2E44B5420ED12046CC
:1067A800FFF774FEFFF75EFFA06801230038A371AE
:1067B8004FF0000318BF01206371F8BD2946204639
:1067C800FFF71AFF0135E8E70220F6E7F8B51F469C
:1067D8008379012B154604460E46DAB22CD143794B
:1067E800012B29D04271FFF761FF06F0EF03A3F1F7
:1067F800840253425341237131462046FFF750FE2D
:10680800FFF7C6FE2F44AF4210D1FFF73FFE842E9C
:1068180002D02046FFF726FFA06801230038A371A5
:106828004FF0000318BF01206371F8BD15F8011B74
:106838002046FFF7ADFEE6E70220F6E7F8B51E466C
:106848008379012B154604460F46DAB227D14379DE
:10685800012B24D04271FFF729FF39462046FFF764
:106868001FFEFFF795FE00212046FFF791FE2E44FC
:10687800B5420ED12046FFF709FEFFF7F3FEA068E8
:1068880001230038A3714FF0000318BF0120637182
:10689800F8BD29462046FFF7AFFE0135E8E702209C
:1068A800F6E737B50023ADF8043001AA0223122118
:1068B8000546FFF7C3FFBDF80440022364BA01AAE6
:1068C800A4B219462846FFF781FFE20702D52846F9
:1068D80009F088FBA30702D5284609F089FB600761
:1068E80002D5284609F0AEFB210702D5284609F053
:1068F800AFFBE20602D5284609F0B0FBA30602D595
:10690800284609F099FB600602D5284609F076FB6F
:10691800210606D514F4807118BF0121284609F014
:1069280073FBA20502D5284609F07EFB630402D555
:10693800284609F099FB03B030BDF8B51E468379A7
:10694800012B154604460F46DAB227D14379012BAD
:1069580024D04271FFF7AAFE0E212046FFF7A0FDC2
:10696800FFF716FE39462046FFF712FE2E44B542C1
:106978000ED12046FFF78AFDFFF774FEA0680123B9
:106988000038A3714FF0000318BF01206371F8BDF0
:1069980015F8011B2046FFF7FBFDE8E70220F6E7A4
:1069A800F8B51E468379012B154604460F46DAB220
:1069B8002BD14379012B28D04271FFF777FE1E2196
:1069C8002046FFF76DFDFFF7E3FD39462046FFF748
:1069D800DFFD00212046FFF7DBFD2E44B5420ED136
:1069E8002046FFF753FDFFF73DFEA068012300385E
:1069F800A3714FF0000318BF01206371F8BD294649
:106A08002046FFF7F9FD0135E8E70220F6E70268BE
:106A180052E8003F23F0C00342E800310268002931
:106A2800F5D102F1080353E8003F23F4000302F113
:106A3800080C4CE800310029F3D12023C0F8883035
:106A48007047000010B5026852E8003F23F49073C5
:106A580042E8003102680029F5D10F4C02F1080321
:106A680053E8003F234002F1080C4CE800310029AC
:106A7800F4D1C36E012B07D152E8003F23F0100375
:106A880042E800310029F7D12023C0F88C300023D8
:106A9800C366436710BD00BFFEFFFFEFF8B50446AD
:106AA8001346D4F88850202D32D1F1B1EAB1E06F05
:106AB800A4F85620A4F8542000262122C4F8906097
:106AC8002165C4F88820226888B1124FC762124F26
:106AD8000763124F2832C0E90D76FEF7D7F830B1B8
:106AE8001023C4F89030C4F8885001200FE02368C0
:106AF80040221A62226802F1080353E8003F43F07B
:106B0800800302F1080141E800300028F3D1F8BD04
:106B18000220FCE7296B0008716B00087D6B0008F8
:106B280008B50346806A1B681B6813F0200317D159
:106B3800A0F85630026802F1080353E8003F23F03A
:106B48008003083242E8003102680029F2D152E895
:106B5800003F43F0400342E800310029F7D108BD67
:106B6800FCF74CFAFBE7704708B5806AFFF7FBFFB4
:106B780008BD7047806A38B50468D0F88830D0F806
:106B88008C50A268120606D5212B04D10023A0F848
:106B98005630FFF73CFFA3685B0606D5222D04D1CB
:106BA8000023A0F85E30FFF74DFFD0F8903043F097
:106BB8001003C0F89030FFF7DCFF38BD08B5806AD5
:106BC8000023A0F85E30A0F85630FFF7D2FF08BDCA
:106BD800704700000368D9691A682DE9F04140F64A
:106BE8000F0631429D68044610D18E0640F1978009
:106BF80002F0200605F080573E4300F09080436F76
:106C0800002B00F08580BDE8F0411847AB4EAC483A
:106C18002E401040304300F08280CF0709D5D005C0
:106C280007D501201862D4F8900040F00100C4F89C
:106C380090008F0709D5E80707D502201862D4F815
:106C4800900040F00400C4F890004F0709D5E80709
:106C580007D504201862D4F8900040F00200C4F868
:106C680090000F070BD502F02000304307D0082012
:106C78001862D4F8900040F00800C4F890000E059F
:106C88000AD5500108D54FF400601862D4F8903046
:106C980043F02003C4F89030D4F89030002B37D05C
:106CA8008B0609D502F0200205F080552A4303D04F
:106CB800636F0BB1204698472668D4F89020B368D4
:106CC80002F0280203F0400353EA0205204621D0CF
:106CD800FFF7B8FEB3685F0617D5226802F108030C
:106CE80053E8003F23F04003083242E8003100290E
:106CF800F3D1D4F8800040B1724B8363FEF73FF8BC
:106D080030B1D4F88000836B7DE72046FFF731FF70
:106D1800BDE8F081FFF72DFFC4F89050F8E7E06E6A
:106D2800012840F08980CE0640F18680D00640F1E7
:106D3800838010221A629A6851064BD5D4F88020B5
:106D480011684A6892B2002AE2D0B4F85C00904216
:106D5800DED9A4F85E200A6892062FD453E8002FE3
:106D680022F4807243E800210029F7D103F10802D8
:106D780052E8002F22F0010203F1080040E8002148
:106D88000029F3D103F1080252E8002F22F0400253
:106D980003F1080040E800210029F3D12022C4F8BB
:106DA8008C20E16653E8002F22F0100243E800210E
:106DB8000029F7D1D4F88000FDF7ACFF0223236740
:106DC800B4F85E30B4F85C10C91A89B22046FFF7EF
:106DD800FFFE9DE7B4F85E20B4F85E00B4F85C10DE
:106DE80080B292B2002893D0891A89B200298FD034
:106DF80053E8002F22F4907243E800200028F7D1CE
:106E0800314D03F1080252E8002F2A4003F1080629
:106E180046E800200028F4D12022C4F88C206067BE
:106E2800E06653E8002F22F0100243E80020002813
:106E3800F7D102232367C9E7CF0209D56E0207D528
:106E48004FF4801220461A62BDE8F04100F0A0BD60
:106E580008060BD502F0800005F40005284305D08C
:106E6800A36F002B3FF454AF2046CCE64F0611D554
:106E780056060FD553E8002F22F0400243E80021C0
:106E88000029F7D12023C4F88830A1672046FCF7F1
:106E9800B5F83DE70D0206D5500004D52046BDE8FB
:106EA800F04100F077BDCB017FF532AF002ABFF685
:106EB8002FAF2046BDE8F04100F06BBD0100001087
:106EC80020010004C56B0008FEFFFFEFD0F88C20FE
:106ED800B0F86010222A08B5036855D15B6A826D44
:106EE8000B401370836D01338365B0F85E30013B4E
:106EF8009BB2A0F85E30B0F85E309BB2002B42D156
:106F0800026852E8003F23F4907342E800310368B6
:106F18000029F5D103F1080252E8002F22F00102FE
:106F280003F1080C4CE800210029F3D12022C0F815
:106F38008C20184A41679342016705D1C26E012A25
:106F48000ED0FCF769F81EE05A681102F6D553E82E
:106F5800002F22F0806243E800210029F7D1EDE7F5
:106F68000022C26653E8002F22F0100243E80021F5
:106F78000029F7D1DA69B0F85C10D20644BF1022B4
:106F88001A62FFF725FE08BD9A6942F008029A6165
:106F9800F9E700BF00800040D0F88C20B0F86010FE
:106FA800222A08B5036852D15A6A1140826D22F824
:106FB800021B8265B0F85E20013A92B2A0F85E200A
:106FC800B0F85E2092B2002A40D153E8002F22F494
:106FD800907243E800210029F7D103F1080252E832
:106FE800002F22F0010203F1080C4CE800210029CF
:106FF800F3D12022C0F88C20174A416793420167D9
:1070080005D1C26E012A0ED0FCF706F81EE05A68B8
:107018001102F6D553E8002F22F0806243E80021E0
:107028000029F7D1EDE70022C26653E8002F22F0CD
:10703800100243E800210029F7D1DA69B0F85C10A2
:10704800D20644BF10221A62FFF7C2FD08BD9A6932
:1070580042F008029A61F9E7008000402DE9F74FF5
:107068000368B0F86080DF691A689D68D0F88C10F2
:1070780001922229044640F0B480B0F86890DFF805
:107088006CA1DFF86CB10026B9F1000F01D0BB0686
:1070980021D4B4F85E309BB2D3B1B4F868209A42D8
:1070A80016D9226802F1080353E8003F23F0805301
:1070B800083242E8003122680029F2D14D4B63675B
:1070C80052E8003F43F0200342E800310029F7D19D
:1070D80003B0BDE8F08F2368A26D5B6A03EA08037A
:1070E8001370A36D0133A365B4F85E30013B9BB206
:1070F800A4F85E302368DF6978072CD0F9070AD531
:10710800019AD20507D501211962D4F8901041F0EF
:107118000101C4F89010B80709D5E90707D502217D
:107128001962D4F8901041F00401C4F890107A075D
:1071380009D5E80707D504211962D4F8903043F03F
:107148000203C4F89030D4F8903023B12046FFF7FA
:1071580010FDC4F89060B4F85E309BB2002B93D158
:10716800216851E8003F23F4807341E80030236828
:107178000028F5D103F1080252E8001F01EA0A01CC
:1071880042E800100028F5D120215B45C4F88C1096
:10719800606720670AD05968090207D553E8001FBD
:1071A80021F0806143E800100028F7D1E16E012941
:1071B80013D1E66653E8001F21F0100143E80010E0
:1071C8000028F7D1D969CA0644BF102119622046A0
:1071D800B4F85C10FFF7FCFC56E72046FBF71CFFF1
:1071E80052E79A6942F008029A6171E7FEFFFFEFE1
:1071F80000800040D56E00082DE9F74F0368B0F80D
:107208006080DF691A689D68D0F88C100192222985
:10721800044640F0B280B0F86890DFF868A1DFF863
:1072280068B10026B9F1000F01D0BB0621D4B4F82B
:107238005E309BB2D3B1B4F868209A4216D922685E
:1072480002F1080353E8003F23F08053083242E874
:10725800003122680029F2D14C4B636752E8003FA5
:1072680043F0200342E800310029F7D103B0BDE81C
:10727800F08F2368A26D596A08EA010122F8021BFF
:10728800A265B4F85E20013A92B2A4F85E20DF69E4
:1072980078072CD0F9070AD5019AD20507D501211C
:1072A8001962D4F8901041F00101C4F89010B807A1
:1072B80009D5E90707D502211962D4F8901041F0E1
:1072C8000401C4F890107A0709D5E80707D5042106
:1072D8001962D4F8903043F00203C4F89030D4F81F
:1072E800903023B12046FFF744FCC4F89060B4F80E
:1072F8005E309BB2002B95D1216851E8003F23F402
:10730800807341E8003023680028F5D103F10802B2
:1073180052E8001F01EA0A0142E800100028F5D1EE
:1073280020215B45C4F88C10606720670AD0596833
:10733800090207D553E8001F21F0806143E80010D7
:107348000028F7D1E16E012913D1E66653E8001F42
:1073580021F0100143E800100028F7D1D969CA06C6
:1073680044BF102119622046B4F85C10FFF730FCC6
:1073780058E72046FBF750FE54E79A6942F00802A6
:107388009A6173E7FEFFFFEF00800040A16F0008DD
:1073980038B5044603682169A2681D68C0690A43B4
:1073A80061690A437D49024329400A431A605A68C1
:1073B800E16822F440520A435A60794AA16993422B
:1073C8001CBF226A11439A6822F06E4222F430628E
:1073D8000A439A60DA6A616A22F00F020A43DA62A3
:1073E800704A93421CD14FF0B043D3F8883003F071
:1073F800030343F44033A3F54033013B022B00F26F
:10740800C780694A9B5CB0F5004F40F08980082B23
:1074180024D8DFE803F061C0832380232323650099
:10742800624A934209D14FF0B043614AD3F8883099
:1074380003F00C0343F44023E4E7594A93420DD187
:107448004FF0B043D3F8883003F44063B3F5006FCE
:107458001AD005D853B1B3F5806F12D0012009E0D6
:10746800B3F5406FFAD14FF400400EE0FEF7D2FCBE
:1074780058B900204FF00113A3660023C4E91D3357
:1074880038BDFEF7CFF8F3E74A4865684A4B626AA9
:1074980005EB450133F81220B0FBF2F39942DDD831
:1074A800B3EB053FDAD800231946FAF72DFB09029A
:1074B80041EA10616B080002C0182A464FF0000329
:1074C80041F10001FAF720FB3C4BA0F540729A42CB
:1074D800C4D82368D860CCE7FEF79CFC0028C8D045
:1074E8006168354B626A33F81220B0FBF2F24B0840
:1074F80003EB42034FF6EF72B3FBF1F3A3F1100174
:107508009142ABD823F00F02216892B2C3F3420331
:107518001343CB60ADE7FEF785F8DFE72548DFE7E3
:10752800082B9BD801A252F823F000BF7D750008F4
:107538008975000895750008657400088F7500083E
:1075480065740008657400086574000859750008BA
:107558004FF400406368616A174A32F81120B0FBA3
:10756800F2F000EB5300B0FBF3F04FF6EF73A0F12D
:107578001002ACE7FEF74EFC00283FF47AAFE9E7CB
:10758800FEF758FCF8E7FEF74DF8F5E70948E1E79C
:10759800B0F5004FF4D1FEF74DFC9FE7F369FFCF3C
:1075A8000080004000380140B0100108004400404D
:1075B800B310F5070024F400C0100108FFFC0F0009
:1075C800836ADA0710B506D50168C46A4A6822F4E6
:1075D800003222434A609C0706D50168046B4A685A
:1075E80022F4803222434A60590706D50168446B69
:1075F8004A6822F4802222434A601A0706D50168A5
:10760800846B4A6822F4004222434A60DC0606D5AD
:107618000168C46B8A6822F4805222438A60990602
:1076280006D50168046C8A6822F4005222438A60F5
:107638005A060FD50168446C4A6822F48012224326
:10764800B4F5801F4A6005D14A68846C22F4C002F0
:1076580022434A601B0606D50268C16C536823F4AE
:1076680000230B43536010BD2DE9F041DDF818806D
:1076780004460E4615461F462268D36936EA0303B8
:107688000CBF01230023AB4201D0002027E0B8F152
:10769800FF3FF2D0FBF708FAC01B4045206802D82C
:1076A800B8F1000F1DD150E8003F23F4D07340E833
:1076B8000032002AF7D100F1080353E8003F23F015
:1076C800010300F1080141E80032002AF3D1202328
:1076D800C4F88830C4F88C3084F884200320BDE8CE
:1076E800F08103685A07C7D5C3691B05C4D54FF491
:1076F8000063036250E8003F23F4D07340E800328F
:10770800002AF7D100F1080353E8003F23F00103F2
:1077180000F1080141E80032002AF3D12023C4F81F
:107728008830C4F88C30C4F89030D5E773B5044677
:107738000026C0F89060FBF7B7F923681B681A07A2
:10774800054619D423681B685B070AD56FF07E438A
:10775800009300222B464FF480012046FFF784FF58
:10776800B0B900202023C4F8883084F88400C4F815
:107778008C30E06620670CE06FF07E430093324661
:1077880003464FF400112046FFF76EFF0028D9D0BA
:10779800032002B070BD10B5044650B3D0F888304D
:1077A8001BB980F88430FBF735FB22682423C4F822
:1077B8008830136823F0010313602046FFF7E8FDC3
:1077C800012816D0A36A13B12046FFF7F9FE2368F3
:1077D8005A6822F490425A609A6822F02A029A6003
:1077E8001A6842F0010220461A60BDE81040FFF70F
:1077F8009DBF012010BD000030B581658168A0F8EB
:107808005C200023B1F5805FA0F85E20436735D186
:107818000369002B40F2FF1318BFFF23A0F8603064
:107828000023C0F890302223C0F88C30016801F1A1
:10783800080353E8003F43F00103083141E80034EE
:107848000368002CF2D1456E84680169B5F1005FC8
:1078580034D1B0F86850954230D8B4F5805F1DD166
:10786800254A264C002918BF22464267C1B153E871
:10787800002F42F4807243E80021F7E729B9036931
:10788800002B14BF7F23FF23C8E7B1F1805FC5D168
:107898000369002B0CBF7F233F23BFE7174AE4E7A8
:1078A80003F1080252E8002F42F0805203F1080069
:1078B80040E800210029F3D1002030BDB4F5805FF5
:1078C8000FD10F4A0F4C002918BF2246426751B109
:1078D80053E8002F42F4907243E800210029F7D1C1
:1078E800EAE7084AF2E753E8002F42F0200243E8AB
:1078F80000210029F7D1DFE7017200086570000850
:10790800A16F0008D56E0008D0F88C30202B30B459
:1079180015D1B9B1B2B100230468C3660A4B9C42C1
:107928000AD063681B0207D554E8003F43F0806320
:1079380044E80035002DF7D130BCFFF75DBF0220C9
:1079480030BC70470120FBE700800040436E30B533
:107958002BB90123A0F86A30A0F8683030BD03685D
:10796800094D9A689968094C490FC2F342626B5CE9
:10797800615CDB00B3FBF1F3A0F86A30AB5CA25C9E
:10798800DB00B3FBF2F3E7E7E0100108D8100108C9
:107998007047704770471FB504AB03E9060090F8BD
:1079A8008430012B04463AD0012380F88430242304
:1079B800C0F8883003681A6822F001021A609A68D1
:1079C80022F440120A439A6071B95A68BDF80C0053
:1079D8009DF80E1022F0100202435A605A6822F0F5
:1079E8007F4242EA01625A601A6842F001021A6054
:1079F800FBF75AF86FF07E42034600924FF480017D
:107A080000222046FFF730FE38B92023C4F888301A
:107A1800002384F8843004B010BD0320F8E7022066
:107A2800F9E790F88430012B0FD0012380F88430D7
:107A3800016851E8002F42F0020241E80023002BC0
:107A4800F6D180F88430184670470220704710B588
:107A580090F88430012B044617D02423C0F88830CE
:107A680003681A68196821F00101196042F0005290
:107A78004FF0005141661A60FFF768FF2023C0F8F5
:107A88008830002084F8840010BD0220FCE770B51F
:107A980090F88430012B044617D005682423C0F8D9
:107AA80088302E682B6823F001032B60AB6823F025
:107AB80060431943A960FFF749FF20232E60C0F8EF
:107AC8008830002084F8840070BD0220FCE770B57F
:107AD80090F88430012B044617D005682423C0F899
:107AE80088302E682B6823F001032B60AB6823F0E5
:107AF80060631943A960FFF729FF20232E60C0F8AF
:107B08008830002084F8840070BD0220FCE7000063
:107B180038B5084D052455F8043B2BB9013C14F041
:107B2800FF04F8D1204638BDDB6898470028F5D017
:107B3800F9E700BFD8070020034BD870034B1B6838
:107B48001B6C03B118477047EC070020D4070020CE
:107B5800034B1874034B1B685B6C03B118477047E1
:107B6800EC070020D4070020F0B5314D314B95F9D2
:107B78000420314E91B00C46012795F905108DF877
:107B8800047002288DF809208DF80A1010D18DF89C
:107B98000800D8711C7202F09FFD337803B114B14C
:107BA80001A803F003FA254B059A1A6011B0F0BD3D
:107BB80059714FF480711A71D9801C7233788DF81D
:107BC800087053BB1F2306A88DF81C208DF81830A9
:107BD80002F064FF20238DF8183006A82B798DF861
:107BE8001C3002F05BFF22238DF8183006A86B7951
:107BF8008DF81C3002F052FF21238DF8183006A8AA
:107C08006B798DF81C3002F049FF29238DF8183064
:107C180006A80B4B079302F041FF02F05DFD01231C
:107C280006A88DF818308DF81C3002F037FFB4E73D
:107C3800EC070020C0000020C8070020CC07002067
:107C4800000400017FB5092301A88DF8043003F072
:107C5800ADF90038044B059A1A6018BF012040425C
:107C680007B05DF804FB00BFCC07002070B50446E0
:107C78000B46134962784A700020A2780A7208708D
:107C88001A884A729A788A72DB780B746368CB60B8
:107C98000C4B1B68DA6A2AB1237803F0FB030A2B22
:107CA80000D09047084E052556F8043B1BB15B6A87
:107CB8000BB120469847013D15F0FF05F4D170BD82
:107CC800CC000020D4070020D807002070B5044657
:107CD80010480123037063784370A3788372E368C4
:107CE800C360E378037623694376237943720A4BAA
:107CF8001B689B6A03B19847084E052556F8043B54
:107D08001BB19B690BB120469847013D15F0FF0553
:107D1800F4D170BDE0000020D4070020D80700206F
:107D2800014B1868704700BFCC07002000B58BB026
:107D3800012368468DF8003002F088FD38B99DF8B7
:107D48000400003818BF01200BB05DF804FB0020C8
:107D5800FAE7000008B501F073FE48B9FFF7E6FF3F
:107D6800012806D0054BD879197AFFF7FDFE0120C6
:107D780008BDBDE80840FFF7CBBE00BFC00000202B
:107D88002DE9F04186B005460E46174601F058FE2B
:107D980000287FD101F06CFE044640B9FFF7C6FF0A
:107DA800012807D03D4B197AD879FFF7DDFE6FF02F
:107DB800020462E0DFF8E88088F80860003E18BF37
:107DC80001268DF80460374E687833798DF81230C3
:107DD800694602F0D9FC00283ED08DF8044003948F
:107DE800ADF810406FF0060495E803002E4B83E8C9
:107DF8000300337988F80A30394601A803F0DAF924
:107E08002A4B059A1A60112841D801A353F820F08B
:107E1800777E00089D7E0008977E0008977E000800
:107E2800977E0008977E0008977E0008B77D0008B7
:107E3800977E0008977E0008977E0008917E0008CC
:107E4800977E0008977E00089D7E00089D7E0008AA
:107E58009D7E00088B7E00082B788DF808306B78A3
:107E6800ADF810306B6803934FF0FF34BCE7104B4C
:107E780000221A70E31D18BF1446204606B0BDE85C
:107E8800F0816FF00404F8E76FF00504F5E74FF0B0
:107E9800FF34F2E76FF00104EFE700BFC0000020F5
:107EA800E0000020EC070020F0000020CC070020B4
:107EB800D007002037B501F0E5FD144D052455F82D
:107EC800043B5BB11B694BB155F8043C9B682BB173
:107ED800984718B155F8043C1B699847013C14F0C1
:107EE800FF04ECD1FFF714FE68B9094D2B7853B1A4
:107EF800084BADF80040D978019422466846FFF750
:107F08003FFF00B92C7003B030BD00BFD807002078
:107F1800D0070020EC07002030B58BB0054601F0F3
:107F28008FFD0446002839D1FFF700FF012838D11A
:107F380068468DF8004002F089FC10B14FF0FF3020
:107F480004E09DF80430AB4202D100200BB030BDF4
:107F5800012DF3D0022D11D0002DF7D1002BF4D034
:107F680068468DF8045002F099FD0028E6D10E4BC2
:107F78001B681B6B002BE8D09847E6E7002BDDD188
:107F880068468DF8045002F089FD0028D6D1064BCA
:107F98001B681B6B002BD8D02846EDE76FF001005B
:107FA800D4E76FF00200D1E7D407002010B50446EB
:107FB8008AB018B94FF0FF300AB010BD00236846E8
:107FC8008DF8003002F042FC0028F3D19DF804300F
:107FD8002370F1E77FB500220B4620498DF8072072
:107FE80001220A7042784A700446002A33D1027985
:107FF8000A721A884A729A788A72DB780B74036953
:10800800CB60C378164D8DF80830037B8DF80930A6
:10801800836803932B68DB6A0BB102A898472B6827
:108028009B6B13B1227E02B198470E4E052556F878
:10803800043B1BB1DB690BB120469847013D15F0A5
:10804800FF05F4D10DF10700FFF7B0FF637913B115
:10805800054B01221A7004B070BD00BFCC0000208F
:10806800D4070020D8070020D007002010B5044608
:108078008AB018B94FF0FF300AB010BD2023684607
:108088008DF8003002F0E2FB0028F3D1024A9DF996
:10809800043023701371EFE7EC07002000B58BB0B4
:1080A8002323019068468DF8003002F0F7FC003871
:1080B80018BF012040420BB05DF804FB70B5654C59
:1080C80001468EB01822204606F0FEF8624B0022C8
:1080D8001A70FBF759FF23784068012202FA03F16E
:1080E800014004D15D4B084608F0E4F8FEE75C491E
:1080F8005C481A4602F032F918B14FF0FF300EB062
:1081080070BD272304A88DF8103002F0C7FC564E26
:10811800564D002870D1012333702B68DB690BB1F1
:1081280000209847272304A88DF8103002F08EFB12
:10813800059B93F84820227093F8182193F81A3178
:108148006270A370464BD3E9020105F0AFFF054604
:108158000028D2D1464E062304A88DF8103002F02C
:1081680075FB059B736104A802F098FC022304A820
:108178008DF81030059602F069FB0836032304A831
:108188008DF81030059602F061FB0F2606F052F8C4
:10819800012304A88DF814308DF8106002F07EFCDD
:1081A80010230DEB03008DF810308DF8145002F0F9
:1081B80075FC04238DF8103004A8A3788DF81430CA
:1081C80002F06CFC3A238DF8103004A8636905931B
:1081D80002F064FC02A920788DF8086004F0E8F841
:1081E800003818BF0120E0711420FFF757FFE0792D
:1081F80003F0A4F9284682E728238DF810302B686D
:108208001B6943B104A802F021FB2B6805981B6980
:1082180040F2C4519847272304A88DF8103002F083
:108228003DFC50B9012304A88DF8103002F00EFB74
:108238009DF81430002B7FF46EAF3378002B7FF459
:108248006CAF052204A88DF81020059302F026FCD7
:1082580078E700BFEC070020D0070020E8100108ED
:10826800140800202C080020C8070020D40700208C
:10827800B007002037B500230D4601930446D0B956
:1082880000F0A8FB0190019BD3B10F4A42F82430BB
:108298000E4A9A620E4A1268916B1963916C59637F
:1082A80092690C49D9625A6128465B680A49F222E8
:1082B8009847002006E001A900F092FB0028E2D0D0
:1082C8004FF0FF3003B030BDD8070020717B0008A5
:1082D800D40700204D7C0008BC060020194B07B5C8
:1082E8001860194B194A1A60194A5A60194A9A6053
:1082F800194ADA60194B02681A6042685A60826843
:108308009A60C268DA60164A1A6182695A61154B26
:10831800C26B5A60144A019119609A601946134A4F
:10832800DA600020FFF7A6FF48B901A800F056FB65
:10833800003818BF0120404203B05DF804FB4FF03D
:10834800FF30F9E7D40700202C080020D57C00086E
:10835800DD7F0008F5830008757C000814080020FC
:1083680069C3000804080020417B0008597B000805
:1083780051B118B1012804D000207047044B0B609C
:108388007047044B0B60F7E74FF0FF30704700BFB2
:10839800000400010100010208B503F0EBF8002811
:1083A80014BF6FF00100002008BD08B502F0BCF949
:1083B800002814BF6FF00100002008BD10B5044666
:1083C8008AB018B94FF0FF300AB010BD21236846B3
:1083D8008DF8003002F03AFA0028F3D1024A9DF9EC
:1083E800043023705371EFE7EC0700202DE9F041CA
:1083F8002E4D2F4F00232B7043786B703B689B6A80
:108408008AB004460BB128469847DFF8A8800526AD
:1084180058F8043B1BB11B6A0BB120469847013E34
:1084280016F0FF06F4D12378052B2FD00B2B35D06F
:10843800012B25D1204C062368468DF8003002F028
:1084480005FA0199E07905F077FE10B91B4B019AFE
:108458005A611B48FFF70AFE1A48FFF7AFFF6B780F
:108468008BB9A371184B5878FFF756FD3B685B6AC8
:108478000BB1114898476B7813B9E07905F0ECFE19
:108488000AB0BDE8F081FF23A371EFE70F4B01228B
:108498005A74227A9A74627ADA74F1E76378002B54
:1084A800EED00AB0BDE8F041FFF7CCBBE0000020F9
:1084B800D4070020D8070020C0000020B007002003
:1084C800C4000020C5000020EC070020CC000020DC
:1084D80030B58BB0FFF769FF0446F0B903F048FFE9
:1084E800831C1DD0F8B9134D2B685B69DBB12723BA
:1084F80068468DF8003002F0A9F92B6801985B698D
:108508004FF4B961984703F045FF78B92CB9094B86
:108518001B68DB690BB10120984720460BB030BDC2
:108528006FF00704EFE74FF0FF34ECE74FF0FF344C
:10853800F3E700BFD4070020014B1878704700BF4D
:1085480040080020014B5878704700BF40080020C1
:1085580070470000044B9A7A0AB101225A70034B03
:108568005B6903B11847704740080020FC000020F1
:1085780073B5224C6378002B33D008F085F9666810
:108588000546FFF7CDFB0644AE4214D2A37A93B159
:10859800E0228DF800208DF80130217AE3680193FC
:1085A80001226846FFF7ECFB08B1073010D1002321
:1085B8006370A372656094F83430EBB1002384F8DB
:1085C80034300F4B5B6BBBB102B0BDE8704018474D
:1085D80040F2DC510B4808F023FA0A4808F0E6F9A3
:1085E800E8E794F83520002AE5D094F8360084F8B6
:1085F8003530FFF791FCDEE702B070BD400800207F
:10860800FC0000207808002037B5104D104CC8B188
:10861800C1B10123627200222860E16023700D4815
:108628000D4B00924FF0FF3108F014F900250B486C
:1086380025822022294605F05BFE6570A574A58673
:1086480003B030BD00232B602370EFE73C08002007
:1086580040080020780800205D85000854080020A4
:108668002DE9F0478E4C23788CB0002B56D0C27879
:108678000AB9837B13B1238A01332382437B002BFE
:108688004CD0E02A4AD10023A372876897F800806B
:10869800B8F1220F27D8B8F1220F30D8DFE818F048
:1086A8004100FB0052005A0061006E0075008E0008
:1086B8009D00B400C7002F002F002F002F002F00AF
:1086C8002F002F002F002F002F002F002F002F002A
:1086D8002F002F002F002F002F002F002F002F001A
:1086E800C900D000D400B8F17E0F00F0CC80B8F1FA
:1086F8007F0F00F0DF80B8F17D0F00F0AB80A57A26
:10870800002D00F05B81674C637A3BB94FF47A71B6
:10871800204608F085F9204608F048F90CB0BDE875
:10872800F087E36801220021A2721970A37AE16838
:108738009818A0720620C854A37AE1689818A07205
:10874800CA54DCE7584B9B6A002BD8D00121022081
:108758009847D4E77B7884F83630012384F835309D
:10876800CDE704238DF804307B78003B18BF012344
:1087780001A88DF8083002F091F9C0E77878003840
:1087880018BF012002F0DAFEB9E7484E0FCE01AD5E
:108798000FC50FCE0FC596E8070085E807007B7860
:1087A8000A2BACD8424A12685268002AA7D00CA9F2
:1087B80001EB830353F82C0C9047A0E77878431E0D
:1087C800012B9CD83A4B01381B6818BF0120207236
:1087D8009B68002B93D0984791E7E2680123082112
:1087E800A3721170627A057BA17AAA4228BF2A4631
:1087F800934284D285685A1CEB5CE56801334E1CB1
:10880800A6726B54D3B2EDE7E3680122A272092283
:108818001A70A37AE268218A581CA072D154A27AED
:10882800238AE1681B0A501CA0728B5467E72382D5
:1088380065E705238DF8043001A802F0B7FB5EE771
:10884800194BDB6A98475AE7194B78781B686075AB
:10885800DB68BEE7037B072B7FF451AF06238DF857
:108868000430B7F80130ADF808307B793A791B0449
:1088780043EA0223FA781343642253430393BB79F0
:108888008DF81030D8E73B2201A88DF804208DF828
:10889800083002F003F9012384F834302FE700BFD1
:1088A8004008002078080020FC000020EC0E010899
:1088B8003C0800202A2301A88DF8043001F0C6FFE7
:1088C80094F80A90E6689DF808009DF809509DF80C
:1088D8000A709DF80BC09DF80D309DF80E209DF88C
:1088E8000F109DF80CE009F1010A84F80AA006F8B7
:1088F8000980354E94F80A903668D4F80C8009F14E
:10890800010A84F80AA096F803A008F809A094F8C8
:108918000A90D4F80C8009F1010A84F80AA096F8A4
:1089280002A008F809A094F80A90D4F80C8009F17C
:10893800010A84F80AA096F801A008F809A094F89A
:108948000A9009F1010A84F80AA096F80080E668FE
:1089580006F8098094F80A80E66808F1010984F8A5
:108968000A9006F808C094F80AC0E6680CF10108F5
:1089780084F80A8006F80C70A77AE66807F1010CFB
:1089880084F80AC0F555A57AE6686F1CA772705579
:10899800A07AE568461CA6722954A17AE0684D1CA5
:1089A800A5724254A27AE168501CA0728B54A37A33
:1089B800E268591CA17202F803E0A0E6034807F038
:1089C800A7FF6570AAE600BF3C08002078080020D1
:1089D8007047000000487047FC00002000207047E6
:1089E8004FF0FF3070470000044B054A93F81831E8
:1089F800022B18BF062382F890347047540E0020CB
:108A08001C140020034BD3F8483313B15B6903B13E
:108A1800184770471C140020034A137843F00403D6
:108A28001370FFF7EFBF00BF181400201FB50A4BE3
:108A38008DF8090093F87C208DF80A2093F88C2093
:108A480093F848000D3202A98DF8082003F0B0FC15
:108A5800C0B205B05DF804FB540E002010B5074CF9
:108A680004F5806007F054FF94F81A3413B1012319
:108A780084F81934BDE81040FFF7C4BF1C14002067
:108A880010B50C4CD4F8403343F08003C4F840339D
:108A980094F81A3413B10020FFF7E0FF94F89134EA
:108AA80023F0120343F0120384F89134BDE8104018
:108AB800FFF79ABF1C1400202DE9F041DFF8AC80C5
:108AC80098F81831022B06460D4602D0284BDB6A6F
:108AD800984702F0E9FD044628B1022002F0DAFDC9
:108AE800002002F0DCFD98F81831012B17D102F0B4
:108AF800DDFD074630B1002002F0CDFD002002F078
:108B0800CFFD3C4602F0D4FD48B1002002F0C4FD80
:108B1800002002F0C6FDBDE8F041FFF765BF002C5C
:108B2800F9D1144C94F8902494F81A34BAB90BB1CA
:108B380084F84164304602F065FFD8F82C0007F04D
:108B4800ADFED4F8B4339842E5D30B4807F0E0FE05
:108B580094F8913443F0100384F89134DBE70BB1B7
:108B680084F84154284602F04DFFF1E7540E0020E6
:108B78006C1801081C140020B417002073B5164C9B
:108B8800164D04F57A76EB6C95F8502095F9781027
:108B980095F84800009603F031FC95F8303184F8D8
:108BA800FC3395F8480040F2012304F22442314690
:108BB800A4F8FA3303F02EFC58B194F8243484F85E
:108BC8006A34074B00205B6B984794F8FB3384F8B2
:108BD800903402B070BD00BF1C140020540E002059
:108BE8006C180108074A10B5137843F00203137094
:108BF800FFF708FFBDE81040034B012200210220C7
:108C080007F058BB1814002031110108074A10B5A5
:108C1800137843F008031370FFF7F4FEBDE8104023
:108C2800034B01220021022007F044BB1814002046
:108C3800411101082DE9F0410F4616461D468046B0
:108C480007F022FE0B4A0C4C1378278123F01103FE
:108C580043F011031370C4E9000866812573FFF718
:108C6800D1FEBDE8F041054B01220021022007F0AA
:108C780021BB00BF18140020C81900205111010899
:108C880013B507F001FE0D4B6C461860204607F03F
:108C98004FFD94E803000A4A0A4B83E8030013785F
:108CA80043F020031370FFF7ADFE074B01220021AC
:108CB800022002B0BDE8104007F0FCBAD819002025
:108CC80018140020541700205E110108F8B5334D20
:108CD80095F81841012C06464BD0022C51D064B9A6
:108CE80038B9D5E91B0105F1740383E80300204670
:108CF800F8BD01283DD0022801D00324F7E7284F0A
:108D080085F8180107F5747EBEE80F0007F57A7C30
:108D1800ACE80F009EE8030095F8E9308CE8030002
:108D280087F8FB63E3B195F80031022B18D1D5F829
:108D380004316B67C7F8EC3395F87D3095F8082156
:108D480087F8F83395F88C3085F8782087F8F93368
:108D580097F81B2487F8E82340F20133A7F8FA3381
:108D6800002387F81A340F4BDB6A9847FFF706FF92
:108D7800BDE702F0A4FC04460028B8D185F81861C4
:108D8800B5E70028B9D1064B85F81801062283F803
:108D98009024044BDB6A98473446A8E7540E002019
:108DA8001C1400206C1801082DE9F04192B0064609
:108DB80002F07AFC002840F05981AD4D95F8183141
:108DC800012B09D02B6BAB4C93B194F80431BBB198
:108DD800042B6FD0032003E002F068FC18B10F20C9
:108DE80012B0BDE8F08102F063FC0028EAD0F6E793
:108DF800B5F82031D4F81C24013B53432B63E4E736
:108E08009D4803F00CFA002840F02C8194F80C31AE
:108E180023802B6B0C930DF1180895F839308DF8D9
:108E28003830404695F81C318DF83A3007F0A6FCEA
:108E3800D5F82831009302AF98E80600D5F8243118
:108E4800384607F032FC97E803000FAB83E80300CD
:108E5800EB6A0D9300238DF844302388ADF8463033
:108E680095F8303101228DF839201BB98DF844204E
:108E78008DF83930814B0093814B95F84800A3F168
:108E880079020CA903F009FBC0B10B28A8D1D4F8CA
:108E9800941499B1002EA3D0D4F84033794843F004
:108EA8002003C4F8403307F0BBFD764807F07EFD89
:108EB800002095E7704803F0E6F9A4E795F84870B4
:108EC80095F9693095F9392095F87D106E4E384638
:108ED80003F0F0FA009641B2EB6C95F85020384652
:108EE800183603F08BFA0096EB6C95F8502095F93C
:108EF800701095F8480003F081FAD4F8C413AB6DEC
:108F0800D4F8DC230B44C4F8B033EB6D1344C4F835
:108F1800B43394F80431042B07D02B6E0B44C4F8F7
:108F2800B0336B6E1344C4F8B4330023089395F838
:108F3800303183B108A802F095FC00284ED195F98C
:108F4800390094F837629DF82070FFF76FFD3E44B2
:108F580080B2B04240D300238DF8133095F83930F1
:108F68008DF8213095F838308DF82230D5F88030DA
:108F78000993D5F884300A932388ADF82C3095F8F6
:108F8800303194F81B648DF82E3095F848003F4B2B
:108F98008DF820600DF1130208A903F043FA0123AC
:108FA80084F8413495F8393084F842349DF8133008
:108FB80084F84334D4F81C34C4F85064C4F84834F2
:108FC800C4F8583402F076FB50B1D4F81C0402F00F
:108FD80083FB28B1102003E7082001E71320FFE6F0
:108FE80095F81831012B01D102F078FB02F065FBEE
:108FF8000023059394F8043195F9395094F81B64CB
:109008009BB1042B7FF4E6AE05A802F067FE58BBBF
:1090180094F8183413B1059B013B0593164B05983A
:109028003246E9B202F0C0FE02E0134802F090FEB8
:10903800C0B9D4F8403394F80C11218043F00203EE
:10904800C4F8403394F8183411480133DBB284F87B
:10905800183484F845340F4B00259B6AC4F898549B
:10906800984725E71120BBE61220B9E60E20B7E69F
:10907800540E00201C14002024150020840E00200B
:10908800B018002084170020D417002038180020BA
:109098001E1400206C180108F0B5504C504EB4F85E
:1090A800DC202287D4E92D0194F8B12084F86920C6
:1090B80004F16C0282E80300D4E92F0104F1740280
:1090C80082E80300B4F8C420A4F87C2091B0D4F856
:1090D800CC20D4F8C810C4F884200025D4F8D020B7
:1090E800C4F888200123A4F82031C4F8801084F83B
:1090F8003051A56284F81B5184F83A5084F81D5108
:1091080084F81E51C4F83451C6F89854A6F8185477
:1091180086F81A54A4F838518DF8183004F50973F4
:10912800039304F50A7394F84800A4F8465104938D
:1091380003A92C4B84F84551C4E94F55059303F016
:1091480045F9E36EC6F8D43394F87D3086F8E033F9
:1091580094F88C3086F8E1334FF48073A6F8E23344
:1091680086F8D05394F8303186F8E43306F57477EE
:109178000FCF06F57A740FC497E8030040F2012375
:1091880084E80300A6F8FA33D6F8483386F81B5467
:10919800CDE901551BB15A685B6901920293124BE4
:1091A8000793A3F148020892A3F1140209920F4A07
:1091B8000B9229330A93A2F19C030C93A2F1980312
:1091C8000D93131D0E9301A902F14C0307A802F594
:1091D80099620F9302F05DFA11B0F0BD540E0020B1
:1091E8001C1400203819002084180020380F002093
:1091F800F8B50D4F0D4C0E4E0D4607F089FB3B6B35
:10920800984796F8480004F22442294603F002F9E8
:1092180048B194F8243484F86A34706D7B6B9847AD
:10922800EB7C84F89034F8BD6C1801081C140020FD
:10923800540E00200F4890F81B3480F8B8330E4BBA
:1092480093F8692080F8BB2393F87D2080F8C82321
:1092580093F88C2080F8C92393F8303180F8CC3308
:109268000022A0F8CA2300F56E7100F56070FFF7C0
:10927800BFBF00BF1C140020540E0020114890F8F6
:109288009034EBB190F81B3480F8D0330E4BDA6E83
:10929800C0F8D42393F87D2080F8E02393F88C203D
:1092A80080F8E12393F8303180F8E4334FF480728A
:1092B800A0F8E22300F5747100F56670FFF798BF17
:1092C800704700BF1C140020540E002070B5344CA9
:1092D8002421204605F00EF8636A984218BF6062A0
:1092E8004FF01C012F4814BF0125002505F002F896
:1092F800636C984218BF60644FF480712A4818BFA5
:1093080045F0020504F0F6FFD4F84831984218BF3A
:10931800C4F848014FF0D401244818BF45F00405AB
:1093280004F0E8FFD4F82032984218BFC4F82002AD
:109338004FF000011E4818BF45F0080504F0DAFF99
:10934800D4F82432984218BFC4F824024FF460714C
:10935800184818BF45F0100504F0CCFFD4F8A8351C
:10936800984218BFC4F8A8054FF01401124818BF56
:1093780045F0200504F0BEFFD4F8C03598420F4BE5
:1093880018BFC4F8C005D3F8483318BF45F04005E6
:109398002BB11B691BB12846BDE87040184770BD4A
:1093A800540E00207C0E00209C0E0020A00F0020F0
:1093B800781000207C100020001400201C140020CD
:1093C8002DE9F04F91B04FF00008012B05460F46EC
:1093D80002928DF81580ADF8188003D8C84EC146A2
:1093E800B94502D311B0BDE8F08F15F8090002F0B5
:1093F80077FA4844B842F5DC15F8093009F1010458
:10940800023BE4B2112BEDD801A252F823F000BFC1
:10941800619400089394000893950008BD9500088E
:10942800459600086D960008DF9600081197000819
:109438008D970008ED930008ED930008EB9700085E
:10944800ED930008ED930008A9980008D19800084A
:109458001599000853990008052002F0EDFA90B11B
:109468000521002002F0ACFA2A5DA64B09F103049D
:1094780009F102095FFA89F983F85C2415F80920D3
:1094880083F85D24E4B2A146AAE700238DF81630DC
:109498008DF817308DF81C308DF82030B8F1000F9A
:1094A8006CD14FF0050896F87C208DF83920631EA2
:1094B80096F839208DF83B202B4496F838200D93E8
:1094C8008DF83C2096F81A3196F868208DF83D20E2
:1094D800D6F82C218DF83A300C9273B37B1C1B1BE9
:1094E800DBB28DF8383008AB019307AB009396F8E0
:1094F80048000DF117030DF116020CA902F09EFFAA
:109508008DF8150000F00700072813D196F93920C7
:109518009DF9163086F839309A429DF8173086F84A
:109528003830B8BF01229DF81C30B8BF86F81D211D
:1095380086F868304FF0000909E00523D1E70122D9
:109548000DF11501032002F0DBF809F101095FFABA
:1095580089F29DF82030B3FBF8F19142EFD823440B
:10956800DCB2631EDBB29F420DD9EA5C032A9AD0B3
:10957800A74288BF1C464FF0010884E709F1050996
:109588005FFA89F4F7E71C46F5E72B5D012203F043
:109598000F0309F1020986F81B3102FA03F35FFA97
:1095A80089F9A6F82031002206A9042002F0A8F8BB
:1095B8004C4668E707238DF815302B5D96F8480070
:1095C800C3F3021203F00F038DF8303009F10303DF
:1095D800DBB28DF83120EA5C09F10403DBB209F152
:1095E8000504EB5C09F102095FFA89F91B0443EAF7
:1095F800022315F809201343642253430CA90D9341
:1096080002F02BFF00F00703072BE4B28DF81500DA
:109618000CD19DF8303086F8703086F878300D9B84
:10962800F36673679DF8313086F869308DF8180055
:10963800012206A9052002F063F824E7314BD3F88C
:1096480048336BB11B685BB19847029B8DF81800D3
:1096580003F03F038DF81930022206A90620EAE735
:10966800FF20F2E703238DF815302B5D8DF82430A9
:109678000CAB089309F10303DBB209F10604EA5CB9
:1096880096F8480009F10403DBB208A9EB5C1B0457
:1096980043EA022309F10202D2B209F10509AA5CE0
:1096A8001343642253435FFA89F90C9300230D9303
:1096B80015F809308DF8383002F0D5FEC3B200280D
:1096C800E4B28DF81530FFF6DEAE8DF818300122C1
:1096D80006A90720AFE72B5D03F00F03012B4FF41A
:1096E8007A7238BF0123534309F10209B365134461
:1096F8005FFA89F9F365002206A9082056E700BF3A
:10970800540E00201C1400202B5D96F84800C3F36B
:1097180040128DF81D2007A9C3F3001203F00F03B0
:109728008DF81C208DF81E3002F0A3FE09F1020905
:1097380001305FFA89F93FF43BAFBDF81C30914A1C
:10974800A6F87C309DF81E309DF81C40D05CF8F7D8
:109758005DF90223C6F880000CA996F848008DF838
:1097680030308DF8324002F023FE96F939300890F7
:1097780040B29842B8BF184686F83900002206A9B8
:10978800092013E703238DF815302B5D8DF8303051
:1097980009F10303DBB209F10504EA5C96F8480015
:1097A80009F10403DBB209F10209EB5C5FFA89F9FC
:1097B8001B0443EA022315F8092013436422534388
:1097C8000CA90D9302F05BFEC3B20028E4B28DF839
:1097D8001530FFF658AE8DF81830012206A90A2078
:1097E80029E7092002F028F9DFF89CA1002854D0C5
:1097F8000921002002F0E4F80023ADF8263009F131
:109808000203DBB24FF47A71EA5C09F10303DBB2BD
:109818000DF1300BEB5C1B0443EA02232A5D134372
:1098280009F10402D2B209F1060409F10509AA5C9A
:109838005FFA89F943EA026315F8092003934A435A
:1098480012125846ADF8242006F072FF039B03F16C
:10985800965303F5A91303F5EC530893DAF83C3350
:1098680000930DF1200999E80600DAF838330AA8C0
:1098780006F01BFF0B9B00939BE806000A9B4846DB
:1098880006F0F8FE99E8030006F02AFF01F021FF30
:109898000123E4B28AF83834F5E58AF83804F2E5A9
:1098A8000C2002F0C9F800283FF4EDAD0C2100208F
:1098B80002F086F8344B93F89034043B012B7FF682
:1098C800E2AD01F002FFDEE509F10203DBB22A5D39
:1098D800E95C09F10303DBB209F10504EB5C09F16A
:1098E80004095FFA89F91B0415F8090043EA012302
:1098F80013436421594300F00F0001F0E7FEE4B27E
:109908008DF81800012206A9112094E60D2002F016
:1099180093F800283FF4B7AD0D21002002F050F86D
:1099280009F10203DBB2194AE85C2B5D126809F100
:10993800040409F103095FFA89F943EA002015F8DC
:109948000910E4B201F0C4FE9DE52A5D09F10203A5
:1099580009F1040409F10309DBB25FFA89F9E95C4A
:1099680015F809301B0443EA0123134364205843C4
:1099780001F0B0FEE4B28DF81800012206A9132008
:1099880059E600BF6B1101081C140020C8190020FB
:109998000E4B93F89124920703D593F88F24012A4C
:1099A80008D90B4991F81A2122B18A6A501C18BFAC
:1099B80001328A620022A3F8182483F81A24D3F803
:1099C800402322F00202C3F8402370471C140020F1
:1099D800540E002070B5184C184D04F55A7006F056
:1099E80097FFD4F84033D4F89804D5F8906023F062
:1099F8002003C4F8403338B106F050FF864203D242
:109A0800002385F83A3070BD0120FFF7CDF9002812
:109A1800F9D00B28F7D095F8393084F8423409206A
:109A280094F8183484F8453484F8410401F0EAFFC6
:109A3800BDE87040FFF7ACBF1C140020540E002096
:109A4800094BD3F84023012A0AD008490978C907E5
:109A580008D43AB993F89204013818BF0120704726
:109A680000207047012070471C14002018140020A3
:109A7800034BD3F84003431E58425841704700BF78
:109A88001C1400202DE9F04FA9B0EFF3108272B634
:109A9800DFF8F4820021D8F80030C8F8001082F30B
:109AA8001088BA4C002B00F0E480DAB29B060392CF
:109AB80064D5B74D95F81831022B02D0B54BDB6A47
:109AC8009847EFF3108972B6B34F06F0DDFE3E6893
:109AD800D4F8B013361A3144B04806F0A1FFAF48A5
:109AE80006F064FFD4F8B413AD48314406F098FF8B
:109AF800AB4806F05BFF89F3108894F81A34002B02
:109B080000F06D81152312A995F848008DF84830AA
:109B180002F04EFCD4F8B4130F900144A14806F0AB
:109B28007FFFA04806F042FF3B6894F81B24EB62D5
:109B38000DAF38468DF870201D9306F01FFED5F83E
:109B48002831009306AE97E80600D5F82431304650
:109B580006F0ABFD96E803001FAB83E80300D4F8DA
:109B68001C341E9395F8303195F84800003B18BF17
:109B780001231CA98DF8713002F023FC039BDF063A
:109B88004BD5834DDFF820A2D5F8E420BAF90A3086
:109B9800059298F800200493002363F300020A93C7
:109BA80088F8002084F84434049AA4F8223484F80D
:109BB8002534C4F82834A4F82C3484F82E34C4F896
:109BC800303484F82034C4F8343484F83834C4F891
:109BD8003C34704B9AF90C90A4F88C2494F8902497
:109BE800DB6A84F88E9484F88F24DAF80470BAF863
:109BF8000860984794F88F3413B9694806F088FECE
:109C08003146384601F04EFD8346002800F0EA80D0
:109C1800049BA4F87E3484F88094039B19071AD512
:109C28005B4B93F81831022B02D05A4BDB6A9847EA
:109C38000220FEF7D9FE84F8410401F0E3FE94F80F
:109C48001A3413B1012384F8193494F8913443F089
:109C5800100384F89134039B5A0703D50621052085
:109C6800FEF72AFF039B9B0703D504210320FEF779
:109C780023FF01F035FD94F89124D7065FD5002322
:109C880084F89234D4F840331E0644BF23F082038C
:109C9800C4F8403312F0050F00F0FC820B2001F0ED
:109CA800CBFE002800F0F68294F89134DD0700F12D
:109CB800F182580740F10883D4F8403323F00203B7
:109CC800C4F84033D4F8402382BB94F8915415F07B
:109CD80001011EBF2B4662F3000384F8913494F807
:109CE80091345E0744BF6FF3820384F891340123F3
:109CF80084F8923421B1D4F844332C481B6898472F
:109D08006D070BD52A4801F0A3FE01F0D1FE28B15A
:109D180094F8913443F0040384F8913401F0CEFCB4
:109D280094F891346FF3041384F89134012384F880
:109D3800923494F8913443F0200384F8913494F8E1
:109D4800913418070AD56FF3C3031A4984F891347C
:109D5800D4F84433A1F12400DB68984794F891348F
:109D680099070AD56FF34103124984F89134D4F85E
:109D78004433A1F16C005B68984794F89034022B47
:109D88001AD1FEF7FBFE17E0181400201C1400205F
:109D9800540E00206C180108D81900209C170020C8
:109DA800B41700201C180020C81900205C180020D7
:109DB80070180020A818002094F891349A0640F1F1
:109DC800C6826FF3451384F89134D4F84033002BDE
:109DD80040F0BD8229B0BDE8F04FFFF777BA84F8AC
:109DE8004134A1E695F81821012A0CD101F05EFC56
:109DF800804668B1584601F04EFC584601F050FCC8
:109E0800042384F88F347EB9012384F8213450E187
:109E180001F04EFC0028F6D0404601F03DFC4046DB
:109E280001F03FFC0523ECE73B7804935B09013B19
:109E3800062B00F21882DFE813F0070016029500DF
:109E48001602920016020702102EDDD995F830315D
:109E58001297F6B28DF84C60002BD5D11CA804F0EF
:109E68005DF912AA1CA9FF2002F0B2F89DF858303B
:109E7800C3F3030307468DF82C3095F8480095F88E
:109E88007D308DF82D3007220BA902F0A4FA002F9F
:109E98005DD100285BD09DF853309DF8522015996C
:109EA800C5F8E4101B0443EA02239DF85120022060
:109EB8001343C5F8E03004F03FF99DF8583095F8A1
:109EC800480085F82E71C3F30212C3F3030385F823
:109ED800703085F878309DF8593085F86920012B65
:109EE80038BF01234FF47A725343AB651344EB65D3
:109EF8000DF15A034FF001081093113E94F81B34EA
:109F08008DF83C300FA985F868808DF8446002F020
:109F18006AFA0223404685F8303101F08DFD18B108
:109F28004146384601F04CFD94F88F34012B00F27D
:109F3800A88194F81A34002B40F09B8194F891344E
:109F480043F0100384F89134FEF74EFD65E60120D6
:109F580001F072FD0028E7D001210720E2E7012384
:109F680084F8203495F87D308DF82E3094F8243418
:109F78008DF82D3095F88C3095F848000D330BA9E5
:109F88008DF82C3002F014FAA6F10D031BB20990DB
:109F980023EAE37300B283423FF736AF0B2E7FF616
:109FA80033AFBB4B25931CA8FF231C978DF8746017
:109FB8008DF8983002F0D8F8074600287FF424AFCF
:109FC80095F81831012B13D101F070FB002873D0DC
:109FD800384601F060FB384601F062FB04239DF827
:109FE8007C101E9884F88F34C1F3001101F077FBC0
:109FF8009DF87C301E99C4F8341413F00F0203D076
:10A008009DF89000002863D19DF89800002862D040
:10A01800002A7FF4F9AE9DF89020002A0CBF4FF07B
:10A0280002084FF0030800220A92D5F8EC2091426A
:10A0380054D195F8E910002950D0D5F80C1195F8AD
:10A04800EAB009680A9195F81811022902D103218A
:10A0580084F88F14B8F1030F7FF4D6AE13F0600FB5
:10A068007FF4D2AE0592012795F82E31BBF1000F8F
:10A0780037D0BBF1010F38D1012B34D16FF009066D
:10A0880046FA08F606F00106C6F10206F6B2BDF871
:10A098007E100AAA304601F02DFE40B307280CBFF7
:10A0A8000823012384F821340A9BC4F83034C4F807
:10A0B8006C34FEF7E5FCB0E501F0FAFA002897D019
:10A0C800384601F0E9FA384601F0EBFA052386E74D
:10A0D8004FF00008A7E74FF00108A4E74FF0010B85
:10A0E800C2E70426D3E70326D1E70123DAE71CAB4E
:10A0F800009305990A9B3246584601F0BBFE20B1F1
:10A1080002280CBF0A230B237FE60A9BC4F83034CD
:10A11800C4F86C349DF87C3084F82104C3F34013F0
:10A1280084F82E3484F8443494F88F3484F82274F4
:10A13800012B9EBF0122A86285F81E21012FC4F8B9
:10A14800280484F82C0484F8410438D1022284F8C5
:10A15800202495F83A20002A4AD19DF87C20D6067A
:10A1680046D4012B94F840149DF87C2005D8012989
:10A1780001D1900601D501F05FFBB8F1020F94F808
:10A188008F3443D0B8F1030F0AD09DF87C10B8F192
:10A19800010F4A4601F00F0120A83BD0FFF710F944
:10A1A8009DF8903084F82334259BC4F828349DF812
:10A1B800983084F82C34012384F82D3430E0049A44
:10A1C80002F0E002A02A1BD195F82E11012285F891
:10A1D8003A2009B927996963012B84F8202407D903
:10A1E800D5F89020C4F83C24DAF80020C4F8982464
:10A1F80095F81821002AB4D1012284F82524B0E763
:10A20800002285F83A2084F82024A6E79DF89810C3
:10A2180025984A46FFF7D4F89DF8903084F82334FF
:10A228009DF89020E02A08D195F81F312BB984F8C1
:10A238002324C4F82834A4F82C3494F8913443F037
:10A24800020384F891346FE6114D013EB2B2791CD5
:10A25800284604F039F80323A4F82034C4F8285415
:10A2680084F82C64E9E7012384F82134FEF708FC1C
:10A278005AE694F84434002B3FF460AE0020FEF711
:10A28800EDFB94F88F34022B3FF45EAE56E600BF28
:10A298005416002094F89134590715D5012001F07F
:10A2A800CBFB60B1012001F09DFB08B984F81804CC
:10A2B800D4F8403323F00203C4F8403304E0062006
:10A2C80001F0BAFB0028F3D194F89134DA077FF54E
:10A2D800F9AC94F840240AB1032A18D11D4A94F81D
:10A2E800181492F86820914205D29B0723D594F858
:10A2F8008F34012B1FD8184806F00AFBD4F84033D6
:10A3080023F02003C4F84033FFF742FBDAE4012AC4
:10A3180011D194F81924002A3FF4D4AC0D4A94F8CA
:10A32800181492F868209142E5D29F0703D594F853
:10A338004434002BDFD194F8913400206FF30413D8
:10A3480084F8913484F81904FFF744FBBAE429B07F
:10A35800BDE8F08F540E0020841700202DE9F04F3F
:10A3680089468DB090460746002800F08F81002965
:10A3780000F08C810368002B00F088814368002B73
:10A3880000F084818368002B00F08081C368002B73
:10A3980000F07C81104602F007F8002800F0788170
:10A3A800BD4CBE4D384601F0C1FA40F2C4520021FE
:10A3B800204603F09DFF40F21C520021284603F07E
:10A3C80097FFB74BC4F82C3104F50973089304F5CB
:10A3D8000A7300264046099308A9B24B84F84880BE
:10A3E8000A9384F8186184F88C608DF82C6001F069
:10A3F800EDFF0F2306A994F848008DF8183001F0F6
:10A40800D7FF801B18BF01204FF00A0B84F81C01EE
:10A4180006A994F848008DF818B001F0C9FF4FF06C
:10A42800060A84F8DC0006A994F848008DF818A0FC
:10A4380001F0BEFF102384F8DD0006A994F8480057
:10A448008DF8183001F0B4FF1123C4F89C0006A958
:10A4580094F848008DF8183001F0AAFF1223C4F8C8
:10A46800A00006A994F848008DF8183001F0A0FF64
:10A478001323C4F8A40006A994F848008DF81830EE
:10A4880001F096FF1423C4F8A80006A994F8480020
:10A498008DF8183001F08CFF1623C4F8AC0006A91B
:10A4A80094F848008DF8183001F082FF172384F8DB
:10A4B800B10006A994F848008DF8183001F078FF2B
:10A4C80018230DEB0301C4F8B400C4F8BC0094F8D9
:10A4D80048008DF8183001F06BFFC0B21D2384F8D6
:10A4E800B80084F8C00006A994F848008DF8183020
:10A4F80001F05EFF1E2384F8C40006A994F8480002
:10A508008DF8183001F054FF1F2384F8C50006A900
:10A5180094F848008DF8183001F04AFF2023C4F859
:10A52800C80006A994F848008DF8183001F040FFDB
:10A538000B23C4F8CC0006A994F848008DF818300D
:10A5480001F036FF0C2306A9A4F8D00094F84800BF
:10A558008DF8183001F02CFFD4F89C306365D4F8DE
:10A56800A030A365D4F8A430E365D4F8A8302366F6
:10A578004FF00108D4F8AC300590A4F8D200636617
:10A5880084F8B080C4F894B084F898A0C4F84CB0AB
:10A5980084F850A084F8688084F81F81C5F848932F
:10A5A800FEF77AFD404B009632464FF0FF3105F535
:10A5B8005A70C5F84473C4E90B6684F8198185F8A4
:10A5C8009164C5F8408306F045F9384B0096324649
:10A5D8004FF0FF3105F5607006F03CF9344B0096FA
:10A5E80032464FF0FF3105F5667006F033F902AFD9
:10A5F800304B009632464FF0FF3105F5806006F08B
:10A6080029F9384606F0BAF897E8030004F592737A
:10A6180083E80300284B294F1E60294BC5F84C33AB
:10A62800284BC5F85433284BC5F85C33274BC5F87D
:10A638005033274BC5F8583305F553703B68984796
:10A6480004F5A67003F088FB20B1112630460DB042
:10A65800BDE8F08F204601F01DFB0028F5D101F080
:10A6680041F8B8B91B4801F067FB06460028ECD151
:10A678007B69984703F006FEBB6D94F8190198476B
:10A68800FB6A9847012385F89234DFE70326DDE764
:10A698000926DBE71326D9E7540E00201C140020F6
:10A6A8000004000138190020DD9900083D920008D7
:10A6B80085920008658A0008181400206C180108A3
:10A6C800898C00083D8C0008218A0008158C000838
:10A6D800ED8B00083C0F002008B5034B0020C3F8A1
:10A6E8004003FEF781F908BD1C14002010B5FFF7E0
:10A6F800A7F90A4C60B90A4B93F81831022B02D11A
:10A70800084BDB6A98470123C4F84033002010BD8A
:10A71800D4F84003013818BF0120F8E71C140020C2
:10A72800540E00206C18010838B5134C04F55A7003
:10A7380006F0EEF804F5607006F0EAF804F56670C5
:10A7480006F0E6F804F5806006F0E2F800F0B5FFE0
:10A758000A4B0025DB6A9847C4F84053FEF7B6FD5C
:10A768000749084840F2C45203F0AEFD0123C4F87B
:10A778004033284638BD00BF1C1400206C1801085F
:10A78800540E00209008002070B52E4B8AB0054664
:10A7980093F8DD008DF8090093F8DC008DF80A00C5
:10A7A80029489A6A90F81804039200268DF80B003D
:10A7B80004960C46002940D00692D3F888200792C8
:10A7C8001A8F93F81A118DF8151052BAADF8202087
:10A7D80093F87C2093F848308DF8243003AB8DF83B
:10A7E80022008DF8232000930DF10A020DF10B03CE
:10A7F8000DF1090105A88DF8146000F0DDFE9DF942
:10A808000900FEF713F9607004A801F02BF8B0B93D
:10A81800049A0F2A0DD863789A420AD81544AB4295
:10A82800A3EB02012CBF002001202170C0000AB058
:10A8380070BD002323700820F9E70320F7E71320F1
:10A84800F5E700BF540E00201C1400201FB5044675
:10A85800002800F012810078412800F20881DFE822
:10A8680010F0420048004D00520056005A005F00A8
:10A878000601060106010601060106010601060198
:10A8880066006A006E0079008000830086008B00F5
:10A8980089008D009100940097009A009D00A00007
:10A8A800AF00B300BB00B700BF00C200C600CF00B6
:10A8B800CB00CD000601D300060106010601060102
:10A8C8000601060106010601060106010601060148
:10A8D800060106010601DB00DF00E300E800EC00EA
:10A8E800F000F400FD00674B93F81831237104B0B1
:10A8F80010BD644B93F83031237102E0606803F0B7
:10A90800C7FB0020F3E7606803F008FCF9E75D4B3C
:10A9180093F81A31F0E75B4BD3F8E0306360F0E767
:10A92800584B211D93F8300103F010FCE9E7554B13
:10A9380093F81931E0E7534B93F88C30DCE71C238C
:10A948008DF808304F4B02A993F8480001F030FD0C
:10A958006060D6E74C4B043493E8030084E80300B6
:10A96800CFE74A4B0434F7E7494B0434F4E7494B43
:10A978000434F1E71A23E3E71923E1E7414B93F89D
:10A988006830B9E73F4B5B6DC8E73E4B9B6DC5E749
:10A998003C4BDB6DC2E73B4B1B6EBFE7394B5B6E35
:10A9A800BCE702238DF80830364B02A993F87C20C7
:10A9B80093F848008DF80A2001F0FAFC2071A0E70E
:10A9C800304B93F8DD3097E72E4B93F8393093E707
:10A9D8002C4B93F8DC308FE72A4B93F838308BE711
:10A9E800284BDB6C9AE7274B93F8503084E7254BCC
:10A9F800D3F88430636084E7224B8FE7264B8DE7DA
:10AA0800204BD3F8CC30F5E71E4BD3F82C316360DC
:10AA180001F05CFDA06074E71A4BD3F890307DE735
:10AA2800184B93F81F3167E7164BB3F88830A380AB
:10AA380067E7144BB3F88A30F9E7124BB3F8D03014
:10AA4800F5E7104BB3F8D230F1E70E4B93F84820F6
:10AA58000AB1062A13D1B3F8A035E8E7094B93F8F1
:10AA680048200AB1062A0AD1D3F8A43556E7204669
:10AA780004B0BDE8104000F024BE032037E71820DA
:10AA880035E700BF540E0020C00E0020080F00203C
:10AA9800C80E0020100F0020900800207FB5044643
:10AAA80010B9032004B070BDA44DD5F840339A07FF
:10AAB80000F171820278412A00F26A82DFE812F01E
:10AAC8004200480056005C00600065006A0077009C
:10AAD800820088008E0094009A00A000A600AC00B6
:10AAE800B6006802BB00DD00F000170139012A0139
:10AAF80044014D015101550159015D01680261018F
:10AB080073019B018901AD01B301BA01BF01C40101
:10AB180068022A026802680268026802680268021B
:10AB280068026802680268026802680268026802CD
:10AB38006802680236023B02400245024A024F029E
:10AB480054025E020079FEF7C1F80028AAD105E098
:10AB58000379022BA5D07A4A82F8303195F89134DE
:10AB680043F0200385F8913400209BE7406803F008
:10AB780081FA0028F2D094E7406803F0BFFAF8E7BA
:10AB88006F4B027983F81A21E8E76D4B4268C3F8E6
:10AB9800E020E3E76A4E416896F8300103F0CCFA0A
:10ABA80000287FF47EAF6368C6F8E430D6E74168D2
:10ABB80000293FF476AF002001F0EEF90028CDD04F
:10ABC80011206FE7416800293FF46BAF0120F3E7DC
:10ABD800416800293FF465AF0820EDE74168002986
:10ABE8003FF45FAF0920E7E7416800293FF459AF18
:10ABF8000C20E1E7416800293FF453AF0D20DBE763
:10AC0800416800293FF44DAF0E20D5E7416800297F
:10AC18003FF447AF0F20CFE74A4C494B007983F800
:10AC28001901A36D9847E36A984797E7444B02795F
:10AC380083F88C2092E7424E037A8DF8043096F818
:10AC4800480096F87D308DF80530072201A901F0FB
:10AC5800C2FB00283FF425AF636896F848000193CB
:10AC6800002201A901F0B7FB00283FF41AAF6C36A7
:10AC7800D4E9010186E8030070E7314E037A8DF8C4
:10AC8800043096F8480096F87D308DF80530072294
:10AC980001A901F0A0FB00283FF403AFB436E7E7B1
:10ACA800274E037A8DF8043096F8480096F87D30E0
:10ACB8008DF80530072201A901F08DFB00283FF42B
:10ACC800F0AED4E9010106F1740383E8030096F8B5
:10ACD8001831022B7FF442AF96F83031002B3FF445
:10ACE8003DAF184BDB6A9847FDF748FF36E7144E2F
:10ACF800037A8DF8043096F8480096F87D308DF880
:10AD08000530072201A901F066FB00283FF4C9AE0F
:10AD1800BC36ADE74368029301238DF80C30084B2D
:10AD280002A993F8480001F063FB00287FF416AFEE
:10AD3800B7E6436802930023EFE700BF1C14002026
:10AD4800540E00206C18010803795A1E0E2A3FF68B
:10AD5800A8AE934A82F8683000E7914B42685A657A
:10AD6800FCE68F4B42689A65F8E68D4B4268DA65D7
:10AD7800F4E68B4B42681A66F0E6894B42685A66DD
:10AD8800ECE6874C037994F848008DF804300622E5
:10AD980001A901F020FB00283FF483AE9DF80430A0
:10ADA80084F8DD30DAE67E4C03798DF8043094F8C7
:10ADB800480094F87C308DF80630052201A901F08E
:10ADC8000AFB00283FF46DAE9DF8043084F8393052
:10ADD800C4E6734C037994F848008DF804300A22CD
:10ADE80001A901F0F8FA00283FF45BAE9DF80430A1
:10ADF80084F8DC30B2E66A4C037994F848008DF8A0
:10AE08000430092201A901F0E6FA00283FF449AE0E
:10AE18009DF8043084F83830A0E6614B4268C3F8E6
:10AE28009420DA649AE65E4B027983F8982083F8D6
:10AE3800502093E65A4B4268C3F884208EE6584B5C
:10AE48004268C3F8CC2089E6012B40F0A480554C19
:10AE58002421204603F04EFA636A984201D0172055
:10AE680020E61C2104F1280003F044FA636C9842A0
:10AE7800F5D14FF4807104F1480003F03BFAD4F89F
:10AE880048319842EBD1D42104F5A67003F032FA88
:10AE9800D4F820329842E2D1002104F5097003F079
:10AEA80029FAD4F824329842D9D14FF4607104F5C4
:10AEB8000A7003F01FFAD4F8A8359842CFD11421AC
:10AEC80004F2AC5003F016FAD4F8C0359842C6D153
:10AED800334E2146304640F2C45203F0F5F920467D
:10AEE80040F2C452002103F003FA95F81B3485F8A8
:10AEF800E833736FC5F8EC3396F87D3085F8F8338E
:10AF080040F20123A5F8FA33274B96F819019B6DF7
:10AF1800984723E68379012B3FF6C3AD204B42685F
:10AF28004068C3F82C2100F0D1FE47E61C4B42686C
:10AF3800C3F8902012E61A4B027983F81F210DE618
:10AF4800174B8288A3F8882008E6154B8288A3F857
:10AF58008A2003E6124B8288A3F8D020FEE5104B26
:10AF68008288A3F8D220F9E50D4B93F848200AB15E
:10AF7800062A12D1A288A3F8A025EFE5084B93F87A
:10AF880048200AB1062A08D16268C3F8A425E5E575
:10AF980000F099FBD9E5012084E5182082E500BF7F
:10AFA800540E0020900800206C1801082DE9F04389
:10AFB80087B00023ADF800300646002800F0ED8089
:10AFC8000361FEF73DFD20B10124204607B0BDE82E
:10AFD800F08300F073FD0028F6D100F069FD01460A
:10AFE80018B96F48142203F083F96E4D95F891341F
:10AFF800012243F0040385F8552485F89134337809
:10B008008DF804300021013B8DF80520ADF80610BD
:10B018000C2B00F2BA80DFE803F007B8B8B87881E3
:10B02800B8B88FB8AC99A800D5F8407317F02007C6
:10B03800CAD196F80480B8F1020F45D1DFF86881CB
:10B048005A4CFEF729F896F9051098F848003A4640
:10B0580001F01BFA88F83900B37988F83830384697
:10B0680007238DF80530FDF731FEFF2304F58670C0
:10B07800A5F80C31C5F8084185F8047103F04EF8BD
:10B0880004F58A7003F004F83846FDF78DFE04468F
:10B0980040B196F9051098F84800012201F0F5F939
:10B0A80088F83900D5F894343361002C71D000F059
:10B0B800FFFC002889D195F8913485F81A0460F3CB
:10B0C800820385F8913480E7B8F1010F4FF002044C
:10B0D800E8D1DFF8D4908DF8144099F8480089F841
:10B0E8001D7102A901F072F9337989F830318DF8B0
:10B0F80005708DF80680FDF785FC95F8913443F0CE
:10B10800100385F891340024CCE700226946022018
:10B1180000F0F6FA0028F6D01324C3E7244BB288CF
:10B12800DB6B96F90C10B0689847D5F8403343F0BC
:10B138000203C5F84033E6E702A90D2000F060FBE2
:10B148000028E0D0002269460D20E1E7164B93F86D
:10B158001831D3B9347904F0070000F0ADFA8DF84E
:10B168000040012269461020D2E7002269461220D9
:10B17800CEE78DF8072000F090FA044638B900F0C1
:10B1880089FA204600F08BFA8CE702248AE701242A
:10B1980088E701A800F0DEFB17E7032415E700BFE6
:10B1A800701800201C140020540E00201E140020CB
:10B1B8006C1801082DE9F04F99B08046059118B92F
:10B1C800032019B0BDE8F08F00230361FEF738FCB7
:10B1D8000646002840F0AB8045460FCD0EAC0FC4A4
:10B1E8005A4C98F800A0B8F80C7098F90EB01422D0
:10B1F80004F58860314603F07BF8012284F8412485
:10B20800534C94F83021022A35460BD194F8182172
:10B21800022A07D194F81E2122B9BAF1010F38BFCA
:10B228004FF0010ABAF1010F2DD0BAF1030F2CD05B
:10B23800BAF1000F35D102229DF83C30DDF840907C
:10B24800029362F34715012694F87C108DF83210AA
:10B2580002220CA994F848008DF8302001F0A8F8D3
:10B2680094F81A3194F830C194F81D1140B20222B2
:10B27800002B6FD0BCF1010F65D1002963D1002EDE
:10B288006DD1104627E00422D6E70023DDF83C9074
:10B29800BDF840709DF942B0029365F01F05012684
:10B2A800D2E74FF0000BD946CDF808B0CCE74FF005
:10B2B800010084F81A04DDE005F29A420BA900F0B7
:10B2C800DDFA002800F020811320049B33871F4BF0
:10B2D800002283F81A241D4BD3F89434C8F8103090
:10B2E8006FE705F29A452A460BA900F0C7FA00282D
:10B2F800EAD10B9B84F82801C4F82C5184F830312A
:10B3080002E1B9F1000F00F0FF80002A00F0FC8094
:10B318004946E01C02F0D8FF94F837320133238005
:10B32800F2E01220D1E70220CFE70720CFE7012083
:10B3380047E7064B93F8912483F840A442F00102B2
:10B3480083F89124C7E7EEB90220C4E71C14002053
:10B35800540E0020002E94D05845B8BF584694F893
:10B368007C308DF82000052294F848008DF82230B2
:10B3780008A901F030F800283FF422AF9DF82030EA
:10B3880084F83930694A6A4BD2F89804D3F8904067
:10B3980038B105F083FA664B84423CBF002283F83B
:10B3A8003A20198F1A8F93F830010491996A0991FC
:10B3B80052BA0028B9D093F81B0100B9186393F862
:10B3C8001801ADF85820013893F87C2093F81A41F9
:10B3D8001491D0F1000BD3F888108DF85B204BEB5B
:10B3E800000B93F8482093F83A0093F868308DF8EA
:10B3F8005A3009AB00934F4B03904FF001008DF882
:10B408004C0015918DF85C20A3F12F01A3F13002B7
:10B4180013A88DF84D4000F0CFF8039B4FEA0B1BA3
:10B428004BEA431B00264BEA801B4BEAC413B14589
:10B438003E4C039308BF37463A46494604F59C708C
:10B44800CDE90A669B46268084F81A6402F03CFF20
:10B45800E9B2A570C5F34215FAB2042D344E039B28
:10B4680084F837223FF423AF072D3FF44AAF022D6B
:10B478007FF459AF304D84F80D110420029984F8F7
:10B488000401FF2084F80C0184F8281184F8143191
:10B49800D6F8E410C4F8085105F59B730AA8C4F857
:10B4A800101184F83021C4F82C3100F017FC002862
:10B4B8007FF437AF0A9BA4F844040BA8A4F816310C
:10B4C800C4F84C3400F0CEF900287FF4FDAE0B9B95
:10B4D800D3B196F93900FDF7A9FA94F83732002B61
:10B4E8003FF4FFAE0B9B0F2B3FF6E6AE05F58B72D4
:10B4F8000BA90F2000F0C2F900287FF4E5AE0B9BE2
:10B5080063F3030B84F814B10598FDF74DFC00288C
:10B518007FF4DBAE099B86F83A00B36200F07EF94F
:10B5280000283FF406AF1320D1E600BF1C1400200A
:10B53800540E0020BC0E00201E14002037B50B4D01
:10B548008DF8040004460F2295F8480001A900F080
:10B5580042FF40B1064A85F81C4192F8913443F005
:10B56800200382F8913403B030BD00BF540E002090
:10B578001C14002010B5FFF7B9F8044688B90A482A
:10B5880005F0C6F9094805F0C3F9094805F0C0F9FE
:10B5980000F093F8FDF780FD064BDB6A98472046DC
:10B5A80010BD0124FBE700BF841700209C17002072
:10B5B800B41700206C1801082DE9F04F8BB04778BC
:10B5C8000093149B90F90C8090F90D6090F80E9000
:10B5D8008B464168196004469246002F57D00223D3
:10B5E8008DF8103004A9C37B007C8DF8123000F070
:10B5F800DFFEB4F808C0618943B2606898454546E3
:10B608006144B8BF1D46604534BF00270127884202
:10B6180009D30A218DF81010207C019304A900F0A9
:10B62800C7FE019B46B2B4F808C0608961680CEB9C
:10B63800400E714520D3A1EB0C01B1FBF0FC00FBDF
:10B648001C11C9B998450ADC237833B10223207C40
:10B658008DF8243006A900F0B9FE4FF00109212326
:10B668008DF81030207CE37B8DF8115004A98DF8FB
:10B67800123000F09DFE45B2009B8BF80050384612
:10B688008AF8006083F800900BB0BDE8F08F45465B
:10B69800F2E770477047704770470020704770475F
:10B6A800704770470020704700207047002070479F
:10B6B800002070470020704770477047704702208D
:10B6C800704702207047022070477047002070477B
:10B6D80070477047002070470020704770477047D8
:10B6E8007047000010B5054C4FF403722046002146
:10B6F80002F0FEFD0020C4E9000010BDDC190020A6
:10B708002DE9F8438146174600293FD0244B0025F0
:10B7180003F1010C1A462801103312F8018FB8F111
:10B72800000F36D19A42F8D11E4E33680BB9C6F8CD
:10B7380000C073680BB1C3F800C03318002401358A
:10B748009C6083F80C900D302B01BAB206EB0515FE
:10B758003044F750C6F804C002F0B6FDB9F1110F35
:10B768004FF0000398BF104C6B71D6F8083298BFA1
:10B7780024FA09F403F1010398BF04F001043B44DF
:10B788002C71C6F808324046BDE8F8834FF001082E
:10B79800F9E70135202DBBD14FF00208F3E700BFD0
:10B7A800E3190020DC1900202007020010B510B3AF
:10B7B800124A1368984204D103681360002304E016
:10B7C8000B4613B119688842FAD15168884208BFFC
:10B7D80053600BB101681960D2F808328168013BE7
:10B7E80000245B1A04602146C2F80832102202F0D5
:10B7F8007FFD204610BD0120FCE700BFDC190020BA
:10B80800054B1B6813B11A798242FAD1002B0B60E1
:10B818000CBF032000207047DC19002010B5054B31
:10B82800186800B910BD037B04680BB9FFF7BEFFA9
:10B838002046F6E7DC19002038B5084B084C186894
:10B8480000B938BD03790568112B05D824FA03F32C
:10B85800DB0701D5FFF7AAFF2846F1E7DC1900202E
:10B868002007020028B1044BD3F8083203600020F7
:10B8780070470120704700BFDC1900202DE9F04116
:10B8880007460E4615463AB331B3144B1C680023DD
:10B898002CB93046FFF7E6FF0020BDE8F081A2682A
:10B8A800F91A0132914210D32279EA54581C22899C
:10B8B8005FFA80F8611D55FA80F002F005FDA36873
:10B8C800246898445FFA88F3E2E720462468FFF783
:10B8D8006DFF002CF9D1DCE70120DEE7DC19002040
:10B8E8000238C0B211289ABF014B185C002070477B
:10B8F8007B11010830B50B4B93F82020044608460D
:10B9080072B100211C330578A54208D00131984254
:10B91800CDB20CBF04480430AA42F4D8002030BD90
:10B928001046FCE7E81B0020F41B002010B5084C6B
:10B9380000232060142204F10C00FF2184F8203039
:10B94800C4E9010002F0D4FC012384F8213010BDC1
:10B95800E81B002010B50E4A92F82010042915D8CB
:10B96800936804781C7044785C70C4788078987008
:10B978000131DC7082F8201002F11C018B4214BFE7
:10B98800043302F10C039360012010BD0020FCE792
:10B99800E81B0020094B93F8200068B15A6803F1AE
:10B9A8001C018A4200F1FF3014BF043203F10C027B
:10B9B80083F820005A600120704700BFE81B002070
:10B9C80010B5074B93F820200446084632B1596851
:10B9D800FFF790FF10B101234470837010BD00BFC2
:10B9E800E81B002008B5064B93F820202AB15968B7
:10B9F800FFF780FF08B1407808BD0120FCE700BFD1
:10BA0800E81B002030B50A4A92F82010536882F8E3
:10BA1800210061B1916801241C32DD78587005B9A4
:10BA28009C7093420CBF034B04339942F5D130BD4F
:10BA3800E81B0020F41B002008B5044B5968FFF7E9
:10BA480059FF003818BF012008BD00BFE81B0020BF
:10BA58002DE9F3410422154E044600210DEB0200A6
:10BA680096F8208002F044FC0025EBB2984502D8F5
:10BA780002B0BDE8F0817368197821705A78627055
:10BA88009F785FB1336820469B689847FFF782FF2D
:10BA980017B901A8FFF75EFF0135E6E7DB788DF8F7
:10BAA80004108DF805208DF80730EFE7E81B00201B
:10BAB800014B93F820007047E81B0020034B93F8D4
:10BAC8002000042894BF002001207047E81B0020B4
:10BAD8001FB50024CDE90244C41F8DF800408DF83D
:10BAE80001100C0AADF80420090C120C8DF8031093
:10BAF8008DF806208DF8073002461B0A012168469A
:10BB08008DF802408DF8083002F04FFA002818BF6F
:10BB18000E2004B010BD2DE9F04188B017460D463F
:10BB28000F9A064600284DD000240121CDE904448F
:10BB38008DF810109DF838108DF81510ADF81630E6
:10BB4800190CCDE900441B0ECDE902448DF81930DB
:10BB5800ADF81A20130C120E07948DF818108DF8F2
:10BB68001C308DF81D20E3B24FEA0318002D5FFA50
:10BB780088F803DC002008B0BDE8F081013310210B
:10BB88008DF81F303A466B460DEB010002F0A3F921
:10BB98000346C8B9102DAC46A8BF4FF0100CDAB256
:10BBA800624503F1010303DB103D2DB20134DAE7EE
:10BBB80008EB020020326A44315C12F8202C4A401B
:10BBC8003254ECE70920D6E70E20D4E701380328E1
:10BBD80015D8DFE800F002080C100A4B1B681B6937
:10BBE8000B6000207047074B1B685B69F8E7054B43
:10BBF8001B689B69F4E7034B1B68DB69F0E70520CA
:10BC0800704700BF0C1C00202DE9F041C4B00C4661
:10BC18004A9E17461D468046B8B3B1F5807F36D890
:10BC28004FF488720021684602F062FB49230093B2
:10BC38004FF48073ADF804302B0C8DF80830330CBA
:10BC4800ADF80650ADF80A608DF80C302246002396
:10BC5800414604A82D0E360E8DF80E308DF8095089
:10BC68008DF80D608DF80F4002F02EFB04F11001E5
:10BC78004B9A3B4689B2684602F017F910B1012881
:10BC880018BF0E2044B0BDE8F0810920FAE70D2066
:10BC9800F8E7000010B590B10A4C28220021206076
:10BCA80002F026FB2368084A1A6000204FF0FF3292
:10BCB800C3E90302C3E90522C3E9072210BD08202E
:10BCC800FCE700BF0C1C002000010101024B1B68AF
:10BCD80018600020704700BF0C1C002030B1044BD6
:10BCE8001B68DB6801330360002070470920704738
:10BCF8000C1C002013B500230C460193D2B101A9F6
:10BD0800FFF764FF18B9019B591C02D1146002B0F7
:10BD180010BD99B2611A002902DD0B441360F6E7E1
:10BD280002D113600720F2E71B0C1B0403F58033D4
:10BD38002344F3E70920EAE728B1044B1B681C33C6
:10BD48004362002070470920704700BF0C1C002088
:10BD58001FB5044600B3002303A8039302F07CF93F
:10BD6800104ABDF80C30126820469380E38200F038
:10BD780056FA98B904F11803009321680123132295
:10BD880002F08AF860B9204600F049FA003818BF76
:10BD98000120000104B010BD0920FBE71020F9E7DD
:10BDA8000E20F7E70C1C0020F0B5054687B01C46AE
:10BDB8003BB32F4E3368DB68834257D894F8202072
:10BDC800002A14BF09220822834205D3204600F026
:10BDD8005AFA70B110200AE0002301900093A3687A
:10BDE80094F82810606AFFF796FE0028EED007B096
:10BDF800F0BD23792168B4F808C0A768043B9AB25B
:10BE080009B90920F3E7B2F5807F2DD8ADF80EC047
:10BE18008DF817304FEA174C04F12C033F0E8DF8BC
:10BE2800117000932F0C08234FF0490EADF80C0049
:10BE38008DF814708DF816002F0E0DEB0300CDF859
:10BE480008E08DF810C0ADF812508DF8157002F0AA
:10BE580023F808B10E20CAE7204600F014FA00289B
:10BE6800B8D13368DD60C2E70D20C0E70620BEE721
:10BE78000C1C00202DE9FF410A9D80460F461646FE
:10BE88001C46002D5AD0002303A910460393FFF740
:10BE98009DFE18B1062004B0BDE8F081039B9C42CA
:10BEA80001D80133F6D1284600F05EF9002847D1C1
:10BEB800264B1A78424503D01A79424542D10120CF
:10BEC800AA68BA4240D103EB8002EB6A92F801807B
:10BED8002979CDE900430439927828683B4689B22C
:10BEE800FFF792FE0028D6D195F820300194002B58
:10BEF8004FF00103009314BF4246082295F828101A
:10BF0800686A3B46FFF707FE0028C4D1013E032EAE
:10BF1800C1D8DFE806F002070B0F0D4B1B681C6148
:10BF28001C62B8E70A4B1B685C61F9E7084B1B68A1
:10BF38009C61F5E7064B1B68DC61ACE70920AAE7C2
:10BF48000F20A8E70B20A6E70220A4E73401002071
:10BF58000C1C00201FB50A460B2A4FF00001CDE942
:10BF68000011CDE9021107D00C2A13D00A2A0FD0EC
:10BF78000A2005B05DF804FB012802D120238DF8C2
:10BF88000030684602F011F8002818BF0E20F0E7CC
:10BF98003023F4E70B21F4E738B5054602F000F842
:10BFA800044678B97DB9094B1B680B219878FFF7CF
:10BFB800D1FF38B90C21FFF7CDFF18B90A21FFF7D7
:10BFC800C9FF00B10E24204638BD00BF0C1C00205C
:10BFD8002DE9F04380468FB00C461746002A6BD0F7
:10BFE800002969D0002529461D2206A8059504F0D8
:10BFF800A1FE8DF81350344D2B680DF114099E885D
:10C00800CDF804900DF1130302933B7900933B683C
:10C0180032462146404601F0E4FF00284ED13868F8
:10C028003A79494602F050F9384600F04FF80028AE
:10C0380046D13C7AFA79BB79240444EA02241C43A9
:10C048002B689A6894423DD99C609DF813000B2197
:10C05800FFF780FF034658BB0C21FFF77BFF034621
:10C0680030BB0A21FFF776FF034608BB7B7ABA7A12
:10C07800FF7A3F0447EA02271F433A4633462146E0
:10C088000920FFF725FD034690B933463A46214675
:10C098000820FFF71DFD034650B92A689DF81310C4
:10C0A80091700021D1604FF0FF31C2E90411916114
:10C0B80018460FB0BDE8F0830923F9E70E23F7E728
:10C0C8000F23F5E70323F3E70C1C002010B5044603
:10C0D800002845D00168002942D011F8013B43717E
:10C0E8000322063002F0F0F82046032250F8091B1C
:10C0F800043102F0E9F82168CB79E3600A7A43EA6F
:10C108000223E3604A7A43EA0243E3608A7A43EA15
:10C118000263E360CB7A23740B7B63742379212B4E
:10C128001AD110220D3104F1120002F0CDF81D22AF
:10C138002168501C8B5C6362085C43EA0023901CF6
:10C148006362085C033243EA004363628A5C43EA41
:10C1580002636362002010BD112B03DC0D22E7E7A8
:10C168000220F8E70120F6E710B50446002854D06D
:10C178000168002951D00B7843714B7883608A7825
:10C1880043EA02238360CA7843EA024383600A7958
:10C1980043EA026383604B7903738B79C381CA795D
:10C1A80043EA0223027BC38102F00F0208311030F8
:10C1B80002F08AF8237B002203F00F0384F8202082
:10C1C80084F82820227903F10800111A04290DDDCA
:10C1D80021680933043AD21A085C84F82000D2B2E4
:10C1E800606A84F82820194402F06EF823792268DE
:10C1F8001A44002012F8043CE36212F8031C43EAD4
:10C208000123E36212F8021C43EA0143E36212F8D5
:10C21800012C43EA0263E36210BD0220FCE710B57B
:10C22800044660B3036853B30279162A29D94279C0
:10C238001A700146082251F8060B013002F04EF838
:10C248002146082251F80E0B093002F047F82368FE
:10C25800E28A5A74E38A22681B0A93742368A269E3
:10C26800DA74A36922681B0A13752368628B5A75EE
:10C278002368E27E9A7517232371002010BD0120E0
:10C28800FCE70220FAE738B50446002863D00168C5
:10C29800002960D0037B90F8282003F00F03002AC0
:10C2A80057D10833207904321344984255D363791F
:10C2B8000B702368A2685A70A36822681B0A9370DF
:10C2C80023686289DA702368E27A1A712368227B0C
:10C2D8005A712368E2899A71E38922681B0A214608
:10C2E800D371227B51F8100B02F00F02083001F0D5
:10C2F800EBFF237B94F8282003F00F0303F10805D4
:10C308002AB1226894F82010515503F109052068D4
:10C3180094F82820616A284401F0D6FF94F8283060
:10C328002268E16A2B44D1545A1CE16A206892B20F
:10C33800090A81549A1C2168E08D92B28854DA1C4B
:10C34800216894F82F0092B2043388542371002096
:10C3580038BD0933A6E70120FAE70220F8E7000014
:10C36800024B1A8810431880704700BF101C002029
:10C3780008B5074B1B883BB1FEF7B8F900280CBF7E
:10C3880000206FF0020008BD6FF00100FBE700BF5E
:10C39800101C002010B5034B00241C80FEF79CF9EC
:10C3A800204610BD101C0020B0FA80F040097047EC
:10C3B80082B018B9084602B000F0CAB8002002B02E
:10C3C800704710B9084600F077B9704710B90846A9
:10C3D80000F08EB970470346084611460BB900F0C5
:10C3E800E5B90020704710B9084600F071BD7047E4
:10C3F80010B9084600F006BA0020704710B4044689
:10C40800084611461A46019B14B910BC00F018BA28
:10C4180010BC70470346084611460BB900F042BAF3
:10C428000020704710B40446084611461A4614B94D
:10C4380010BC00F0AFBA002010BC704730B40546FD
:10C44800084611461A46DDE902341DB9029430BC8B
:10C4580000F02EBB002030BC704710B9084600F031
:10C46800DFBB0020704710B9084600F06FBD002000
:10C47800704710B9084600F0EEBB0020704710B9AD
:10C48800084600F0EBBB00207047034608461146FB
:10C498000BB900F005BC0020704710B404460846EC
:10C4A80011461A46019B14B910BC00F0FBBB0920C9
:10C4B80010BC704710B40446084611461A4614B911
:10C4C80010BC00F063BDC8B210BC7047004870478C
:10C4D80001000102064B10B51B6A0446984730B1AB
:10C4E8000448054B204498428CBF0020012010BD11
:10C4F8006C18010840C220C980B92A00F0B5114B58
:10C5080085B00C4610491F56054601F049F80F4BF7
:10C51800E4B25E6A072D4FF00103CDE902430146FC
:10C528000AD105220023CDE900234FF47A727A4319
:10C538001846B04705B0F0BD08220020CDE900201C
:10C548003A46F5E7B7110108901101086C1801087F
:10C558001FB5002300930378013B372B21D8DFE870
:10C5680003F01C242020201E202020204143454E7B
:10C578002055585B5E6164206C1E6E73787A2020AB
:10C588007D812620202020202020202020202020DF
:10C5980083858A2020838A208C90C3780BB102235C
:10C5A8000093009805B05DF804FB8378F6E74378BC
:10C5B8008DF8043005238DF805308378003B18BFCB
:10C5C80001235B008DF8063010238DF80730304BBF
:10C5D8001B6801A803F55872CDE9022300F0C0FFDB
:10C5E8000090DEE74023DBE72023D9E7827890F943
:10C5F800013012B9274AD35CD2E7274AFBE7827891
:10C6080090F90130002AF8D1244AF4E740F6B8330B
:10C61800C6E74FF47A73C3E74FF4FA63C0E741F211
:10C628008833BDE741F27073BAE71D484FF47A7159
:10C6380001F02EFE00F5FA60D2E71A4BB0E7144B72
:10C648001B6803F55873ABE7114B1B6803F55B7365
:10C65800A6E71023A4E70E4B1B68A1E74FF083431E
:10C6680000939EE7104BFBE7104B99E740F211133C
:10C67800ADF8003095E7032392E790F901300C4AB2
:10C68800B9E70C4990F9010000F08AFFA8E700BF5C
:10C69800181C00203F120108471201084F12010818
:10C6A80018FCFFFF00EA06379A99094040F7093756
:10C6B800B71101089011010837B50B4B02781B68B8
:10C6C8000C2101FB02335B7A03EB4304074B1D6823
:10C6D80003690093C3684278816805EBC40000F0E1
:10C6E800DFFC03B030BD00BF181C0020141C002064
:10C6F80070B586B0027B6423ADF80030012A4FF094
:10C708000003CDE90133CDE903338DF802308DF80C
:10C71800143030D0022A39D05ABB03684BB343686F
:10C728003BB31F4D80682B601E4B1822694618606A
:10C7380001F0CAFD1C4B2C6893E807000C3384E811
:10C74800070093E8070004F10C06032386E80700B6
:10C75800A4F86C33012204F55B7104F5587000F0FD
:10C7680090FC2B684FF6B072A3F878230522C3F823
:10C778007C2306B070BD0A4908684360036100F570
:10C788005B7100F5587000F07CFCF2E7044B1B6805
:10C79800B3F86023B3F86C130A43A3F86023E8E7FF
:10C7A800181C0020141C0020180F010808B50346A7
:10C7B8000A2924D8DFE801F006232323230B161BBC
:10C7C80023212100BDE808400068FFF783BE90F9E7
:10C7D80000009978052271B900F013FC003818BFE1
:10C7E800012008BD052293F900000021F4E790F923
:10C7F80000005978EEE70221EEE70722F3E7002070
:10C80800EFE7000010B504791CB1012C0BD0002013
:10C8180010BD0A4B01681B68012203F5587000F02F
:10C8280030FC0120F4E7054B01681B68224603F53C
:10C838005B7000F026FC2046EAE700BF181C0020C9
:10C84800F7B50528144D1C46A8BF052058700E469C
:10C858002946174600F0A4FE94F90130A070072B72
:10C8680013D1322000F09CFD0C4BDB6D0546984738
:10C8780004F10C0208340346019200943A4631460A
:10C88800284600F092FD03B0F0BD054A55F8231084
:10C89800D05C00F07DFDE7E7901101086C180108F5
:10C8A800B71101082DE9F04F344F90F901607B680A
:10C8B800D0F804908BB0044688469847054600286F
:10C8C80059D1E37C73B92E4A2378126803EB4303EA
:10C8D800990002EB8303D3F80490B9F1000F01D15A
:10C8E80052F80190274B484613F906B0FB68984761
:10C8F800A37CD7F818A022890993072E28D10023F2
:10C908000121CDE90223204A0693CDE90431CDE97E
:10C9180007330521CDE900214FF47A7202FB0BF2AF
:10C928004CF250311846D047637C13B3174B995DCE
:10C938007B6D0D31C9B228469847E07C324649469E
:10C9480000F040FE88F8006001200BB0BDE8F08FD1
:10C95800002101250823CDE90013CDE90715CDE90C
:10C968000511CDE903110292A1782B465A462846B3
:10C97800D9E7074BDBE70020E7E700BF6C180108A1
:10C98800181C0020B7110108854501004F12010845
:10C998003F1201082DE9F04F8DB090F90130DFF812
:10C9A800FCA0DFF8FC90CDE90A123E4A12F903B068
:10C9B8000278DAF800300C2505FB02333A4A5B7A34
:10C9C800126803EB430302EBC303044693F9021016
:10C9D80090F9020000F0DFFD3449064694F90100A1
:10C9E80000F0DEFDA26861688046304600F005FD73
:10C9F8002178DAF80020D9F80C30694307465058F6
:10CA08009847D9F81C309C4694F901300025072B2B
:10CA18004FF47A63CDE90753CDE905552DD10123AC
:10CA2800CDE903530523CDE901534FF47A7303FB92
:10CA38000BF300933946434646F2A8122846674648
:10CA4800B8472378DAF800200C214B4394F90110F9
:10CA5800D05800F0D9FDA18994F90100FFF74EFDE7
:10CA68000B9B217B1860D9F85430284698470A9BBD
:10CA780001201E700DB0BDE8F08F01200823CDE91C
:10CA88000350CDE901032A46CDF800B06546434678
:10CA98003946A84701200546D3E700BF181C0020E7
:10CAA8006C180108B7110108141C00209011010826
:10CAB8002DE9F04F8FB0002405468A4691469846E6
:10CAC8000494ADF81440ADF8024007264FF0010B6E
:10CAD8002B7AA34206D9686804A9204400F0F2FB27
:10CAE80000285ED102238DF8083002A86B7A8DF8F1
:10CAF8000A30FFF72DFDAB7A8DF81D309DF8113007
:10CB08008DF81E309DF812308DF81F309DF81030CA
:10CB18008DF82030EB7A8DF821302B7B8DF8223080
:10CB28006B7B8DF8233010238DF81C608DF8243032
:10CB38003A4E8DF82C000DF102030A9305238DF867
:10CB48002D3033680C930723ADF834302B680693E7
:10CB58000DF1120204AB0DF1110106A800F0CCFB97
:10CB6800072805460BD130680C22002100F55870C3
:10CB780001F0BEFB3368BDF80220A3F860239DF8DE
:10CB880011308AF800309DF8123089F800309DF88D
:10CB9800103088F80030189B28461C700FB0BDE88C
:10CBA800F08F9DF81330BDF81470ADF80270204472
:10CBB800C4B2F3B917B3194A002011680726024610
:10CBC8004FF00C0C062B1BD10CFB00FE51F80EE0AD
:10CBD800BEF1000F04D00BFA00F23A4397B20122DB
:10CBE80001301028EED1002A3FF472AFADF8027080
:10CBF8006EE75A1E042A01D9062BDCD0062667E701
:10CC080047FA00FE1EF0010FEAD00CFB00FE51F8B7
:10CC18000EE0BEF1000F08BF0626E1E7181C002051
:10CC280038B505464068FFF755FC0522841D0021EC
:10CC380095F90000E4B200F0E4F908B904F0FD0445
:10CC480095F901000722002100F0DBF908B904F08A
:10CC5800FB04204638BD00207047000010B503785B
:10CC68000F2B044618D84068FFF734FC22780B498C
:10CC780002EB42020968831C01EB820051F8222072
:10CC8800DBB21AB903F0FD0358B210BD032B06BF7F
:10CC9800626842600223F7E70020F6E7181C0020CC
:10CCA800022070472DE9F04FDFF838810446D8F8A4
:10CCB800000099B08946174600211E460122032329
:10CCC80000F55870CDE90611CDE908118DF814105A
:10CCD8008DF81510ADF8163000F0B5F938B9D8F858
:10CCE8000020B2F8603343F00303A2F86033D8F8A9
:10CCF8000020637A8DF8283002F55871CDE90B12BF
:10CD0800394A94F9083012680D920DF116020F9203
:10CD18002268109262681192D4E90301A27A8DF810
:10CD2800482001228DF8492013AA82E80300102523
:10CD3800227DE18A8DF8293018468DF85420ADF807
:10CD48003850FFF7DBFB0AAB17930DF1150316906C
:10CD580000933146019705AB06AA10A800F0BCFB6A
:10CD6800064698BB9DF81410204F013901F090FA3F
:10CD78001F4B1B690393C4B24FF00C0B04F1600303
:10CD88006B44D8F8000013F848AC9DF814300BFB3E
:10CD98000AFC01343946B4FBF3F203FB1244D0F821
:10CDA8007C33B0F9782350F80C00DDF80CC0E4B2FD
:10CDB800E04728B189F800A0304619B0BDE8F08FE7
:10CDC800013D15F0FF05D9D10D26F5E70C2801BF67
:10CDD800D8F80020B2F8603343F00303A2F86033B8
:10CDE800EAE700BF181C0020141C0020400D0300B7
:10CDF8006C180108F8B50679012E054601D80620F9
:10CE0800F8BD0F2E2BD80368187A40F303000522CB
:10CE1800002140B200F0F5F82B680446187A40F378
:10CE280003100522002140B200F0EBF8A8B1B4FAD3
:10CE380084F4640929680B7A086843F3030243F30E
:10CE4800031352B25BB29A42C8BF0124FFF742FBF8
:10CE580048B9002CD3D10420D2E70124EAE7032003
:10CE6800CEE70520CCE7002CFBD10C4F29683B68A6
:10CE780006EB460003EB80000C2201F025FA3A6825
:10CE88000C2303FB062320465C72B2F860130123CF
:10CE9800B3400B43A2F86033B2E700BF181C002070
:10CEA80010B4017801290ED9084B18680C234B439C
:10CEB800C4180022C250C4E9012200F5587010BC01
:10CEC800102200F0A7B8002010BC7047181C0020E2
:10CED8002DE9F04186B050238DF81430037A102BD9
:10CEE800074630D14368DD7B6DBB0224A846642623
:10CEF800062C14D87A68535D03932A44517843EA80
:10CF080001230393927843EA02437343CDE903383C
:10CF180063B968468DF80040FFF7C2FF0DE0CDF811
:10CF28000C808DF81480CDF81080F2E703AB01A8CF
:10CF380001938DF80840FFF75DFF0134E4B2102C2F
:10CF480005F10305D4D106B0BDE8F0811FB502682C
:10CF58000379116851B901A88DF80430FFF7A0FFD3
:10CF680078B9002040B205B05DF804FB02A802922F
:10CF78008DF80C30FFF73EFF0628F2D8024B185CFC
:10CF8800F0E70320EEE700BFB0110108C90020B99F
:10CF9800034B0B449856C0B27047024BF9E700BFE9
:10CFA800BF110108FF110108F0B59A42069D03DB85
:10CFB8009DF914309A4220DD0020F0BD03EB4303B5
:10CFC80031F814C005EB830300264CFA06F7FF0777
:10CFD80007D51F7A07F00F0E724502DBB2EB171F59
:10CFE8000DDD0136102E03F10C03EED10134E4B24D
:10CFF8002301DBB29842E1D8DEE70024F8E70120FC
:10D00800DBE7884204DB9042CCBF00200120704758
:10D018000020704710B51409B4EB111F03464FEAFE
:10D0280011100ED391420CD202B201F00F0133F865
:10D038001240012000FA01F124EA010123F812103C
:10D0480010BD0020FCE7F0B528B100EB4105012731
:10D058000020914200D3F0BD002435F802CB2346CE
:10D0680007FA04F636EA0C0608BF013304F1010496
:10D0780008BFDBB2102CF3D118440131C0B2C9B2D9
:10D08800E7E710B500B149B910BD31F8134020F8F1
:10D0980013400133DCB2A242F7D8F5E70023F9E7E1
:10D0A80082B030B5048804936AB9B3F5616F18D3B8
:10D0B80049F6AF2542F21072AB4298BF4FF47A722C
:10D0C800944238BF1446012C38BF01246143BDE89F
:10D0D8003040C3688B428CBF5B1A0023C36002B028
:10D0E80070476422ECE700002DE9F04F91B0154637
:10D0F800DDF86C8004939DF8683009930C46064669
:10D1080003F0C2FB684ADFF8A4B10590A8F5F6332E
:10D11800303BB3FBF2F3534303F5F63203F5A83380
:10D1280003F5C0730393182313FB054330320692AB
:10D13800089300254FF0FF3A089BA34207D1002D22
:10D1480014BF50464FF0FF3011B0BDE8F08FBDF965
:10D158007030ADF82C300B99CDF86C804046CDF886
:10D16800288003F021FBB4F800906EB9B8F5616F20
:10D178005BD349F6AF2242F21073904598BF4FF443
:10D188007A73994538BF99464B46012B38BF01231E
:10D198000793002E52D1B9F1640F48D1A0605F46C1
:10D1A800A1680EA803F022FB0F9B0093DDE90A1289
:10D1B8000E9B0CA803F079FA049B0C9A0BB9099BF7
:10D1C8002BB12369BB4202D1394B9A420DD9394B55
:10D1D800E760984509D90023ADF83430069B0D99CE
:10D1E8000C93184603F0E0FAA060606800B9E760A5
:10D1F800276126B103F052FBE3680344E360D4E9F6
:10D2080003329342059B1D996360079B88BFE260C8
:10D218004B43E168994202D20498A8B9A6B1012308
:10D228001D442375EDB2183486E76423A9E7B9F5E0
:10D238007A7F0ABF204F214FA060B1E7049B0BB94A
:10D24800C4F80CB05F46D0E700209342207506D89A
:10D258005B1A9A4505F1010528BF9A46EDB2002EE2
:10D26800E1D1B9F1640F164AADF8346019D049F626
:10D27800B023B9F57A7F18BF1346904584BF039A47
:10D288009B180C931C9B00930CAF97E806001B9B04
:10D29800384603F00AFA97E8030003F085FA824655
:10D2A800C1E74FF46163E8E78051010040771B0054
:10D2B8007F5101002FEC010080A81201002E93027B
:10D2C80030EC01000378032B14D1437803F00F02EC
:10D2D8001B098A704B7083788B80C27843EA0223DB
:10D2E8008B800379C3F3021203F00F03CA700B702B
:10D2F80005207047002070472DE9F3479846437989
:10D30800057990F907609146044690F906208A4607
:10D3180083B190F9087075B30F2A12D194F90920D6
:10D328000F2E1ED194F90A60072D24D1002F08BFB3
:10D33800012720E090F90B7090F9092090F90A6014
:10D34800E9E7A369019394F915300093216994F9E9
:10D358001430207BFFF728FE0028E1D105F0FD05F9
:10D36800DEE794F91D30B3420FDC94F91C30B34268
:10D37800DADA05F0FB0528468AF8002089F800600B
:10D3880088F8007002B0BDE8F0871E46CCE70000C0
:10D39800024B03FA00F0B0FBF1F0704740420F0077
:10D3A8004FF4FA53B3FBF0F0704730B54FF47A7589
:10D3B8000C1F6A4300FB042252001EBF00F1FF3419
:10D3C8001219B2FBF0F2914238BF1146039A11606C
:10D3D800820048431CBF013040084FF47A71121A8A
:10D3E80001FB1323002BCABF03F2E73393FBF1F1D0
:10D3F800B3FBF1F1049B196030BD38B54000144609
:10D408000D46F4F703FB01462846F4F74DFA21468A
:10D41800F4F74AFAF4F73CF903F0D2FCF4F718FAF7
:10D4280040B238BD2DE9F74F019300231F469C46B3
:10D438001C01058A5FFA84FE04F0F004A54206D8B0
:10D44800019B82F800C01F7003B0BDE8F08F0EEB9F
:10D458004E054FEA4309AD000024466836F80960D6
:10D468002641F60727D5866806EB050A765916B3CE
:10D47800067836B9466926B136F809602641F607B6
:10D4880019D59AF8086090F901B046F303084FFAE5
:10D4980088F8D8450FDC46F3031676B25E450ADBFA
:10D4A8009AF8096006EB4608C66806EBC806367D9A
:10D4B8004EB90137FFB20134102C05F10C05CCD15F
:10D4C8000133DBB2B4E70CF101060EEB040801F8F6
:10D4D8000C805FFA86FCEEE72DE9FF4704464068BA
:10D4E800DDE90C671D468A46914603F0D7F92368A3
:10D4F8001B1A3B604FF000080123337085F8008049
:10D50800636813B12368834224D8CAF80080D4F82A
:10D518001CC0A3699CF800E00393D4E9030101ABA4
:10D5280083E80300237D0093DCF80C10237A627AE9
:10D538007046FFF7D9FD334638602A46E069494608
:10D54800FFF770FF2B782BB1C7F80080002004B0DC
:10D55800BDE8F0873378002B14BF0B200C20F6E7CA
:10D5680037B590F9002090F90250954204460FD043
:10D57800013A52B295420BD0A368019394F9013055
:10D5880000936168E0782B46FFF70EFD0028EFD086
:10D59800104603B030BD8842B8BF08467047000047
:10D5A80051F82000054B984205D0054BC31A584244
:10D5B8005841400070470120704700BF90D00300D9
:10D5C80020A1070005281FB50ED80C4B53F82030B2
:10D5D8000093CDE901120A4B01220021022002F03A
:10D5E80069FE05B05DF804FBCDE90012054B012288
:10D5F8000021022002F05EFEF3E700BFC41201081A
:10D60800571201087612010807B5054BCDE900014C
:10D6180001220021022002F04DFE03B05DF804FB58
:10D628009212010810B5102204460021F13000F0D2
:10D638005FFE0021C4F814112046F022BDE8104016
:10D6480000F056BE02460846102100F0A5B92DE9A3
:10D65800F0430446D0F8140185B00E46154604F28E
:10D66800011988B3C0F110089045474628BF1746EE
:10D67800BAB2484400F028FED4F814313B440F2BCA
:10D68800C4F814312DD9A8452BD204F1F00304F5C0
:10D69800807113F8012F187C8B4282EA00021A70FD
:10D6A800F7D104F1F10810224146684600F00CFE5B
:10D6B80022466946684600F0E9F910226946404664
:10D6C80000F002FE3E44ED1B04F5807804F1F107FA
:10D6D800102D09D8AAB23146484600F0F5FDC4F825
:10D6E800145105B0BDE8F08304F1F003711E13F87E
:10D6F800012F11F8010F434582EA00021A70F6D192
:10D7080010223946684600F0DFFD22466946684621
:10D7180000F0BCF910226946384600F0D5FD1036F5
:10D72800103DD5E7F0B589B00C461022002105461A
:10D73800684600F0DDFD22466946684600F0A6F915
:10D748009DF90030002B6A464FF0000143DA137848
:10D7580012F8010F01315B0043EAD0130F2902F8D8
:10D76800013CF4D19DF80F305B0083F08703D4F8B7
:10D778001401DBB210288DF80F303BD104F580730B
:10D78800694604F5887013F8016F11F8012B984267
:10D7980082EA06021A70F6D104F1F00304F58071EA
:10D7A80013F8012F187C8B4282EA00021A70F7D115
:10D7B80010220DEB020004F1F10100F085FD224674
:10D7C800294604A800F062F910220021684600F0FA
:10D7D8008FFD09B0F0BD137812F8010F01315B001D
:10D7E80043EAD0130F2902F8013CF4D19DF80F3019
:10D7F8005B00BCE79DF90030002B6A464FF0000142
:10D8080037DA137812F8016F01315B0043EAD61357
:10D818000F2902F8013CF4D19DF80F305B0083F02A
:10D828008703471CDBB28DF80F30102F04EB000381
:10D83800C0F10F064FF0800288BF002600F5817006
:10D8480083F801210021324620443E4403F072FA55
:10D85800C4F8146104F58073694604F5887013F8F8
:10D86800016F11F8012B984282EA06021A70F6D16C
:10D8780092E7137812F8016F01315B0043EAD6137F
:10D888000F2902F8013CF4D19DF80F305B00C8E77E
:10D898000A780378534003704A78437853404370BA
:10D8A8008A78837853408370CA78C3785340C370AA
:10D8B8000A790379534003714A7943795340437194
:10D8C8008A79837953408371CA79C3795340C37184
:10D8D8000A7A037A534003724A7A437A534043726E
:10D8E8008A7A837A53408372CA7AC37A5340C3725E
:10D8F8000A7B037B534003734A7B437B5340437348
:10D908008A7B837B53408373CA7BC37B5340C37337
:10D91800704710B50B7814786340037054784B78CF
:10D928006340437094788B7863408370D478CB7865
:10D938006340C37014790B796340037154794B7950
:10D948006340437194798B7963408371D479CB793F
:10D958006340C371147A0B7A63400372547A4B7A2A
:10D96800634043728B7A947A63408372D47ACB7A19
:10D978006340C372147B0B7B63400373547B4B7B04
:10D9880063404373947B8B7B63408373CB7BD27BF5
:10D998005340C37310BD0000A1F11003DBB2102B7C
:10D9A8002DE9F04704D8374C24FA03F3DB0705D4F4
:10D9B800002382F8F030FF20BDE8F087531E44189A
:10D9C800A0424ED101F11C039B005FFA83F9C3F317
:10D9D8000313013B2C4D82F8F03001240B46D61876
:10D9E800B3FBF1F001FB103010F0FF0016F804ACA7
:10D9F80016F803EC16F802CC16F8017C36D115F8A7
:10DA08000E8015F80CE015F807C015F80A70E00943
:10DA180000EB400084EA080800EBC0006400C0B2D4
:10DA2800E4B24440C246581AC0B212F800808AEAEA
:10DA3800080A02F803A01044043390F801808EEA23
:10DA4800080E86F801E090F802E08CEA0E0C86F8E1
:10DA580002C0C078DBB247409945F770BFD80020B4
:10DA6800AAE710F8015B03F8015FA9E71829DAD9DA
:10DA7800102801BF15F80AA015F80EE015F80CC01B
:10DA8800EF5DD0E701010100DC1401082DE9F04F3A
:10DA9800A3B092F8F0301D911B920193002B00F077
:10DAA800538101461EA8FFF734FF1B9BA74CA84DC6
:10DAB800A84E10330293002303939DF87C00049032
:10DAC8009DF886000590205C06909DF87B000790E5
:10DAD800205C089004989DF881C0205C099014F897
:10DAE8000C000A909DF880000B909DF885009DF829
:10DAF80078809DF87DE09DF882A09DF887900C9035
:10DB08009DF87A00029B1C9314F80A2014F8093037
:10DB180014F8081014F80E700D90205C0E909DF803
:10DB28007F000F90205C10900B98205C11900C984F
:10DB3800205C12909DF8840013909DF87900149051
:10DB48009DF87E001590205C16909DF88300179034
:10DB5800205C18901398205C19901498205C1A90F7
:10DB68000398013003900298DDF804B01030029059
:10DB78009DF80C00834536D88DF878108DF87A20FA
:10DB880009990E9A8DF87C108DF882201199069AC1
:10DB98008DF880108DF87E201999169A8DF88410CA
:10DBA8008DF886200A99189A8DF87D108DF88720AF
:10DBB8001299109A8DF87B301B9B8DF881108DF887
:10DBC80083201A99089A1D988DF885108DF87F2062
:10DBD8001EA903EB0B128DF87970FFF79AFE00204F
:10DBE80023B0BDE8F08F15F808B082EA03008BEA8D
:10DBF800000016F80EB080EA0B008DF8780015F8D2
:10DC08000E004B40434016F80A0043408DF8793027
:10DC180081EA070315F80A10594016F809305940E7
:10DC280016F808308DF87A107A40534015F8092014
:10DC380053408DF87B30089A069B5340049AAA5C9F
:10DC4800534016F80C2053408DF87C30DDE908323B
:10DC58005A4015F80C305340059AB25C53408DF881
:10DC68007D30DDE909325A40059BEB5C5340079A49
:10DC7800B25C53408DF87E30069B0A9A5340049A52
:10DC8800B25C5A40079BEB5C5A408DF87F200E9B94
:10DC9800109A53400B9AAA5C53400C9AB25C5340BA
:10DCA8008DF88030DDE910325A400C9BEB5C534014
:10DCB8000D9AB25C53408DF88130DDE911325A403B
:10DCC8000D9BEB5C53400F9AB25C53408DF8823049
:10DCD800129A0E9B53400B9AB25C5A400F9BEB5C16
:10DCE8001C995A408DF88320169B189A5340139A12
:10DCF800AA5C5340149AB25C53408DF88430DDE935
:10DD080018325A40149BEB5C5340159AB25C53404E
:10DD18008DF88530DDE919325A40159BEB5C53408C
:10DD2800179AB25C53408DF886301A9A169B534066
:10DD3800139AB25C5340179AAA5C1EA853408DF8F8
:10DD48008730FFF7A5FDB8E6FF2049E7DC14010896
:10DD5800DC120108DC13010808B538B1044A05498A
:10DD68001060D82200F0B0FA002008BD0220FCE7BD
:10DD78001C1C00200C1A01080A4B1A6870B50023F5
:10DD880002F1180503EB03142E5D864204D1183402
:10DD980022440A60002070BD01330B2BF2D103200E
:10DDA800F9E700BF1C1C00202DE9F041CCB0064665
:10DDB800DDF8488117461C460D4631B3B8F1000F0F
:10DDC80023D006A8FFF72EFC204601A9FFF7D4FFB1
:10DDD8000446B0B9019906A80131FFF733FC26B112
:10DDE8001022314606A8FFF732FC3A46294606A813
:10DDF800FFF72DFC06A902A8FFF794FC029BC8F8C0
:10DE0800003020464CB0BDE8F0810224F9E700005C
:10DE180030B595B013A90446FFF7AEFF002830D1FE
:10DE28001B490C2303FB00F2555CA5422BD1139B25
:10DE3800187C1090D87B0F90987B0E90587B0D9093
:10DE4800187B0C90D87A0B90987A0A90587A099097
:10DE5800187A0890D879079098790690587905909B
:10DE680018790490D8780390987802900A445B78DF
:10DE78000193936800930022064B1146022002F09A
:10DE880019FA15B030BD01300B28CBD1F9E700BF26
:10DE980054170108DC1501080B2B10B402D810BC6C
:10DEA800FFF782BF032010BC704730B50D4685B020
:10DEB8001446014668B103AA002000922A4603903E
:10DEC800FFF772FF18B90398001B18BF012005B0AF
:10DED80030BD0220FBE72DE9F0430D46BFB01446E4
:10DEE8009946804620B31BB311F00F0122D1F022CE
:10DEF80001A800F0FDF920466946FFF73DFF0446FA
:10DF080048B9009801AA10210130FFF745FD2E46B7
:10DF1800AF1BFFB21EB920463FB0BDE8F08301AA8F
:10DF280009EB070108EB0700FFF7B0FD103EEFE72C
:10DF38000224F0E70524EEE7F0B5184E34680246EF
:10DF480085B00846002304F1180103EB03154F5D63
:10DF580097421ED10D2A05F1190513D10023CDE9E9
:10DF68000033CDE902330C2210216B46FFF7B3FFD3
:10DF78000446306810226946284400F0A5F9204676
:10DF880005B0F0BD01461022601900F09DF900248B
:10DF9800F5E701330B2BD8D10324F0E71C1C002034
:10DFA80009B1FFF7C9BF022070471FB51446A0B1D9
:10DFB8000C2A01D10B2912D10023CDE90033CDE978
:10DFC80002330A466B461021FFF785FF18B96946E8
:10DFD8002046FFF7B1FF04B010BD0220FBE7032085
:10DFE800F9E7F8B51E46DDE907479DF818505BB319
:10DFF80054B34FB3212D29D819462A46204600F09C
:10E0080063F90122631C691EB018FFF764FFF8B9B1
:10E01800E37ADB093B70EBB96319204613F8012C4E
:10E0280013F8021C120642EA014213F8041C0A43C0
:10E0380013F8031C012342EA0122291FFFF735FFC9
:10E04800003818BF0120F8BD0220FCE70520FAE7D8
:10E058000720F8E70420F6E710B5044628B1044B7A
:10E068005B6998472060002010BD0220FCE700BFD4
:10E078006C18010808B5014630B1044B082218682D
:10E0880000F022F9002008BD0220FCE71C1C00203B
:10E0980008B530B1044B0822196800F015F90020C2
:10E0A80008BD0220FCE700BF1C1C00207FB5124EF3
:10E0B8000023044602A801930D46FFF7E9FF3368E1
:10E0C8005B6901936CB102AA082312F8011B41B9DC
:10E0D800013B13F0FF03F8D102A8A04702A8FFF7FD
:10E0E800C9FF35B1019B23B901A8A8473368019A34
:10E0F8005A61002004B070BD1C1C002008B5014600
:10E1080038B1054B18680822104400F0DDF80020EB
:10E1180008BD0220FCE700BF1C1C002008B538B170
:10E12800044B19680822114400F0CEF8002008BDFD
:10E138000220FCE71C1C0020034B1B6802280CBFB4
:10E1480019615961002070471C1C002041B1054B22
:10E158001B6802280CBF1B695B690B6000207047B5
:10E16800022070471C1C002030B58FB000240546E3
:10E178000CA80994FFF78CFF9DF8373007939DF89A
:10E18800363006939DF8353005939DF83430049366
:10E198009DF8333003939DF8323002939DF8313067
:10E1A80001939DF830300093224621461E4B0220F1
:10E1B80002F080F80AA8FFF7B1FF9DF82F30079307
:10E1C8009DF82E3006939DF82D3005939DF82C3040
:10E1D80004939DF82B3003939DF82A3002939DF801
:10E1E800293001939DF82830009322460F4B214691
:10E1F800022002F05FF809A92846FFF7A7FF9DF85B
:10E20800243003939DF8253002939DF8263001931E
:10E218009DF8273000932246054B2146022002F044
:10E2280049F80FB030BD00BF38160108761601084E
:10E23800B416010808B50020FFF7EAFD0120FFF732
:10E24800E7FD0920FFF7E4FD0820FFF7E1FD0020C6
:10E25800FFF78AFF002008BD10B504460B20FFF722
:10E26800D7FD0C20FFF7D4FD0920FFF7D1FD0820CA
:10E27800FFF7CEFD0A20FFF7CBFD2046FFF774FF1E
:10E28800002010BD014B1860704700BF3C01002002
:10E298000B4A30B514680B4D43F2390305FB0433C0
:10E2A8001360091A6FF00042B3FBF2F2C2EBC272BC
:10E2B80001319B1A93FBF1F201FB1233184430BD74
:10E2C8003C0100206D4EC64101380A44914200D1FC
:10E2D800704711F8013B00F8013FF7E710440A4482
:10E2E800914200D1704711F8013B00F8013DF7E772
:10E2F80002F020BD30B530B10A4D01444FF0FF3374
:10E30800814201D1D84330BD10F8012B5340082277
:10E3180043F30004013A2C4092B284EA5303002AE2
:10E32800F6D1EDE72083B8ED01207047054B4FF497
:10E3380000529A62044B1B6813B15B6803B118471B
:10E34800704700BF00040048201D0020054B4FF413
:10E3580080529A62044B1B6813B1DB6803B11847FB
:10E36800704700BF00040048201D002001207047AE
:10E378000120704701F048B901F036B910B501F035
:10E3880019FE0E21044640F61F1001F02DF9204613
:10E39800012101F0F9FDBDE8104001F0D7BA0000F5
:10E3A80070B50C4E01EB40030D46B3654FF6FF7197
:10E3B800002304461A46084601F05EFB96F856000C
:10E3C800002101F0E1FD29462046BDE8704001F03A
:10E3D80095BA00BF3C1D002010B5044601F0AAFE06
:10E3E80001281CD101F0AEFE34B11248214602F0DA
:10E3F80017FB104802F0DAFA0F4C104B00214FF4CB
:10E408008052A1659A6194F8560001F0BDFD6378C9
:10E418006BB16FF07F40BDE8104001F053BA0023A4
:10E4280040F262211A46084601F026FBDCE7A068A4
:10E438008001F0E7241D00203C1D00200004004856
:10E44800002001F0BFB9000008B501F0C7F8043892
:10E45800C0B2032896BF024B0020185C08BD00BF5D
:10E468006818010808B501F0BAFD033008BD01F0CD
:10E4780049B901F009B908B501F000FD00B208BDBD
:10E4880038B50D46144601F05DFB284601F092FDB3
:10E498000E21054640F61F1001F0A6F82846012176
:10E4A800074D01F071FD01F051FA4FF47A716143A3
:10E4B800284602F0B5FA2846BDE8384002F076BA98
:10E4C800981D002001F03EBB08B5084B002193F8C9
:10E4D800560001F059FD00234FF4C0711A46084652
:10E4E80001F0CAFABDE8084001F024BA3C1D00203A
:10E4F80010B5044601F01EFE01281CD101F022FED1
:10E5080034B11248214602F08BFA104802F04EFA54
:10E518000F4C104B00214FF48052A1659A6194F87A
:10E52800560001F031FD63786BB16FF07F40BDE8B4
:10E53800104001F07DB9002340F262211A460846D6
:10E5480001F09AFADCE7A0688001F0E7241D0020BA
:10E558003C1D00200004004808B54FF0040001F0FD
:10E5680017F9BDE808400220F4F7A6BA08B5002359
:10E578001A461946184601F07FFABDE8084001F02E
:10E588006DB900001D4B73B51D4D186000241D4862
:10E598006C70C5E90144AC6501F098FAAC8101F0F2
:10E5A80003FA2146204601F04BFC214604220120B3
:10E5B80001F0FCFA144E154D4FF6FF712346224622
:10E5C800084601F059FAFFF7C7FF2246104B00949E
:10E5D8004FF0FF31304602F03DF90E4B00942246D1
:10E5E8004FF0FF31284602F035F9304602F090F935
:10E5F800284602B0BDE8704002F08AB9201D00200C
:10E608003C1D0020D5F50008981D0020241D002081
:10E6180035E3000855E300080128084805D1084BF0
:10E62800C17719700E3001F0A7BB437D012B03D1D0
:10E63800034B81751970F5E7704700BF3C1D00203A
:10E64800400100200D4B10B5044618735873012083
:10E6580000F016F85CB134214FF4E86000F0C4FF14
:10E668004421BDE8104040F2417000F0BDBF1421C4
:10E678004FF4E86000F0B8FF2421F2E73C1D0020C9
:10E6880038B5114C0546207001F061FD052D04D800
:10E69800DFE805F0090B03171709032001F070FAEA
:10E6A8000023637338BD0020F8E7012001F068FA01
:10E6B800207B637B8342F5D06073BDE83840FFF769
:10E6C800C1BF0220EAE700BF3C1D00202DE9F0434E
:10E6D8001E4687B000230546CDE901330C46174690
:10E6E80001F027FD032D61D8DFE815F07B00C3009A
:10E6F8000E010400A27C082A04D94FF0FF3007B0AD
:10E70800BDE8F083A16801A801F0DCFE21680029BA
:10E71800F3D042F210729142E37C864D51D8032225
:10E72800AA7385F83820E96385F844304FF0020869
:10E738006368A17DDB002B820423AB74A37CDB0020
:10E74800EB7402294FF000032B75637D02D0227D04
:10E75800022A42D103F10F02D2B2012A01D9012BB8
:10E76800CBD1754B754A196803944FF0010903A87A
:10E778008DF8149001F0DAFC0028BED1287685F8CF
:10E7880017906875FFF75CFE4046FFF779FF6C4805
:10E7980001F086FA6B4801F0EFFA01A800F084FF57
:10E7A800208A00F055FFA08900F09AFF384601F052
:10E7B80001FC604C84F8560001F0C0FC6660002043
:10E7C8009DE74FF00008E963890885F80E8085F811
:10E7D800388085F844302964AAE7EB7529766A758C
:10E7E800D0E72368002B88D0A27C082A85D8514D11
:10E7F800A16801A801F066FE002385F83830226878
:10E80800EA63E27C85F84420A269AB732A646268F3
:10E81800A17DD2002A820422AA74A27C2B75D20080
:10E828000229637DEA7402D0227D022A1DD103F1F8
:10E838000F02D2B2012A02D9012B7FF45EAF3E4B00
:10E848003E4A196803944FF0010803A88DF8148014
:10E8580001F06CFC00287FF450AF287685F817800B
:10E868006875FFF7EDFD00208FE7EB7529766A756F
:10E87800F7E7304D012185F83810227885F85020C7
:10E88800637885F85130A37885F85230E3788B4265
:10E8980002D0022B03D03BB985F8533004E00B3A81
:10E8A800012A29D885F853104FF0010885F80E8001
:10E8B800A388AB83A379AB77E37985F82030237AF3
:10E8C80085F82130FFF7BCFD4046FFF7D9FE1C480C
:10E8D80001F0E6F91B4801F04FFA95F85130062B84
:10E8E80040F689000AD100F08FFE00F0FB0140F6E7
:10E8F800890000F079FE59E70023CDE700F084FE97
:10E9080040F00401C9B2F2E72368013BB3F57A7F0E
:10E91800BFF4F3AE0320FFF7B3FE0648022380F8E6
:10E92800383023688364162380F84C30383001F07F
:10E93800B7F93BE73C1D0020201D0020981D002052
:10E94800741D00204A1D00202DE9F041002686B0E4
:10E958001F461446CDE9016680460D4601F0E9FBE5
:10E96800B442764C16BF0123334637466370B8F17C
:10E97800000F06D0B8F1010F7CD0002006B0BDE82A
:10E98800F081AB68002B00F0D680EB68002B00F01C
:10E99800D280AA7F082A00F2CE80296901A801F056
:10E9A80091FD2868003818BF012000F0D9FF84F8CD
:10E9B8003880AB68E36395F8203084F844306868A1
:10E9C80001F05AFB84F80E8084F84500EB68DB0000
:10E9D8002382EB7FA374AB7FDB00E37495F82130CF
:10E9E800237595F82230002B3ED12A7D95F8241006
:10E9F800A275022995F8232001D0022B36D102F105
:10EA08000F03DBB2012B02D9012A40F094800023C6
:10EA18008DF814304A4B4B4A1968049503A801F045
:10EA280085FB002840F0878001232076E375607518
:10EA3800FFF706FD0020FFF723FE434801F030F9F9
:10EA4800424801F099F901A800F02EFEA88B00F0C9
:10EA5800FFFD288B00F044FE4FF4FA53AA687B436D
:10EA6800B3FBF2F3A36088E7FF22BFE7E2752176E4
:10EA78006375DDE72B8E002B5DD095F83230A86AE0
:10EA8800012B0CBF95F814804FF0FF08003818BF11
:10EA9800012000F065FFF8B200F06EFF012184F854
:10EAA800381095F82C2084F8502095F82D3084F8EB
:10EAB800513095F82E3084F8523095F82F308B422B
:10EAC80002D0022B03D03BB984F8533004E00B3A50
:10EAD800012A28D884F853102B8EA38395F8323056
:10EAE800A377AB8E23840126A67384F81F80FFF7D3
:10EAF800A7FC3046FFF7C4FD134801F0D1F81348CE
:10EB080001F03AF994F82130B34240F236700CD152
:10EB180000F07AFD00F0FB0140F2367000F064FD71
:10EB28004FF6FF739EE70023CEE700F06DFD40F03F
:10EB38000401C9B2F0E74FF0FF301FE73C1D002089
:10EB4800201D0020241D0020741D00204A1D0020C7
:10EB58002DE9F04F85B082460E9DBDF840B09DF876
:10EB680044709DF84890019288461E4601F0E1FAEB
:10EB7800BAF1010F524C54D0BAF1040F00F0918051
:10EB8800BAF1000F3AD10B22304684F8442084F8B9
:10EB980038A0E56301F070FA019B23644FEACB03C8
:10EBA800B9F1000F238241F60403638214BFF223F4
:10EBB8000123E37587F001070123237684F84500D4
:10EBC80084F80EA084F814A06775FFF739FC504646
:10EBD800FFF756FD04F1380001F062F804F10E0069
:10EBE80001F0CAF8374A1068516802AB03C302A89B
:10EBF80000F05AFD40F2FF1000F02AFD404601F0F7
:10EC0800D9F90E2184F8560040F61F1000F0ECFCEC
:10EC180094F8560001F092FA169B636005B0BDE8BF
:10EC2800F08F294984F838A0EAB2895D84F8502029
:10EC380076BB0B3D012D8CBF00250125053A012A25
:10EC480004D8BBF10C0F38BF4FF00C0B1F4B9DF8CD
:10EC58003C201B7884F85350E37701259DF8543005
:10EC680084F8511084F8522084F82130A573A4F850
:10EC78001CB0A77784F82090FFF7E2FB2846FFF73F
:10EC8800FFFC134801F00CF8124801F075F8B5E7DD
:10EC9800012E04D1A5F10C035D425D41CEE70025AC
:10ECA800CCE75046FFF7ECFC022384F8383004F137
:10ECB80038001623A56484F84C3000F0F1FF9DE776
:10ECC8003C1D0020300F01083618010840010020C3
:10ECD800741D00204A1D00202DE9F04F87B0DFF891
:10ECE800B4B29DF864A09DF84C90029314469DF828
:10ECF80054309DF85020BDF84880039205468BF8A3
:10ED080001A0BDF8446001930F4601F012FABAF170
:10ED1800000F18BF4FF00008DFF87CA2039AB9F182
:10ED2800000F08BFFF22012D8AF8002000F0C880DC
:10ED3800052D48D0002D40F0C080284600F010FE78
:10ED48000B2238468BF844208BF83850CBF83C40DF
:10ED580001F092F9019B8BF8450041F60402002B63
:10ED6800ABF812209AF800208BF8162014BFF22274
:10ED780001228BF81720F600012289F001098BF88F
:10ED880018208BF80E50ABF810608BF814508BF8E5
:10ED98001590FFF755FB2846FFF772FC0BF138007A
:10EDA80000F07EFF0BF10E0000F0E6FF7B490868DB
:10EDB800496804AA03C204A800F076FC40F2FF10D8
:10EDC80000F046FC71E0012000F0CAFD09224FF076
:10EDD80000098BF8442038464FF44872CBF840209D
:10EDE8008BF83890CBF83C4001F046F94FF480524C
:10EDF800ABF812209AF800208BF845008BF8162003
:10EE080028460122F6008BF817208BF80E90ABF8F5
:10EE18001060ABF814908BF81890FFF731FC0BF1E9
:10EE2800380000F03DFF0BF10E0000F0A5FF5B4934
:10EE38008868C96804AA03C204A800F035FC40F237
:10EE4800FF1000F005FC40F6B80000F0DDFB00F014
:10EE5800EF0140F6B80000F0C7FB042140F6B90006
:10EE680000F0C2FB40F69B0000F0CEFB00F0E3018F
:10EE780041F0080140F69B0000F0B6FB40F2D1607B
:10EE880000F0C2FB40F01801C9B240F2D16000F0B6
:10EE9800ABFB40F2AC6000F0B7FB00F08F0141F033
:10EEA800500140F2AC6000F09FFB4FF4FA5202FBB5
:10EEB80008F2B2FBF4F2CBF8082007B0BDE8F08FF7
:10EEC800002000F04DFD36498BF83850E2B2C95D9C
:10EED8008BF85020002F4DD10B3C012C8CBF002407
:10EEE8000124053A012A02D80C2E38BF0C26029BB1
:10EEF8009AF800208BF852308BF85340019B8BF81E
:10EF08001F2001249DF860208BF821208BF85110D8
:10EF18008BF820308BF80E40ABF81C608BF81E90F5
:10EF2800FFF78EFA2046FFF7ABFB1E4800F0B8FE4D
:10EF38001D4800F021FF5FFA88F000F01DFD40F643
:10EF4800A30000F061FB00EA040140F6A30000F012
:10EF58004BFB9BF82120A24240F2367013D100F0FF
:10EF680053FB00F0FB0140F2367000F03DFB4FF61A
:10EF7800FF72A0E7012F04D1A4F10C035C425C41AD
:10EF8800AFE70024ADE700F03FFB40F00401C9B251
:10EF9800E9E700BF3C1D002040010020300F0108B8
:10EFA80036180108741D00204A1D0020F0B58BB0EA
:10EFB8000D46044617461E46FFF742FA0020FFF7A3
:10EFC8005FFB204600F0BEFD00240123CDE9084385
:10EFD80003234FF4167229462046CDE90644CDE9AD
:10EFE8000444CDE90244CDE900532346FFF774FEFB
:10EFF8002046FFF77DFAFFF735FAF3F75DFD01F0DC
:10F0080043FC0446204601F049FCB04205D30124E4
:10F01800FFF716FA20460BB0F0BD00F02FFF00B244
:10F028008742EFDA0024F3E7F7B500230C4640F2F5
:10F0380001211A460646084600F01EFD644B654D40
:10F048004FF400529A6195F85600012100F09CFF98
:10F058002B78012B40F6890013D195F85130062BF7
:10F068000FD100F0D1FA00F0FB0140F6890000F062
:10F07800BBFA2B78042B6CD8DFE803F0524B527F95
:10F08800090000F0C1FA40F00401C9B2EDE7524AA4
:10F09800731E1046C6F101074FF0000CF9188C4298
:10F0A8006FDC0022E7001346BA4271D19A0142EAA6
:10F0B800C3125B0183F020031343661C0355F6B2A9
:10F0C80002234648AB73AE7600F056FE0021F120CD
:10F0D80000F08AFA0021F02000F086FAAB6C642B6D
:10F0E80070D17021F32000F07FFA1D21F22000F08A
:10F0F8007BFAE1008C1CF420090A00F075FA04F090
:10F10800FE01F52000F070FA33486FF07F42314677
:10F118001DE0EC77314800F02FFE0022214615E073
:10F1280001F008F80128074625D121460DF107020C
:10F13800304601F004F80446A0B99DF80730274886
:10F14800AB7500F019FE9DF807102246304600F016
:10F1580065FB6968224801F063FC214801F026FC40
:10F16800002006E01F4B3A460021022001F0A2F8D9
:10F17800032003B0F0BDAC75CCE70223AB73AC76CB
:10F18800C8E713F8011FC943197002F801CB85E7D6
:10F19800D1106FEA020C715C0CF0070C013241FAD5
:10F1A8000CF101F001014FEAE20C4B40D14310F899
:10F1B8000CE001F0070103FA01F141EA0E0100F841
:10F1C8000C1071E7E121F32000F00EFA04218DE71D
:10F1D800000400483C1D0020201C00204A1D00207F
:10F1E800981D0020D8170108F0B5BDF814409DF807
:10F1F80018709DF81CE09DF8205040B1012814D0EB
:10F208000122002398180138B0FBF2F0F0BD87F016
:10F218000107E30003EBC70318330EEB450503EBC7
:10F22800C5034FF47A714B43ECE7501F012803F1F3
:10F23800040302D80C2C38BF0C24D1B9A2F10B0C52
:10F24800BCF1010F8CBF4FF0000C4FF0010C2801EE
:10F25800002F00EBCE0014BF00251425A0EB820080
:10F26800062A4FEA82062844A2F102070DD835463D
:10F2780010E0012906D1A2F10C00D0F1000C4CEBF2
:10F28800000CE4E74FF0000CE1E70830BCF1000F98
:10F29800EDD0BD000028ACBF2E182E1C701E90FBB0
:10F2A800F5F003FB0044094B062A5A5C8CBF0C346A
:10F2B8000E340A2A09D8A30001334FF47A71BB40EF
:10F2C8004B43034951F822209CE7FFDE361801081A
:10F2D8003C18010808B5094B012193F8560000F0C5
:10F2E80053FE4FF4D7602D2100F07EF900F033FB78
:10F2F800BDE80840024800F07BBA00BF3C1D002072
:10F30800FFFF0F0073B5A44CB4F854300025202B30
:10F318008DF80350019500F01B8114D8082B0DD8E7
:10F328007BB1013B072B0CD8DFE813F042005B00F0
:10F338000B00CD000B000B000B00FD00102B00F0A4
:10F34800008102B070BDB3F5807F00F0988011D8BD
:10F35800402B00F01081802BF3D1284600F032FAC0
:10F368008E4B1B68002BECD09B69002BE9D02846FC
:10F378009847E6E7B3F5007FE3D1894B0122294698
:10F38800022000F097FF00F029F9042840F085805A
:10F39800844B85484FF400529A6201F0B9FA284626
:10F3A80000F010FA7D4B1B68002BCAD05B6814E094
:10F3B8007C4B7D484FF400529A6201F0A9FA002074
:10F3C80000F000FA00F0B8FE012801D100F0BDFEFF
:10F3D800724B1B68002BB4D01B68002BB1D0984728
:10F3E800AFE7704B71484FF480529A6201F090FA7F
:10F3F800657895B9284600F0E5F9294640F60210E7
:10F4080000F0F2F840F6441000F0FEF840F0020177
:10F41800C9B240F6441000F0E7F8FF220DF10301ED
:10F4280063485E4D00F05AFD624800F071FD2B689C
:10F43800002B86D09E68002E83D094F82430012BB0
:10F4480008D194F9313094F930209DF803105848C8
:10F45800B04776E7E06B01A900F022FE019B9DF81A
:10F46800031053484FF47A7203F5FA7393FBF2F3DF
:10F478002A685BB2956894F92920A84761E728466D
:10F4880000F0A0F9454B1B68002B3FF45AAF9B696D
:10F49800002B3FF456AF01206AE700F09FF80528DB
:10F4A8007FF44FAF3F4B41484FF480529A6201F0CE
:10F4B8002FFA284600F086F9384B1B68002B3FF4DA
:10F4C80040AFDB6889E700213B4B0122022000F0B6
:10F4D800F1FEA16D00293FF434AFC1F3074140F6B6
:10F4E800031000F081F894F8591040F6041000F069
:10F4F8007BF894F8581040F6051000F075F840F6BF
:10F50800021000F081F840F00101C9B240F6021083
:10F5180000F06AF8002340F262211A460846A36503
:10F5280000F0AAFA0DE7254B01220021022000F085
:10F53800C1FE00F0FFFD01287FF403AF00F006FED6
:10F54800FFE61F4B01220021022000F0B3FEF8E67F
:10F55800164801F0DDF9607808B900F033F90F4B6F
:10F568001B68002B3FF4EDAEDB68002B3FF4E9AEDF
:10F578009847144BE6E7144B01222946022000F075
:10F5880099FE607808B900F01DF9044B1B68002B40
:10F598003FF4D7AE1B6920E73C1D0020201D00204A
:10F5A800ED17010800040048981D0020241D0020C4
:10F5B800201C0020601D0020011801080A180108FD
:10F5C800141801081D18010826180108024BA3F891
:10F5D8005400FFF797BE00BF3C1D0020014B187870
:10F5E800704700BFB61D002007B501238DF807102E
:10F5F8000DF1070201460348F7F774F803B05DF808
:10F6080004FB00BF4C03002007B5012301460DF1A0
:10F6180007020448F7F79FF89DF8070003B05DF864
:10F6280004FB00BF4C03002010B50446F4F716FD98
:10F6380001280CD140F62310FFF7E6FF00F0F9018E
:10F64800214340F62310BDE81040FFF7CDBF10BDA1
:10F6580010B50C4B1B7804469BB94FF4D760FFF7E5
:10F66800D3FFC4F3002100F0FE0001434FF4D7603C
:10F67800FFF7BAFFE1B240F2B960BDE81040FFF70A
:10F68800B3BF10BDB71D002010B51346EFF31084AB
:10F6980072B60A4601460348F7F724F884F310883F
:10F6A80010BD00BF4C03002008B5014608224FF4E6
:10F6B800D860FFF7E9FF002008BD000007B5074B39
:10F6C8001B7840BAADF804002BB9022201A940F218
:10F6D800BC60FFF7D9FF03B05DF804FBB71D00203D
:10F6E80007B5074B1B7840BAADF804002BB90222C6
:10F6F80001A940F2BE60FFF7C7FF03B05DF804FB45
:10F70800B71D002010B51346EFF3108472B60A46F1
:10F7180001460348F7F71FF884F3108810BD00BFAF
:10F728004C03002010B51346EFF3108472B60A4656
:10F7380001460348F7F701F984F3108810BD00BFAC
:10F748004C0300200A4601460020FFF7EBBF0000EB
:10F7580010B51346EFF3108472B60A460146034803
:10F76800F7F71EF984F3108810BD00BF4C03002082
:10F7780010B51346EFF3108472B60A4601460348E3
:10F78800F7F724F884F3108810BD00BF4C0300205D
:10F7980013B504460020F4F73BFC0220FFF744FFB2
:10F7A80004F0070401220DF1070184208DF80740B9
:10F7B800FFF7DEFF024B00221A7002B010BD00BF37
:10F7C800B61D002007B501228DF807000DF10701CD
:10F7D8008020FFF7CDFF9DF80730002B034B0CBFAF
:10F7E800012202221A7003B05DF804FBB61D002046
:10F7F80007B5094B8DF8060004221A70030C8DF822
:10F8080004300322030A01A983208DF80530FFF78D
:10F81800AFFF03B05DF804FBB61D002010B5144619
:10F82800FFF790FF2046BDE81040FFF7E1BF00005A
:10F8380007B5094B8DF8060005221A70030C8DF8E0
:10F8480004300322030A01A982208DF80530FFF74E
:10F858008FFF03B05DF804FBB61D002073B50026CA
:10F8680040F6E2000196FFF7CFFE00F0FE010546E4
:10F8780040F6E200FFF7B8FE40F6E500FFF7C4FEE9
:10F8880000F07F01044640F6E500FFF7ADFE6FF09B
:10F898007F40FFF7CDFF04220DEB020140F619006F
:10F8A800FFF730FF3046FFF78DFF294640F6E200AC
:10F8B800FFF79AFE214640F6E500FFF795FE01980E
:10F8C80002B070BD13B50C4B04460522972140F6D3
:10F8D800AC001A70FFF788FE230C8DF80430032261
:10F8E800230A01A982208DF805308DF80640FFF71C
:10F8F8003FFF02B010BD00BFB61D002007B5030CC6
:10F908008DF80030030A8DF801300B0C49BA8DF8D8
:10F918000200ADF804100622694694208DF80330E1
:10F92800FFF726FF024B06221A7003B05DF804FBAE
:10F93800B61D0020002208B51146C520FFF718FFA4
:10F94800014B07221A7008BDB61D0020002211467F
:10F95800D120FFF70DBF00221146D220FFF708BFC4
:10F9680007B501228DF807000DF107019F20FFF769
:10F97800FFFE03B05DF804FB07B501228DF8070010
:10F988000DF10701A020FFF7F3FE9DF807103F29AE
:10F9980007D901F0F8010131C9B240F20670FFF74A
:10F9A80023FE03B05DF804FB07B5F4F757FB431ECD
:10F9B800584258418DF8070001220DF107019620A1
:10F9C800FFF7D6FE03B05DF804FB07B500F07F0033
:10F9D8008DF8070001220DF107018920FFF7C8FE05
:10F9E80003B05DF804FB0000154B984207B51BD81F
:10F9F800144B98421BD8144B98421BD8134B98426F
:10FA08001BD8134B984295BF29226B222B236F23B7
:10FA18008DF8042001A9022298208DF80530FFF7FF
:10FA2800A7FE03B05DF804FBE122E923F0E7D72243
:10FA3800DB23EDE7C122C523EAE775228123E7E747
:10FA480000E9A43580F8A9328044E52D000B6B1B32
:10FA580040FC541907B58DF8062004228DF80400DF
:10FA68008DF8051095200DEB02018DF80730FFF792
:10FA78007FFE03B05DF804FB07B552BAADF8042069
:10FA880040BA082249BAADF80000ADF802105BBAD6
:10FA980069461046ADF80630FFF76AFE03B05DF818
:10FAA80004FB07B50B0C042200F0070049BA8DF8D7
:10FAB8000400ADF8061097200DEB02018DF8053013
:10FAC800FFF756FE03B05DF804FB000010B508B15F
:10FAD800194B1860F2F7F0FE0220FFF7A5FD00248D
:10FAE800164B20461C70FFF76DFEF4F7B5FA012897
:10FAF80017D14FF42071FFF7D4FF40F611102146BB
:10FB0800FFF772FD4FF07F00FFF75FFF0E2140F611
:10FB18001F10FFF769FDF4F747FA094B01221A7025
:10FB280010BD102140F61110FFF75EFD102140F6C0
:10FB38001210FFF759FDE9E7B81D0020B41D002099
:10FB4800B61D002037B50C4D2B7804461BB9FFF7BE
:10FB58004BFF01232B700023084A6006E109F1F7E7
:10FB6800D3FF042200BA01900DEB02018620FFF7B3
:10FB7800FFFD03B030BD00BFB41D00200048E80100
:10FB880007B5094B8DF807000146187018B940F2FF
:10FB9800AC60FFF729FD01220DF107018A20FFF76C
:10FBA800E7FD03B05DF804FBB71D0020012873B51D
:10FBB8000C46164637D10020F4F752FAA042B8BFD7
:10FBC80044B20E2805461AD101231A460021042002
:10FBD800FFF740FF6FF010039C42B8BF1C46182186
:10FBE80040F6E700FFF700FD022201A98E208DF8FC
:10FBF80004408DF80560FFF7BBFD02B070BD01231E
:10FC08000A28E4B21A464FF0000105D11846FFF75A
:10FC180021FF033464B2DDE70720C5F10E05FFF7C5
:10FC280019FF2C44F6E740F6D800FFF7EDFC40F04A
:10FC38001E01C9B240F6D800FFF7D6FC0120F4F740
:10FC48000FFAA042B8BF44B2142805464FF001038A
:10FC58004FF000020CD105210320FFF7FBFE023410
:10FC680064B26FF008039C42B8BF1C463821B7E75E
:10FC7800112805D103210220FFF7ECFE0534EFE738
:10FC88000E2804D102210846FFF7E4FEE9E7C5F192
:10FC98001605072104202544FFF7DCFE6CB2E0E7D7
:10FCA80013B5314A0446516810686B4603C32F4B9D
:10FCB80020781B78834201D0FFF762FF2378032B5B
:10FCC80027D8DFE803F00239283C6268284BB3FBE9
:10FCD800F2F31A0CA1688DF800208DF802301A0A88
:10FCE800237B8DF80330637B8DF801208DF8043079
:10FCF800204A00234806C909F1F706FF030C40BA59
:10FD08008DF80530ADF80600082269468B20FFF70C
:10FD18002FFD02B010BD2269154BB3FBF2F31A0C8C
:10FD28008DF800208DF802301A0A237D8DF8012005
:10FD38008DF803300422E8E7A3690093FAE76268C4
:10FD48000B4BB3FBF2F31A0C8DF800208DF8023040
:10FD58001A0A237B8DF80330637B8DF801208DF818
:10FD680004300522D1E700BF400F0108B71D00206D
:10FD78000000093D0048E8011FB52E4A0446D16835
:10FD88009068127C01AB03C31A702B4B20781B7848
:10FD9800834201D0FFF7F4FE2378032B26D8DFE84F
:10FDA80003F002383302637AF12B21D14FF6FF704A
:10FDB800FFF784FC48F20500FFF792FC02236288F3
:10FDC800A188ADF8061052BAE188ADF804208DF884
:10FDD8000B30227AA37A8DF80A20ADF808108DF836
:10FDE8000C30092201A98C20FFF7C2FC04B010BD19
:10FDF800F22BE4D141F60F50FFF760FC41F22100ED
:10FE0800FFF76EFC0623DAE7237B8DF80430012226
:10FE1800E8E7E389094A5BBAADF80430237C13703C
:10FE28008DF80630637C8DF80730638AADF80830AA
:10FE38000622D7E7400F0108B71D0020B51D002096
:10FE480007B502228DF804008DF805108F2001A94E
:10FE5800FFF78EFC03B05DF804FB000010B51346F5
:10FE6800EFF3108472B60A4601460348F6F7E6FC3B
:10FE780084F3108810BD00BF4C03002007B5012291
:10FE880001A91520FFF7EAFF9DF804004042401041
:10FE980003B05DF804FB000037B505460C460222A6
:10FEA80001A91320FFF7DAFF0A4B1B78012B0DD1AC
:10FEB800094B1B78012B09D140F20270FFF7A4FB14
:10FEC8009DF805302870237003B030BD9DF80400FC
:10FED800F6E700BFB71D0020B51D0020F7B50D4699
:10FEE800064600240DF10701284617468DF80740FD
:10FEF800FFF7D2FF2A78BA4207D89DF807003146A3
:10FF0800FFF726FC204603B0F0BD0120FBE7000008
:10FF180013B50322044601A91420FFF79FFF184BCD
:10FF28001A7822704AB1012A17D0142200212046DB
:10FF380000F0D2FA0F2323700DE09DF804302371EE
:10FF48009DF80530A2605B425B10A3719DF80630F6
:10FF58005B425B10637102B010BD9DF804305B42D8
:10FF68005B1023739DF9053002339B1063739DF872
:10FF780006305B425B10A373024B1B682361EAE700
:10FF8800B71D0020B01D0020012908B5034608460A
:10FF98000ED1012B07D10420FFF746FB0220BDE854
:10FFA8000840F4F735B8022B14BF08460320F6E7DB
:10FFB8000120F4E738B50446F4F74CF850B10228AC
:10FFC80014BF01250225284602222146FFF7EEFD2F
:10FFD800284638BD0F2CCCBF02250125F3E70A209F
:10FFE80070470000014B01201B681847B81D00200E
:08FFF800014B02201B681847B1
:020000040801F1
:10000000B81D0020014B40201B681847B81D002078
:1000100011B1012904D07047044B1B688020184798
:10002000024B4FF480701B68F9E700BFB81D002039
:10003000024B4FF400701B68184700BFB81D00202A
:10004000014B20201B681847B81D0020014B0420DD
:100050001B681847B81D0020014B08201B68184773
:10006000B81D0020014B10201B681847B81D002048
:10007000024B4FF480401B68184700BFB81D00209A
:1000800068B1084A002352F83310814203D902EBC9
:10009000C302107970470133162BF4D1FEE71F20FD
:1000A000704700BFF818010873B51D4B0193044653
:1000B00040F607000D46FFF7ABFAC0F3C103083363
:1000C0006B4413F8042C00F00703013302FA03F326
:1000D000144AB2FBF3F2B2FBF4F007281ED840003A
:1000E00003288CBF022304234FF4D66002FB03F4E1
:1000F000FFF78EFA060240F2B160FFF789FA06F4C4
:1001000070663043030544BF6FEA00506FEA105039
:1001100063094343DB112B6002B070BD0123E3E7A9
:1001200004080A0C0048E8014FF0FF3070474FF018
:10013000FF3070474FF0FF30704770470020704726
:100140000020704770474FF0FF3070474FF0FF308E
:10015000704770477047704770B5EFF3108672B6FE
:10016000144B5C8A1A8A944213D1C4F5806292B20D
:10017000904206D3844218D901229A7000221C8032
:100180005A825A8A0A800244C2F309025A82002023
:100190000DE006D9C4F58065ADB28542F1D8824242
:1001A000E9E7121B92B28242EBD84FF0FF3086F3A0
:1001B000108870BDBC210020EFF3108172B6034A95
:1001C000D38A0133D38281F310887047BC21002089
:1001D000EFF3108172B6034AD38A013BD38281F3D5
:1001E00010887047BC21002010B508481822002153
:1001F00000F076F906484FF48062002100F070F9B3
:10020000044B05481B68BDE810401847BC2100207E
:10021000BC1D0020E00F010889030108014B586054
:10022000704700BFBC210020014B1872704700BF0F
:10023000BC21002073B5EFF3108572B61C4CE08A28
:1002400000282FD1FFF7B8FF218A628A914227D078
:10025000A378012B12D1238820805B1A9BB2022144
:10026000A382A17063B9A3702382238A9A428BBFB1
:10027000D21AC3F58063A282A38201E0002BF4D0DE
:10028000238A0C4E1E4485F31088F2F707FC0A4BB4
:10029000A18ADB680193304602B0BDE87040184780
:1002A000FFF796FF85F31088002002B070BD00BFF5
:1002B000BC210020BC1D0020E00F010808B4F0B5EF
:1002C00086B00023ADF800302C4B0B9C1D7A854284
:1002D0004DD3D86881434DD15B681BB112B16946DB
:1002E00002A898470CAB22464FF4007124480193B2
:1002F00000F0F6FBFFF760FFBDF8003018440DF189
:10030000020180B2FFF728FF01302BD00022BDF898
:100310000030BDF802701B480DF1080C164691B272
:1003200017FA82F58B42ADB216D83B449BB20EB1A0
:10033000ADF80230BDF80250019B22464FF4007127
:10034000284400F0CDFBFFF743FFFFF773FF06B033
:10035000BDE8F04001B070471CF8011B4155013267
:100360000126DCE7FFF734FF6FF00200EFE76FF0E4
:100370000400ECE76FF00500E9E700BFBC210020B6
:10038000D4210020BC1D002013B5EFF3108472B6F9
:10039000204B9A78588A022A1DBF1A8A998A5218C5
:1003A000002214BFC2F309029A7090421A8228D028
:1003B000D98A012925D19978012913D119888A1A56
:1003C000022192B2997000219A82198062B99A70C2
:1003D0001A821A8A90428BBF801AC2F58062988274
:1003E0009A8201E00029F4D01A8A0B48104484F361
:1003F00010880A4A998AD368019302B0BDE8104078
:10040000184784F31088F2F74DFB02B0BDE81040A6
:10041000FFF7DEBEBC210020BC1D0020E00F01085C
:10042000024A00231360024A13607047D823002059
:10043000D423002010B5EFF3108472B641B1012926
:1004400003D1064A13680343136084F3108810BD78
:10045000024A136823EA0003F6E700BFD82300200E
:1004600010B5EFF3108472B641B1012903D1064AE9
:1004700013680343136084F3108810BD024A1368A5
:1004800023EA0003F6E700BFD423002038B5EFF3DA
:10049000108572B60A4B0B4C1B6833B12368984722
:1004A0006368984785F3108838BD074B1B681BB1FC
:1004B000A3689847E368F4E7236998476369F0E71E
:1004C000D82300206C0F0108D423002001380A44EF
:1004D000914200D1704711F8013B00F8013FF7E766
:1004E00000F02CBC10B5EFF3108472B6064A136806
:1004F00003431360054A52F83130034342F8313068
:1005000084F3108810BD00BF282400202024002080
:1005100070477047030C1B04C3B90004102310F08C
:100520007F4F02BF08330002DBB210F0704F08BFEC
:1005300000014FEA1070064A08BF0433125C08BF7E
:10054000DBB2C3F11F03981AC0B270470023E6E77D
:10055000A81901082DE9F84F384D394ED5F800801B
:10056000DFF8E0B0DFF8E0A0DFF8E090D6F800C0F8
:10057000374FDBF80010374CDAF80020D9F800309C
:1005800008EA00002860286800EA020E1EEA0C0F44
:1005900001D019421ED04FF0FF333B60FFF7B8FF88
:1005A000EFF3108472B63368DBF80020DAF800103D
:1005B0000B4029680B4205D1D9F80030134201D114
:1005C000F2F7FAF984F31088FFF7A3FFC5F800806B
:1005D000BDE8F88F236823680340134062681A421D
:1005E00004BF4FF0FF32626060681840FFF792FF6F
:1005F00062683860012303FA00F022EA00026260B8
:10060000EFF3108172B63A689340326822EA03022F
:100610003260226822EA0303236081F310880E4AC5
:100620003B6852F823309847D6F800C0DBF800103A
:10063000DAF80020D9F80030A5E700BF4401002017
:1006400028240020E023002048010020E42300208B
:10065000DC23002020240020E823002010B51146D0
:10066000EFF3108472B6FFF755FF034B43F82010E9
:1006700084F3108810BD00BFE823002082B082B050
:100680000DF1080C0CE90600BDF8042003930B449F
:10069000BDF810100A4491B212B2B2F57A7FA2BF2F
:1006A000A1F57A72013312B20360828002B002B007
:1006B000704782B082B00DF1080C0CE90600BDF85D
:1006C00004200393CB1ABDF81010521A91B212B243
:1006D000002ABEBF01F57A7203F1FF3312B2036044
:1006E000828002B002B0704730B585B0114D6B46C4
:1006F00083E8030000230293ADF80C3003A82B69B4
:100700009847009BBDF804400290181ABDF80C30C1
:10071000E41AA3B224B2002CBEBF03F57A731CB254
:1007200000F1FF302B689847AB682046984705B02A
:1007300030BD00BFA00F010873B5114E0023054660
:100740000093ADF8043001A833699847F36800902E
:100750009847736804469847009B1844BDF80430D6
:1007600023449AB21BB2B3F57A7FA2BF0130A2F53F
:100770007A731BB228602846AB8002B070BD00BF00
:10078000A00F010837B500230093ADF80430074BE4
:1007900004461B6901A898476D46009095E8030040
:1007A00084E80300204603B030BD00BFA00F01085D
:1007B00037B50F4D02AB03E90300EB6898476B6850
:1007C00004469847BDF80430009A1B1B99B21BB22F
:1007D000002BA2EB0002BEBF01F57A7102F1FF32DD
:1007E0000BB24FF47A7000FB023003B030BD00BF93
:1007F000A00F01082DE9F0414FF47A75B1FBF5F532
:10080000C5EB4513DFF83C8005EB8303A1EBC30385
:100810009CB2D8F80C3006469847D8F80430074602
:100820009847E31999B21BB2B3F57A7F2844A2BF67
:10083000A1F57A7301301BB23060B3803046BDE859
:10084000F08100BFA00F0108024B00221A60024B8A
:100850001B6818472C240020B40F0108F8B5044683
:10086000174608461E467CB173B1084B00255B6AEB
:1008700025609847069B60602581A572E66023612C
:10088000E77265612846F8BD0120FCE7B40F010856
:1008900010B5034CE3699847A36ABDE810401847B8
:1008A000B40F010870B5064DEB69064698476B6AB0
:1008B000044630469847AB6A201ABDE87040184796
:1008C000B40F0108054B1B680BB9184670478342EB
:1008D00001D05B69F8E70120704700BF2C2400209D
:1008E0002DE9F3410B4E336A044698470123B7695B
:1008F0002372D4F800800546B8472844804502D2C8
:10090000B84728442060B3682068019302B0BDE86E
:10091000F0411847B40F010870B520B3EFF310860B
:1009200072B6124D2B680122827253B100224272BC
:1009300098425C690ED102723CB120462C60FFF7F0
:10094000CFFF86F31088002070BD094BDB68984705
:100950002C60F6E71A465B69002BF2D09842F9D179
:1009600043695361EDE70120EEE700BF2C2400202E
:10097000B40F0108084B10B51A685369516911B9D1
:100980005061416110BD046819688C4202D91A4651
:100990005B69F3E71946F3E72C240020044A136847
:1009A0000BB10021197243611060FFF799BF00BFBE
:1009B0002C2400202DE9F041044600282DD0FFF71B
:1009C00081FF50BB657A45BBEFF3108872B6144EB9
:1009D0006768336A984787422CBF27602060114FB1
:1009E000A5724FF4807323813B684BB933699847F4
:1009F0002046FFF7D3FF88F310882846BDE8F08132
:100A0000B3699847236818443B6820601B68984284
:100A10002046EED3FFF7AEFFEDE70125EDE700BF7F
:100A2000B40F01082C24002010B5044608467CB100
:100A3000084B5B6A984760602046FFF743FF40B170
:100A40002046FFF769FF2046BDE81040FFF7B2BF20
:100A5000012010BDB40F01082DE9F041EFF310871C
:100A600072B61D4E1D4D7369984733690446984709
:100A70002B684BB94FF000082B688BB9286828BB4E
:100A800087F31088BDE8F081011B241A1A688A4296
:100A90008CBF121900221A605B69002BF6D1E9E7BE
:100AA0001C681CB1B36998478442E7D22C6863691B
:100AB0002B60A4F80880D4E9033098476389B3F524
:100AC000807FD9D12046FFF775FFD5E7037A002B49
:100AD000D6D1FFF705FFD3E7B40F01082C2400207F
:100AE0002DE9F04F97B000298046039140F30E8125
:100AF0009A46044603991378A4EB0800013923B9F8
:100B00000023237017B0BDE8F08F8842F8DA252B58
:100B100004D004F8013B1646721CEBE792F801C0C2
:100B2000ACF13003D3F1000E4EEB030EACF1300309
:100B3000092B02F1010629D8324600254FF00A0997
:100B4000164612F8013BA3F13000092819D9337871
:100B5000692B00F09C801CD8632B28D0642B00F0FC
:100B60009680582B5BD0252B19D13378002B00F0C1
:100B7000928004F8013BA4EB08038B4280F2898049
:100B8000CAE709FB0533A3F13005D9E74FF0FF357C
:100B9000DDE7752B7DD0782B43D0732B1ED025231A
:100BA00004F8013BA4EB08038B4272DADDE7002D69
:100BB00005F1FF39D8BF4FF000094A4620462021F1
:100BC00000F0BCF85346A144002D53F8042B89F8DB
:100BD0000020D8BF01252C449A469DE74C4B5AF87B
:100BE000047B002F08BF1F463846F0F7E9FBA5EB52
:100BF000000B8542B8BF4FF0000B5A4681462021BA
:100C0000204600F09BF8A34400234B4502DB0BEB8E
:100C1000090481E7FA5C0BF803200133F5E74EF095
:100C2000400E1020DFF8EC903B4F1EF0400F08BF45
:100C30004F465346BCF1300F0197A4EB08020CBF9E
:100C4000302720271EF0020FA1EB0202029753F873
:100C5000041B22D0002920DA4942013D4FF02D0E1D
:100C600005AF009700278946DDF804A0B1FBF0F13D
:100C700000FB119B48451AF80BB0DDF800A00AF8FC
:100C800001BB07F10107CDF800A0ECD90EE04EF052
:100C9000020E0A20C6E7013E6DE711B14FF0000ECB
:100CA000DEE730208DF814008E460127BCF1300FAE
:100CB000A5EB070504D02020002D05F1FF3509DC48
:100CC000BEF1000F04D02D21013A04F8011B83D09E
:100CD00025440AE0013A04F8010BEDD17CE70299C2
:100CE00004F8011B013A3FF477AF291B0029F6DC19
:100CF00005A9394422442744A7423FF46DAF11F8B7
:100D0000010D04F8010B9442F6D165E70020F9E6E5
:100D1000B8190108BF190108E419010810B5013913
:100D20000244904201D1002005E0037811F8014F00
:100D3000A34201D0181B10BD0130F2E70244034664
:100D4000934200D1704703F8011BF9E770B50D4DD0
:100D50000D4C641BA4100026A64209D10B4D0C4C6F
:100D600000F0B2F8641BA4100026A64205D170BDA5
:100D700055F8043B98470136EEE755F8043B984791
:100D80000136F2E7EC1A0108EC1A0108EC1A010826
:100D9000F01A010800F003B8002200F00EB80A446F
:100DA000914200F1FF3300D1704710B511F8014BAB
:100DB00003F8014F9142F9D110BD13460A46194676
:100DC000FFF7BCBF00000000C1F30A522DE9F84351
:100DD000A2F2FF36132E0B4607460C46054632DCC0
:100DE000002E14DA34A3D3E90023F0F7F7FA002237
:100DF0000023F0F727FD38B1002C56DA24F0004428
:100E0000254355D02E4C002523462F4625E02D4A5C
:100E100042FA06F801EA080202431ED026A3D3E9EB
:100E20000023F0F7DBFA00220023F0F70BFD002887
:100E3000EAD0002CBEBF4FF480133341E41824EAFB
:100E400008040025E0E7332E0BDDB6F5806F04D1F2
:100E50000246F0F7C3FA07460B4638461946BDE886
:100E6000F883A2F213424FF0FF3828FA02F810EA92
:100E7000080FF2D010A3D3E90023F0F7AFFA002255
:100E80000023F0F7DFFC0028BED0002C0ADA142E75
:100E900001D1013406E0C6F134060123B3401D44FC
:100EA000AF42F6D825EA0805AEE700252C46ABE7A9
:100EB0004FF00044A8E700BF9C7500883CE4377EF3
:100EC0000000F0BFFFFF0F00F8B500BFF8BC08BC82
:100ED0009E467047F8B500BFF8BC08BC9E467047F8
:100EE00000000000010000000200000000000000FF
:100EF0008813000010270000204E0000307500000D
:100F0000409C000050C3000060EA0000C0D4010013
:100F100080A903000053070000EA06370000000024
:100F20005000000040F709370000000050000000AA
:100F3000C194C10000000000B227000000000000C2
:100F400000000000000000000000000000000000A1
:100F500000000000B5010008F1010008540F01086D
:100F6000FC7F003F00350113C412000887270008EA
:100F7000692700084D2700086D2700084927000849
:100F8000992700085975336E3148344F3152354E28
:100F9000395332543653256473253033643A000094
:100FA000692C0008092D0008792C0008152D00086F
:100FB000D92C0008212D000800000000892C000811
:100FC000412C00080D2C0008C52B00081D2C000822
:100FD000312C0008D12B0008D52B0008E92B000884
:100FE000892F0008B12F0008352F0008212F000895
:100FF00052464143005056585858002159756E4882
:101000006F726E20535453205265766976652100C5
:1010100001000000030000000500000001000000C6
:1010200001000000060000000A000000200000008F
:101030000200000004000000080000001000000092
:1010400040000000800000000001000000020000DD
:101050000000000000000000000000000000000090
:101060000100000002000000030000000400000076
:10107000A0860100400D0300801A060000350C0018
:1010800040420F0080841E0000093D0000127A00DB
:101090000024F40000366E010048E801006CDC0218
:1010A0000000000000000000000000000000000040
:1010B0000402080010101004101010021010100884
:1010C000010002000400060008000A000C001000E5
:1010D0002000400080000001080402040801010112
:1010E00001010103070100006572726F723A20521C
:1010F0006567696F6E206973206E6F742064656622
:10110000696E656420696E20746865204D573A20C9
:10111000736574206C6F726177616E5F636F6E666A
:101120002E68206163636F7264696E676C790D0A63
:10113000004D414320727854696D654F75740D0AF6
:10114000004D414320747854696D654F75740D0AE4
:10115000004D4143207278446F6E650D0A004D4189
:1011600043207478446F6E650D0A00080A0C0D0E5A
:1011700010121415181A1B1D1E2124030502050147
:10118000060202050000060000010504040000003C
:1011900048E8010048E8010048E8010048E801008B
:1011A00048E8010048E8010090D00300000000007A
:1011B000030000000201000C0B0A090807073200B7
:1011C0000000000000010201000000000002030214
:1011D00001000000000304030201000000040504F4
:1011E00003020100000506050403020100060706CC
:1011F00005040302010707070605040302070702A7
:1012000002020202020202020202020202020302BD
:1012100002020202020304030202020202040504A3
:101220000302020202050605040302020206070683
:101230000504030202070707060504030207073334
:10124000337373F2F2F2F200000B357DF2F2F233F7
:10125000337373DEDEDEDE52585F2573206F6E203F
:101260006672657120256420487A2061742044529A
:101270002025640D0A005258206F6E206672657139
:1012800020256420487A2061742044522025640D72
:101290000A005458206F6E20667265712025642004
:1012A000487A2061742044522025640D0A003100E0
:1012B00032004D756C74695F43004D756C74695FE5
:1012C00050000000AE120108B0120108F30F01082F
:1012D000B2120108C0120108BA120108C6F8EEF6EF
:1012E000FFD6DE916002CE56E7B54DEC8F1F89FA2E
:1012F000EFB28EFB41B35F452353E49B75E13D4C58
:101300006C7EF5836851D1F9E2AB622A0895469D5F
:1013100030370A2F0E241BDFCD4E7FEA121D5834C2
:1013200036DCB45BA476B77D52DD5E13A6B900C18E
:1013300040E379B6D48D67729498B085BBC54FED04
:10134000869A66118AE904FEA078254BA25D800585
:101350003F2170F16377AF4220E5FDBF811826C3BE
:10136000BE35882E9355FC7AC8BA32E6C0199EA3C2
:1013700044543B0B8CC76B28A7BC16ADDB647414BC
:10138000920C48B89FBD43C43931D3F2D58B6EDA85
:1013900001B19C49D8ACF3CFCAF447106FF04A5C56
:1013A00038577397CBA1E83E96610D0FE07C71CC66
:1013B0009006F71CC26AAE6917993A27D9EB2B221F
:1013C000D2A907332D3C15C987AA50A50359091A7C
:1013D00065D784D082295A1E7BA86D2CA584998D4F
:1013E0000DBDB1545003A97D1962E69A459D408711
:1013F00015EBC90BEC67FDEABFF7965BC21CAE6A42
:101400005A41024F5CF434089373533F0C52655EAB
:1014100028A10FB509369B3D2669CD9F1B9E742ED2
:101420002DB2EEFBF64D61CE7B3E7197F568002C38
:10143000601FC8EDBE46D94BDED4E84A6B2AE516DC
:10144000C5D75594CF100681F044BAE3F3FEC08AA5
:10145000ADBC4804DFC17563301A0E6D4C14352FD6
:10146000E1A2CC3957F28247ACE72B95A098D17F07
:10147000667EAB83CA29D33C79E21D763B564E1E6D
:10148000DB0A6CE45D6EEFA6A8A4378B324359B734
:101490008C64D2E0B4FA0725AF8EE918D5886F7254
:1014A00024F1C751237C9C21DDDC86859042C4AAAF
:1014B000D8050112A35FF9D0915827B93813B33377
:1014C000BB7089A7B622922049FF787A8FF88017DF
:1014D000DA31C6B8C3B07711CBFCD63A637C777BE0
:1014E000F26B6FC53001672BFED7AB76CA82C97D20
:1014F000FA5947F0ADD4A2AF9CA472C0B7FD9326B1
:10150000363FF7CC34A5E5F171D8311504C723C3B4
:101510001896059A071280E2EB27B27509832C1AF8
:101520001B6E5AA0523BD6B329E32F8453D100ED52
:1015300020FCB15B6ACBBE394A4C58CFD0EFAAFB36
:10154000434D338545F9027F503C9FA851A3408FFE
:10155000929D38F5BCB6DA2110FFF3D2CD0C13EC16
:101560005F974417C4A77E3D645D197360814FDCAB
:10157000222A908846EEB814DE5E0BDBE0323A0A8F
:101580004906245CC2D3AC629195E479E7C8376D13
:101590008DD54EA96C56F4EA657AAE08BA78252E38
:1015A0001CA6B4C6E8DD741F4BBD8B8A703EB566C1
:1015B0004803F60E613557B986C11D9EE1F89811B2
:1015C00069D98E949B1E87E9CE5528DF8CA1890DA1
:1015D000BFE6426841992D0FB054BB162323232345
:1015E000232320257320253032583A253032583AAB
:1015F000253032583A253032583A253032583A257B
:101600003032583A253032583A253032583A25305F
:1016100032583A253032583A253032583A2530324D
:10162000583A253032583A253032583A2530325817
:101630003A253032580D0A00232323232323204444
:1016400065764555493A2020202020202530325803
:101650003A253032583A253032583A253032583A05
:10166000253032583A253032583A253032583A250A
:101670003032580D0A002323232323232041707086
:101680004555493A202020202020253032583A253F
:101690003032583A253032583A253032583A2530CF
:1016A00032583A253032583A253032583A253032BD
:1016B000580D0A0023232323232320446576416405
:1016C00064723A2020202020253032583A253032CA
:1016D000583A253032583A253032580D0A004170B8
:1016E000704B65793A2020202020004E776B4B65A7
:1016F000793A2020202020004E776B534B65793AB1
:101700002020202000417070534B65793A20202022
:1017100020004442496E744B65793A202020004DE8
:1017200043526F6F744B65793A2020004D434B450F
:101730004B65793A20202020004D43417070534B77
:1017400065795F303A004D434E776B534B65795F57
:10175000303A0000000000004150505FDE160108E2
:10176000010000004E574B5FEB1601080800000017
:101770004E574B53F81601080900000041505053D2
:10178000051701080A0000004442495F12170108CA
:101790000B0000004D4352541F1701080C000000BD
:1017A0004D434B452C1701080D0000004D434B30B5
:1017B000391701080E0000004D4153303917010858
:1017C0000F0000004D4E5330461701081000000076
:1017D0005A45524F13180108526164696F53656E80
:1017E00064204F76657273697A650D0A004952511B
:1017F0005F52585F54585F54494D454F55540D0A38
:1018000000505245204F4B0D0A0053594E43204F74
:101810004B0D0A00484452204F4B0D0A00484452D9
:10182000204B4F0D0A004952515F4352435F4552CE
:10183000524F520D0A00040506000000841E0000ED
:10184000093D0000127A000024F4000048E801007D
:1018500090D0030020A1070000000000B128000084
:1018600061510000C3A20000020100038DE50008E1
:1018700051E4000889E60008CDE40008B5EF00084F
:1018800075E50008E1EC000859EB000831E30008B9
:10189000F1F1000831F0000861E5000849E40008B2
:1018A000F9E40008D1E4000889E400087FE40008B6
:1018B00081E300087DE300087BE4000877E400088A
:1018C00021E600084DE600086DE400080DF300086D
:1018D000E1E30008A9E30008DDF2000885E3000861
:1018E00051E90008D5E60008290101082F01010887
:1018F00075E3000879E30008C01200001F00000033
:10190000A816000017000000841C00000F00000053
:10191000E42500001E000000B42D000016000000A9
:10192000083900000E0000002C4C00001D000000D3
:10193000685B000015000000747200000D000000DC
:10194000589800001C00000034B70000140000008C
:10195000E8E400000C000000783101001B000000EA
:10196000686E01001300000034CA01000B00000083
:10197000286202001A00000040DB02001200000092
:101980003C9303000A000000C0C2040019000000DC
:1019900060B30500110000003820070009000000B6
:1019A00020A1070000000000040302020101010160
:1019B00000000000000000003C4E554C4C3E003042
:1019C000313233343536373839616263646566677E
:1019D00068696A6B6C6D6E6F70717273747576770F
:1019E00078797A00303132333435363738394142FC
:1019F000434445464748494A4B4C4D4E4F5051523F
:0C1A0000535455565758595A0000000026
:101A0C0000000000000000000000000000000000CA
:101A1C000000000000000000002B7E151628AED23E
:101A2C00A6ABF7158809CF4F3C012B7E151628AEB7
:101A3C00D2A6ABF7158809CF4F3C082B7E1516287C
:101A4C00AED2A6ABF7158809CF4F3C092B7E1516E5
:101A5C0028AED2A6ABF7158809CF4F3C0A00000080
:101A6C00000000000000000000000000000B00005F
:101A7C0000000000000000000000000000000C004E
:101A8C000000000000000000000000000000000D3D
:101A9C00000000000000000000000000000000003A
:101AAC000E0000000000000000000000000000001C
:101ABC00000F00000000000000000000000000000B
:101ACC0000001000000000000000000000000000FA
:081ADC00000000000000000002
:081AE4005C00FF7F010000001F
:041AEC005D01000890
:041AF00039010008B0
:101AF400020000000000000072040020C0D40100B5
:101B0400BD290008ED290008052A0008712A0008EB
:101B1400C53200089D320008ED310008EB3400089E
:101B24000000000059320008C1310008DD3E000801
:101B3400A7310008A5310008F1340008F531000888
:101B4400A9310008B5310008B534000800000100CF
:101B5400000000000000000000000000040000007D
:101B6400401F000010270000005601013053054DAE
:101B74000400002008190F28040A413F00050A0147
:101B84000000050203FFFFFFFFFFFFFFFFFFFF0F42
:101B9400010300020000000000000000000000003B
:101BA400000000000000000000093D0010000000DB
:101BB400B00700200000FF0000000000000000004B
:101BC400B00700200000000000000000FF0000003B
:101BD40000000000B007002000000000000000002A
:101BE400000000000000000000000000E000000011
